:020000040800F2
:1000000000060020E1010008E3010008E301000808
:10001000E3010008E3010008E3010008E301000830
:10002000E3010008E3010008E301000825300008AF
:10003000E3010008E3010008E3010008E301000810
:10004000E3010008E3010008E3010008E301000800
:10005000E3010008E3010008E3010008E3010008F0
:10006000E3010008E3010008E3010008E3010008E0
:10007000E3010008E3010008E3010008E3010008D0
:10008000E3010008E3010008E3010008E3010008C0
:10009000E3010008E3010008E3010008E3010008B0
:1000A000E3010008E3010008E3010008E3010008A0
:1000B000CD320008E3010008E3010008E301000875
:1000C000E3010008E3010008E3010008E301000880
:1000D000E3010008E3010008E3010008E301000870
:1000E000E3010008E3010008E3010008E301000860
:1000F000E3010008E3010008E3010008E301000850
:10010000E3010008E3010008E3010008E30100083F
:10011000E3010008E3010008E3010008E30100082F
:10012000E3010008E3010008E3010008E30100081F
:10013000E3010008E3010008E3010008E30100080F
:10014000E3010008E3010008E3010008D9270008E3
:10015000E3010008E3010008E3010008E3010008EF
:10016000E3010008E3010008E3010008E3010008DF
:10017000E3010008E3010008E3010008E3010008CF
:10018000E3010008E3010008E3010008E3010008BF
:10019000E3010008E3010008E3010008E3010008AF
:1001A000E3010008E3010008E3010008E30100089F
:1001B000E3010008E3010008E3010008E30100088F
:1001C000E3010008E3010008E3010008E30100087F
:1001D000E3010008E3010008E3010008E30100086F
:1001E00002E000F000F8FEE772B6374880F30888B6
:1001F000364880F3098836483649086040F20000E6
:10020000CCF200004EF63471CEF200010860BFF36C
:100210004F8FBFF36F8F40F20000C0F2F0004EF638
:100220008851CEF200010860BFF34F8FBFF36F8F8C
:100230004FF00000E1EE100A4EF63C71CEF20001E4
:100240000860062080F31488BFF36F8F01F08CFFE5
:1002500002F086FE4FF055301F491B4A91423CBFC9
:1002600041F8040BFAE71D49184A91423CBF41F896
:10027000040BFAE71A491B4A1B4B9A423EBF51F83E
:10028000040B42F8040BF8E700201849184A914281
:100290003CBF41F8040BFAE701F06AFF02F0B4FE3C
:1002A000144C154DAC4203DA54F8041B8847F9E7A7
:1002B00000F0A0F8114C124DAC4203DA54F8041BC4
:1002C0008847F9E701F052BF000600200022002015
:1002D0000000000808ED00E00000002000060020FB
:1002E000303600080022002040220020402200205A
:1002F000E02D0020E0010008E0010008E001000816
:10030000E00100082DE9F04F2DED108AC1F80CD066
:10031000C3689D46BDEC108ABDE8F08F002383F3CF
:1003200011882846A047002001F0CAFAFEE701F034
:1003300053FA00DFFEE7000080EA0102844612F073
:10034000030F4FD111F0030F32D14DF8044D11F0CE
:10035000040F51F8043B0BD0A3F101329A4312F081
:10036000803F04BF4CF8043B51F8043B16D100BF5A
:1003700051F8044BA3F101329A4312F0803FA4F1EB
:1003800001320BD14CF8043BA24312F0803F04BF72
:1003900051F8043B4CF8044BEAD023460CF8013BDF
:1003A00013F0FF0F4FEA3323F8D15DF8044B704789
:1003B00011F0010F06D011F8012B0CF8012B002AC7
:1003C00008BF704711F0020FBFD031F8022B12F0B6
:1003D000FF0F16BF2CF8022B8CF8002012F47F4F71
:1003E000B3D1704711F8012B0CF8012B002AF9D179
:1003F000704700BF38B500F0A5FB01F081FE05464F
:1004000001F0A4FE0446C8B90E4B9D4218D001333A
:100410009D4218BF044641F2883504BF01240025DF
:10042000002001F077FE0CB100F072F800F0EAFC59
:10043000284600F0BDF800F06BF8F9E70025EFE77B
:100440000546EDE7010007B008B500F04DFBA0F14F
:1004500020035842584108BD07B5042101900DEB17
:10046000010000F05FFB03B05DF804FB38B53023FA
:1004700083F31188174803680BB101F0EDFA164AAF
:10048000144800234FF47A7101F0DCFA002383F35F
:100490001188124C236813B12368013B2360636801
:1004A00013B16368013B63600D4D2B7833B963680A
:1004B0007BB9022000F010FC322363602B78032B01
:1004C00007D163682BB9022000F006FC4FF47A7361
:1004D000636038BD402200206D04000860230020C6
:1004E00058220020084B187003280CD8DFE800F0D1
:1004F00008050208022000F0E5BB022000F0D8BB8E
:10050000024B00225A6070475822002060230020CE
:10051000234B244A10B51C46196801313FD00433DF
:100520009342F9D16268A24239D31F4B9B6803F111
:10053000006303F540439A4231D2002000F01CFBD7
:100540000220FFF7CFFF194B1A6C00221A64196EB4
:100550001A66196E596C5A64596E5A665A6E5A69FF
:1005600042F080025A615A6922F080025A615A6947
:100570001A6942F000521A611A6922F000521A6197
:100580001B6972B64FF0E0233021C3F8084DD4E95F
:10059000003281F311889D4683F30888104710BD0F
:1005A00000C0000820C000080022002000380240DF
:1005B0002DE9F04F93B0DFF8049302902022FF2141
:1005C0000AA8D9F8085000F0C7FBB34A1378A3B9BA
:1005D000B248012103601170302383F3118803684E
:1005E0000BB101F039FAAE4AAC4800234FF47A71EE
:1005F00001F028FA002383F31188029B13B1A94B61
:10060000029A1A60A84A029C1378032B1EBF00238B
:100610001370A44A4FF0000B18BF5360CDF804B01C
:100620005E46DA46012000F04DFB24B19D4B1B686D
:10063000002B00F0F981002000F056FA071EF4DBD1
:10064000012000F035FBA7F121001628EAD801A30C
:1006500053F820F0B1060008CD0600085B0700083B
:10066000250600082506000825060008DF07000803
:100670009F090008C10800081D0900084309000877
:1006800069090008250600087B09000825060008FE
:10069000E709000839070008250600082F0A0008A6
:1006A000BD06000839070008250600081D090008D6
:1006B0000220FFF7C9FE002840F0E381029B7B483F
:1006C000BBF1000F08BF1C46022140E04FF47A70D6
:1006D00000F00AFA071EF1DB0220FFF7B5FE002842
:1006E000ECD0013F052F00F2CE81DFE807F00307D1
:1006F0000A0D10330520FFF7AFFE14E0D9F8000013
:10070000F9E7D9F80400F6E7D9F80800F3E74FF065
:100710001C08404600F032FA08F10408FFF79CFE7E
:10072000B8F12C0FF5D1019B012000FA07F71F4308
:10073000FBB201934FF0000A00F05AFB2EB1019B6F
:1007400003F00B030B2B08BF00245948022100F0D3
:10075000E9F967E7D9F80C00CDE7002EAED0019B90
:1007600003F00B030B2BA9D10220FFF76DFE074608
:100770000028A3D0012000F0FFF90220FFF7B2FE0D
:1007800000261FFA86F8404600F006FA044670B1CB
:100790000021404600F010FA01360028F1D1BB4696
:1007A00004464448022100F0BDF93E463AE70120E4
:1007B000FFF798FE2546D9F80830AB4207D92846FE
:1007C00000F0DCF9013040F061810435F3E7364B8D
:1007D00000251D70334BBB465D603E46ACE7002EE6
:1007E0003FF46CAF019B03F00B030B2B7FF466AF60
:1007F0000220FFF777FE322000F076F9B0F1000812
:10080000FFF65CAF18F003077FF458AFD9F8082063
:1008100008EB050393423FF651AFB8F5807F3FF7F1
:100820004DAF254B0393B8450BDD4FF47A7000F0C4
:100830005BF90028FFF642AF039B013703F8010B79
:10084000F0E7C820FFF700FE074600283FF436AF68
:100850001F2D11D8C5F1200242450AAB25F0030037
:1008600028BF424614490392184400F04FFA039AF5
:100870001148FF2100F070FA4FEAA8030E490393D4
:10088000C8F38702284600F06FFA0646002888D091
:10089000039B05EB83054FE75C23002040220020EB
:1008A0006D04000860230020582200201033000847
:1008B000083300080C3300085C22002000220020CE
:1008C0000220FFF7C1FD00283FF4F8AE00F0A0F9C8
:1008D00000283FF4F3AE0027B846D9F80830BB42F1
:1008E00018D91F2F11D80A9B01330ED027F003030C
:1008F00048336B4453F8203C05934046042205A935
:1009000000F0AAFA04378046E7E7384600F036F9E7
:100910000590F2E74046FFF79FFD0DE700236421B5
:1009200005A8059300F0F4F800287FF4C7AE022074
:10093000FFF78AFD00283FF4C1AE059800F050F99A
:10094000E9E70023642105A8059300F0E1F80028F9
:100950007FF4B4AE0220FFF777FD00283FF4AEAE7F
:10096000059800F04DF9D6E70220FFF76DFD00284D
:100970003FF4A4AE00F05CF9CDE70220FFF764FD80
:1009800000283FF49BAE05A9142000F057F903900E
:10099000FFF762FD039905A800F0C4F8CCE6322009
:1009A00000F0A2F8071EFFF689AEBB077FF486AE03
:1009B000D9F8082007EB0A0393423FF67FAE0220E6
:1009C000FFF742FD00283FF479AE27F003075744B4
:1009D000BA453FF4B1AE504600F0D0F8FFF73CFD09
:1009E0000AF1040AF4E74FF47A70FFF72DFD0028AE
:1009F0003FF464AE00F00CF9002849D00A9B0133A3
:100A00000BD008220AA9002000F0AEF900283FD040
:100A10002022FF210AA800F09FF91E48022100F0C1
:100A200081F81D4800F052FF13B0BDE8F08F002E92
:100A30003FF444AE019B03F00B030B2B7FF43EAE5F
:100A40000023642105A8059300F062F807460028FA
:100A50007FF434AE0220FFF7F7FC804600283FF415
:100A60002DAE02210B4800F05DF841F2883000F015
:100A70002DFF059800F0EEF9464600F0B9F93C4626
:100A8000D0E5064658E64FF0000A17E6BB4688E672
:100A9000374686E608330008A086010070B50F4B84
:100AA0001B780133DBB2012B0C4611D80C4D2968A1
:100AB0004FF47A730E6AA2FB03320146224628469F
:100AC000B047844204D1074B00221A70012070BD48
:100AD0004FF4FA7000F0FAFE0020F8E71022002030
:100AE000082600209423002007B500230246012198
:100AF0000DF107008DF80730FFF7D0FF20B19DF80A
:100B0000070003B05DF804FB4FF0FF30F9E7000089
:100B10000A4608B50421FFF7C1FF80F00100C0B20A
:100B2000404208BD30B4054C2368DD69044B0A46D9
:100B3000AC460146204630BC604700BF0826002076
:100B4000A086010070B501F0E1F9094E094D308031
:100B5000002428683388834208D901F0D1F92B6832
:100B600004440133B4F5404F2B60F2D370BD00BF95
:100B7000962300206823002001F076BA00F100607F
:100B800000F540400068704700F10060920000F5F9
:100B9000404001F001BA0000054B1A68054B1B8864
:100BA0009B1A834202D9104401F0AAB90020704771
:100BB000682300209623002038B5084D044629B14B
:100BC00028682044BDE8384001F0BAB928682044BC
:100BD00001F09EF90028F3D038BD00BF6823002043
:100BE00010F003030AD1B0F5047F05D200F10050E4
:100BF000A0F51040D0F80038184670470023FBE7F6
:100C000000F10050A0F51040D0F8100A7047000025
:100C1000064991F8243033B10023086A81F8243062
:100C20000822FFF7B1BF0120704700BF6C230020EE
:100C3000014B1868704700BF002004E070B5194BE5
:100C40001D68194B0138C5F30B0408442D0C042210
:100C50001E88A6420BD15C680A46013C82421346BC
:100C60000FD214F9016F4EB102F8016BF6E7013AA9
:100C700003F10803ECD181420B4602D22C2203F887
:100C8000012B0A4A05241688AE4204D1984284BF3B
:100C9000967803F8016B013C02F10402F3D1581A73
:100CA00070BD00BF002004E054330008403300084A
:100CB000022802BF024B4FF000529A61704700BFFA
:100CC00000080240022802BF024B4FF400529A6112
:100CD000704700BF00080240022801BF024A536962
:100CE00083F40053536170470008024070B5044616
:100CF0004FF47A764CB1412C254628BF412506FB9E
:100D000005F000F0E3FD641BF4E770BD10B50023AF
:100D1000934203D0CC5CC4540133F9E710BD00000A
:100D200010B5013810F9013F3BB191F900409C42E8
:100D300003D11AB10131013AF4E71AB191F9002057
:100D4000981A10BD1046FCE703460246D01A12F965
:100D5000011B0029FAD1704702440346934202D096
:100D600003F8011BFAE770472DE9F8431F4D1446BD
:100D700095F824200746884652BBDFF870909CB354
:100D800095F824302BB92022FF2148462F62FFF727
:100D9000E3FF95F82400C0F10802A24228BF2246D2
:100DA000D6B24146920005EB8000FFF7AFFF95F801
:100DB0002430A41B1E44F6B2082E17449044E4B21B
:100DC00085F82460DBD1FFF723FF0028D7D108E0A6
:100DD0002B6A03EB82038342CFD0FFF719FF002871
:100DE000CBD10020BDE8F8830120FBE76C23002075
:100DF000024B1A78024B1A70704700BF94230020F0
:100E00001022002010B5104C104800F0B5F8214613
:100E10000E4800F0DDF82468626DD2F8043843F023
:100E20000203C2F804384FF47A70FFF75FFF0849F5
:100E3000204600F0D3F9626DD2F8043823F00203A3
:100E4000C2F8043810BD00BF203400080826002076
:100E5000283400087047000030B5094D0A4491421B
:100E60000DD011F8013B5840082340F30004013B2A
:100E70002C4013F0FF0384EA5000F6D1EFE730BDB9
:100E80002083B8ED026843681143016003B118473D
:100E90007047000013B5446BD4F894341A68117885
:100EA000042915D1217C022912D119791289012333
:100EB0008B4013420CD101A904F14C0001F00CFF4E
:100EC000D4F89444019B21790246206800F0D0F9BF
:100ED00002B010BD143001F08FBE00004FF0FF33A0
:100EE000143001F089BE00004C3001F061BF0000F9
:100EF0004FF0FF334C3001F05BBF0000143001F0C5
:100F00005DBE00004FF0FF31143001F057BE00000D
:100F10004C3001F02DBF00004FF0FF324C3001F09B
:100F200027BF00000020704710B5D0F894341A682D
:100F300011780429044617D1017C022914D159796A
:100F4000528901238B4013420ED1143001F0F0FD81
:100F5000024648B1D4F894444FF480736179206814
:100F6000BDE8104000F072B910BD0000406BFFF703
:100F7000DBBF0000704700007FB5124B0360002309
:100F80004360C0E90233012502260F4B0574044675
:100F90000290019300F18402294600964FF4807379
:100FA000143001F0A1FD094B0294CDE9006304F572
:100FB00023724FF48073294604F14C0001F068FE5F
:100FC00004B070BD743300086D0F0008950E000862
:100FD0000B68302282F311880A7903EB8202906158
:100FE0004A79093243F822008A7912B103EB82036D
:100FF00098610223C0F894140374002080F31188D0
:101000007047000038B5037F044613B190F85430A0
:10101000ABB9201D01250221FFF734FF04F11400B4
:1010200025776FF0010100F079FC84F8545004F149
:101030004C006FF00101BDE8384000F06FBC38BDD6
:1010400010B5012104460430FFF71CFF002323776D
:1010500084F8543010BD000038B504460025143023
:1010600001F05AFD04F14C00257701F029FE201D06
:1010700084F854500121FFF705FF2046BDE83840B1
:10108000FFF752BF90F8443003F06003202B07D1E4
:1010900090F84520212A4FF0000303D81F2A06D8D4
:1010A00000207047222AFBD1C0E90E3303E0034A37
:1010B00082630722C263036401207047112200206B
:1010C00037B5D0F894341A681178042904461AD137
:1010D000017C022917D11979128901238B4013420F
:1010E00011D100F14C05284601F0AAFE58B101A922
:1010F000284601F0F1FDD4F89444019B2179024681
:10110000206800F0B5F803B030BD0000F0B500EB8A
:10111000810385B09E6904460D46FEB1302383F3FA
:10112000118804EB8507301D0821FFF7ABFEFB6833
:101130005B691B6806F14C001BB1019001F0DAFD00
:10114000019803A901F0C8FD024648B1039B294656
:10115000204600F08DF8002383F3118805B0F0BD20
:10116000FB685A691268002AF5D01B8A013B1340BC
:10117000F1D104F14402EAE7093138B550F82140D1
:10118000DCB1302383F31188D4F8942413685279A6
:1011900003EB8203DB689B695D6845B1042160183D
:1011A000FFF770FE294604F1140001F0CBFC204645
:1011B000FFF7BAFE002383F3118838BD70470000A3
:1011C00001F02AB8012303700023C0E90133C36191
:1011D00083620362C36243620363704738B50446A7
:1011E000302383F311880025C0E90355C0E9055574
:1011F000416001F021F80223237085F3118828460D
:1012000038BD000070B500EB810305465069DA6017
:101210000E46144618B110220021FFF79DFDA0696B
:1012200018B110220021FFF797FD31462846BDE88E
:10123000704001F0CBB80000826802F001128260B9
:101240000022C0E90422826101F04CB9F0B400EB45
:1012500081044789E4680125A4698D403D434581A7
:1012600023600023A2606360F0BC01F067B9000056
:10127000F0B400EB81040789E468012564698D40BE
:101280003D43058123600023A2606360F0BC01F050
:10129000E1B9000070B50223002504460370C0E9DF
:1012A0000255C0E90455C564856180F8345001F0E9
:1012B00029F863681B6823B129462046BDE87040C1
:1012C000184770BD0378052B10B504460AD080F886
:1012D00050300523037043681B680BB10421984705
:1012E0000023A36010BD00000178052906D190F805
:1012F0005020436802701B6803B118477047000014
:1013000070B590F83430044613B1002380F83430BF
:1013100004F14402204601F007F963689B68B3B901
:1013200094F8443013F0600535D00021204601F0D8
:10133000A7FB0021204601F099FB63681B6813B1ED
:10134000062120469847062384F8343070BD204695
:1013500098470028E4D0B4F84A30E26B9A4288BF3C
:10136000E36394F94430E56B002B4FF0300380F2D7
:101370000381002D00F0F280092284F8342083F3E9
:1013800011880021D4E90E232046FFF771FF0023C6
:1013900083F31188DAE794F8452003F07F0343EAEA
:1013A000022340F20232934200F0C58021D8B3F507
:1013B000807F48D00DD8012B3FD0022B00F09380C6
:1013C000002BB2D104F14C02A2630222E263236437
:1013D000C1E7B3F5817F00F09B80B3F5407FA4D1D6
:1013E00094F84630012BA0D1B4F84C3043F00203FE
:1013F00032E0B3F5006F4DD017D8B3F5A06F31D000
:10140000A3F5C063012B90D8636894F846205E680A
:1014100094F84710B4F848302046B047002884D0EC
:101420004368A3630368E3631AE0B3F5106F36D033
:1014300040F6024293427FF478AF5C4BA3630223F1
:10144000E3630023C3E794F84630012B7FF46DAFCC
:10145000B4F84C3023F00203C4E90E55A4F84C3024
:10146000256478E7B4F84430B3F5A06F0ED194F852
:10147000463084F84E30204600F09CFF63681B68BD
:1014800013B1012120469847032323700023C4E9A8
:101490000E339CE704F14F03A3630123C3E72378D2
:1014A000042B10D1302383F311882046FFF7C4FEAC
:1014B00085F311880321636884F84F5021701B68FD
:1014C0000BB12046984794F84630002BDED084F8C4
:1014D0004F300423237063681B68002BD6D0022191
:1014E00020469847D2E794F848301D0603F00F01D4
:1014F00020460AD501F00AF8012804D002287FF41A
:1015000014AF2B4B9AE72B4B98E700F0F1FFF3E772
:1015100094F84630002B7FF408AF94F8483013F06D
:101520000F01B3D01A06204602D501F0BDFAADE78F
:1015300001F0B0FAAAE794F84630002B7FF4F5AE3C
:1015400094F8483013F00F01A0D01B06204602D5B6
:1015500001F096FA9AE701F089FA97E7142284F8E5
:10156000342083F311882B462A4629462046FFF76C
:101570006DFE85F31188E9E65DB1152284F834200B
:1015800083F311880021D4E90E232046FFF75EFE85
:10159000FDE60B2284F8342083F311882B462A467B
:1015A00029462046FFF764FEE3E700BFA4330008A6
:1015B0009C330008A033000838B590F83430044656
:1015C000002B3ED0063BDAB20F2A34D80F2B32D88C
:1015D000DFE803F037313108223231313131313136
:1015E00031313737C56BB0F84A309D4214D2C368E9
:1015F0001B8AB5FBF3F203FB12556DB9302383F35D
:1016000011882B462A462946FFF732FE85F31188BA
:101610000A2384F834300EE0142384F83430302365
:1016200083F3118800231A4619462046FFF70EFE61
:10163000002383F3118838BD036C03B1984700235E
:10164000E7E70021204601F01BFA0021204601F0C7
:101650000DFA63681B6813B10621204698470623DC
:10166000D7E7000010B590F83430142B044629D089
:1016700017D8062B05D001D81BB110BD093B022B92
:10168000FBD80021204601F0FBF90021204601F0A3
:10169000EDF963681B6813B10621204698470623BD
:1016A00019E0152BE9D10B2380F83430302383F374
:1016B000118800231A461946FFF7DAFD002383F349
:1016C0001188DAE7C3689B695B68002BD5D1036C8E
:1016D00003B19847002384F83430CEE70023037524
:1016E000826803691B6899689142FBD25A6803605B
:1016F0004260106058607047002303758268036978
:101700001B6899689142FBD85A6803604260106078
:101710005860704708B50846302383F311880B7D65
:10172000032B05D0042B0DD02BB983F3118808BDF2
:101730008B6900221A604FF0FF338361FFF7CEFF01
:101740000023F2E7D1E9003213605A60F3E70000AA
:10175000FFF7C4BF38B50A4BDD681C6828752268DE
:101760001A605360DC60A36801229342227501D1A4
:1017700000F0F6FC29462046BDE83840FEF7C2BD21
:101780009823002030B50C4BDD684B1C87B0044615
:101790000FD02B46094A684600F054F92046FFF75F
:1017A000D9FF009B13B1684600F056F9A86907B04D
:1017B00030BDFFF7CFFFF9E7982300201517000889
:1017C000044B1A68DB6890689B68984294BF0020BD
:1017D000012070479823002038B50B4B1C68DD684A
:1017E00022681A60536001222275DC60AB68934264
:1017F00001D100F0B7FC2846FFF77EFF01462046E6
:10180000BDE83840FEF77EBD9823002038B5074C70
:1018100007490848012300252370656001F048FB53
:101820000223237085F3118838BD00BF00260020F5
:10183000AC3300089823002000F044B9034A5168F3
:1018400053685B1A9842FBD8704700BF001000E055
:101850008B60022308618B82084670478368A3F17E
:10186000840243F8142C026943F8442C426943F87B
:10187000402C094A43F8242CC26843F8182C022251
:1018800003F80C2C002203F80B2C044A43F8102C0C
:10189000A3F12000704700BF1D030008982300201B
:1018A00008B5FFF7DBFFBDE80840FFF751BF0000B8
:1018B000024BDB6898610F20FFF74CBF9823002094
:1018C000302383F31188FFF7F3BF000008B501460A
:1018D000302383F311880820FFF754FF002383F39C
:1018E000118808BD064BDB6839B1426818605A6040
:1018F000136043600420FFF745BF4FF0FF3070478F
:10190000982300200368984206D01A68026050604D
:1019100099611846FFF71CBF7047000038B50446B0
:101920000D462068844200D138BD036823605C60A6
:101930008561FFF70DFFF4E710B503689C68A242CC
:101940000CD85C688A600B604C60216059609968B3
:101950008A1A9A604FF0FF33836010BD1B68121B18
:10196000ECE700000A2938BF0A2170B504460D468D
:101970000A26601901F096FA01F082FA041BA542CA
:1019800003D8751C2E460446F3E70A2E04D9BDE899
:101990007040012001F0CCBA70BD0000F8B5144BC6
:1019A0000D46D96103F1100141600A2A196982606C
:1019B00038BF0A22016048601861A818144601F077
:1019C00063FA0A2701F05CFA431BA342064606D3DA
:1019D0007C1C281901F066FA27463546F2E70A2FE3
:1019E00004D9BDE8F840012001F0A2BAF8BD00BF5B
:1019F00098230020F8B506460D4601F041FA0F4A3B
:101A0000134653F8107F9F4206D12A4601463046BE
:101A1000BDE8F840FFF7C2BFD169BB68441A2C1972
:101A200028BF2C46A34202D92946FFF79BFF224636
:101A300031460348BDE8F840FFF77EBF98230020F9
:101A4000A823002010B4C0E9032300235DF8044B51
:101A50004361FFF7CFBF000010B5194C23699842CE
:101A60000DD0D0E90032816813605A609A680A4448
:101A70009A60002303604FF0FF33A36110BD23463B
:101A8000026843F8102F53600022026022699A42D4
:101A900003D1BDE8104001F0FFB9936881680B44A1
:101AA000936001F0EDF92269E1699268441AA2425B
:101AB000E4D91144BDE81040091AFFF753BF00BF35
:101AC000982300202DE9F047DFF8BC8008F11007CB
:101AD0002C4ED8F8105001F0D3F9D8F81C40AA6861
:101AE000031B9A423ED81444D5E900324FF0000956
:101AF000C8F81C4013605A60C5F80090D8F8103040
:101B0000B34201D101F0C8F989F31188D5E9033155
:101B100028469847302383F311886B69002BD8D06F
:101B200001F0AEF96A69A0EB04094A4582460DD27C
:101B3000022001F0FDF90022D8F81030B34208D19C
:101B400051462846BDE8F047FFF728BF121A224445
:101B5000F2E712EB090938BF4A4629463846FFF733
:101B6000EBFEB5E7D8F81030B34208D01444211A80
:101B7000C8F81C00A960BDE8F047FFF7F3BEBDE858
:101B8000F08700BFA8230020982300200020704782
:101B9000FEE70000704700004FF0FF307047000084
:101BA00002290CD0032904D00129074818BF0020BE
:101BB0007047032A05D8054800EBC2007047044867
:101BC00070470020704700BF8434000820220020A6
:101BD0003834000870B59AB00546084601A9144685
:101BE00000F0C2F801A8FFF7AFF8431C5B00C5E99D
:101BF00000340022237003236370C6B201AB0234A9
:101C00001046D1B28E4204F1020401D81AB070BD60
:101C100013F8011B04F8021C04F8010C0132F0E770
:101C200008B5302383F311880348FFF749FA0023EE
:101C300083F3118808BD00BF0826002090F84430C7
:101C400003F01F02012A07D190F845200B2A03D187
:101C50000023C0E90E3315E003F06003202B08D108
:101C6000B0F848302BB990F84520212A03D81F2A14
:101C700004D8FFF707BA222AEBD0FAE7034A8263B7
:101C80000722C26303640120704700BF18220020AE
:101C900007B5052917D8DFE801F01916031919202F
:101CA000302383F31188104A01900121FFF7AAFA2B
:101CB00001980E4A0221FFF7A5FA0D48FFF7CCF96B
:101CC000002383F3118803B05DF804FB302383F312
:101CD00011880748FFF796F9F2E7302383F311885C
:101CE0000348FFF7ADF9EBE7D8330008FC330008F1
:101CF0000826002038B50C4D0C4C0D492A4604F13D
:101D00000800FFF767FF05F1CA0204F11000094956
:101D1000FFF760FF05F5CA7204F118000649BDE837
:101D20003840FFF757BF00BFD02A002020220020F4
:101D3000B8330008C2330008CD33000870B504463C
:101D400008460D46FFF700F8C6B220460134037876
:101D50000BB9184670BD32462946FEF7E1FF002850
:101D6000F3D10120F6E700002DE9F84F05460C46B7
:101D7000FEF7EAFF2B49C6B22846FFF7DFFF08B19E
:101D80000336F6B228492846FFF7D8FF08B11036C7
:101D9000F6B2632E0DD8DFF88C80DFF88C90234FDD
:101DA000DFF890A0DFF890B02E7846B92670BDE835
:101DB000F88F29462046BDE8F84FFEF7BDBA252E1C
:101DC0002BD1072241462846FEF7AAFF58B9DBF877
:101DD00000302360DBF804306360BBF808302381F7
:101DE00007350A34E0E7082249462846FEF798FFFF
:101DF00098B90F4BA21C197809090232C95D02F883
:101E0000041C13F8011B01F00F015345C95D02F8D2
:101E1000031CF0D118340835C6E704F8016B01350E
:101E2000C2E700BFA4340008CD330008B73400086F
:101E3000107AFF1F1C7AFF1FAC340008BFF34F8FCE
:101E4000024AD368DB03FCD4704700BF003C024069
:101E500008B5094B1B7873B9FFF7F0FF074B1A69F8
:101E6000002ABFBF064A5A6002F188325A601A68D7
:101E700022F480621A6008BD2E2D0020003C024032
:101E80002301674508B50B4B1B7893B9FFF7D6FFC5
:101E9000094B1A6942F000421A611A6842F48052F2
:101EA0001A601A6822F480521A601A6842F480623A
:101EB0001A6008BD2E2D0020003C02400B28F0B512
:101EC00016D80C4C0C4923787BB90C4D0E460C23CC
:101ED0004FF0006255F8047B46F8042B013B13F0E9
:101EE000FF033A44F6D10123237051F82000F0BDDE
:101EF0000020FCE7602D0020302D0020C8340008B1
:101F0000014B53F820007047C83400080C2070477C
:101F10000B2810B5044601D9002010BDFFF7CEFFF5
:101F2000064B53F824301844C21A0BB90120F4E7C9
:101F300012680132F0D1043BF6E700BFC834000854
:101F40000B2810B5044621D8FFF778FFFFF780FF74
:101F50000F4AF323D360C300DBB243F4007343F0B2
:101F600002031361136943F480331361FFF766FFC3
:101F7000FFF7A4FF074B53F8241000F0D9F8FFF740
:101F800081FF2046BDE81040FFF7C2BF002010BD12
:101F9000003C0240C8340008F8B512F001031446B2
:101FA00042D18218B2F1016F57D82D4B1B6813F044
:101FB000010352D02B4DFFF74BFFF323EB60FFF7EC
:101FC0003DFF40F20127032C15D824F001046618C8
:101FD000244C401A40F20117B142236900EB01057D
:101FE00024D123F001032361FFF74CFF0120F8BD4A
:101FF000043C0430E7E78307E7D12B6923F44073FF
:102000002B612B693B432B6151F8046B0660BFF3D6
:102010004F8FFFF713FF03689E42E9D02B6923F02F
:1020200001032B61FFF72EFF0020E0E723F440734C
:10203000236123693B4323610B882B80BFF34F8FC0
:10204000FFF7FCFE2D8831F8023BADB2AB42C3D0A6
:10205000236923F001032361E4E71846C7E700BFC3
:1020600000380240003C0240084908B50B7828B10E
:102070001BB9FFF7EDFE01230B7008BD002BFCD050
:10208000BDE808400870FFF7FDBE00BF2E2D002000
:1020900010B50244064BD2B2904200D110BD441C90
:1020A00000B253F8200041F8040BE0B2F4E700BF9F
:1020B000502800400F4B30B51C6F240407D41C6F10
:1020C00044F400741C671C6F44F400441C670A4C01
:1020D000236843F4807323600244084BD2B29042D9
:1020E00000D130BD441C00B251F8045B43F82050CD
:1020F000E0B2F4E700380240007000405028004091
:1021000007B5012201A90020FFF7C2FF019803B023
:102110005DF804FB13B50446FFF7F2FFA04205D0BB
:10212000012201A900200194FFF7C4FF02B010BDF5
:1021300070470000034B1A681AB9034AD2F8742892
:102140001A607047642D00200030024008B5FFF788
:10215000F1FF024B1868C0F3407008BD642D0020E9
:10216000704700007047000070470000FEE7000065
:102170000A4B0B480B4A90420BD30B4BDA1C121A3A
:10218000C11E22F003028B4238BF00220021FEF75D
:10219000E3BD53F8041B40F8041BECE7703600085D
:1021A000E02D0020E02D0020E02D002070B5D0E9CA
:1021B00015439E6800224FF0FF3504EB4213510196
:1021C000D3F800090028BEBFD3F8000940F08040D2
:1021D000C3F80009D3F8000B0028BEBFD3F8000BEA
:1021E00040F08040C3F8000B013263189642C3F8F8
:1021F0000859C3F8085BE0D24FF00113C4F81C384B
:1022000070BD0000890141F02001016103699B0656
:10221000FCD41220FFF712BB10B5054C2046FEF788
:10222000D1FF4FF0A0436365024BA36510BD00BF13
:10223000682D00201C35000870B50378012B054679
:1022400050D12A4B446D98421BD1294B5A6B42F016
:1022500080025A635A6D42F080025A655A6D5A697B
:1022600042F080025A615A6922F080025A610E21BE
:1022700043205B6900F022FC1E4BE3601E4BC4F858
:1022800000380023C4F8003EC02323606E6D4FF475
:102290000413A3633369002BFCDA012333610C20A0
:1022A000FFF7CCFA3369DB07FCD41220FFF7C6FA3C
:1022B0003369002BFCDA0026A6602846FFF776FF7C
:1022C0006B68C4F81068DB68C4F81468C4F81C684C
:1022D0004BB90A4BA3614FF0FF336361A36843F02E
:1022E0000103A36070BD064BF4E700BF682D00201A
:1022F000003802404014004003002002003C30C07F
:10230000083C30C0F8B5446D054600212046FFF773
:1023100079FFA96D00234FF001128F68C4F834389B
:102320004FF00066C4F81C284FF0FF3004EB431256
:1023300001339F42C2F80069C2F8006BC2F8080975
:10234000C2F8080BF2D20B686A6DEB65636210236A
:102350001361166916F01006FBD11220FFF76EFA12
:10236000D4F8003823F4FE63C4F80038A36943F4BA
:10237000402343F01003A3610923C4F81038C4F8C4
:1023800014380A4BEB604FF0C043C4F8103B084BC5
:10239000C4F8003BC4F81069C4F80039EB6D03F1D0
:1023A000100243F48013EA65A362F8BDF834000814
:1023B00040800010426D90F84E10D2F8003823F49F
:1023C000FE6343EA0113C2F8003870472DE9F84371
:1023D00000EB8103456DDA68166806F00306731E8C
:1023E000022B05EB41130C4680460FFA81F94FEAA8
:1023F00041104FF00001C3F8101B4FF0010104F130
:10240000100398BFB60401FA03F391698EBF334EEF
:1024100006F1805606F5004600293AD0578A04F1A5
:102420005801490137436F50D5F81C180B43C5F8C4
:102430001C382B180021C3F8101953690127611E9D
:10244000A7409BB3138A928B9B08012A88BF5343F2
:10245000D8F85C20981842EA034301F1400205EBEA
:102460008202C8F85C00214653602846FFF7CAFE86
:1024700008EB8900C3681B8A43EA8453483464012B
:102480001E432E51D5F81C381F43C5F81C78BDE8F3
:10249000F88305EB4917D7F8001B21F40041C7F872
:1024A000001BD5F81C1821EA0303C0E704F13F0321
:1024B00005EB83030A4A5A6028462146FFF7A2FE2D
:1024C00005EB4910D0F8003923F40043C0F8003977
:1024D000D5F81C3823EA0707D7E700BF00800010B3
:1024E00000040002826D1268C265FFF75FBE000043
:1024F0005831436D49015B5813F4004004D013F484
:10250000001F0CBF02200120704700004831436DBE
:1025100049015B5813F4004004D013F4001F0CBFB2
:10252000022001207047000000EB8101CB68196A8E
:102530000B6813604B6853607047000000EB810329
:1025400030B5DD68AA691368D36019B9402B84BF20
:10255000402313606B8A1468426D1C44013CB4FB39
:10256000F3F46343033323F0030302EB411043EA24
:10257000C44343F0C043C0F8103B2B6803F003038F
:10258000012B09B20ED1D2F8083802EB411013F436
:10259000807FD0F8003B14BF43F0805343F00053DA
:1025A000C0F8003B02EB4112D2F8003B43F0044379
:1025B000C2F8003B30BD00002DE9F041244D6E6DA6
:1025C00006EB40130446D3F8087BC3F8087B3807B2
:1025D0000AD5D6F81438190706D505EB8403214629
:1025E000DB6828465B689847FA071FD5D6F8143889
:1025F000DB071BD505EB8403D968CCB98B69488A06
:102600005A68B2FBF0F600FB16228AB91868DA683D
:1026100090420DD2121AC3E90024302383F31188AB
:102620000B482146FFF78AFF84F31188BDE8F0814B
:10263000012303FA04F26B8923EA02036B81CB685E
:10264000002BF3D021460248BDE8F041184700BFF7
:10265000682D002000EB810370B5DD68436D6C6967
:102660002668E6604A0156BB1A444FF40020C2F8BF
:1026700010092A6802F00302012A0AB20ED1D3F827
:10268000080803EB421410F4807FD4F8000914BF4B
:1026900040F0805040F00050C4F8000903EB4212B3
:1026A000D2F8000940F00440C2F80009D3F8340819
:1026B000012202FA01F10143C3F8341870BD19B9BF
:1026C000402E84BF4020206020682E8A8419013C5F
:1026D000B4FBF6F440EAC44040F000501A44C6E7A8
:1026E0002DE9F8433B4D6E6D06EB40130446D3F8DD
:1026F0000889C3F8088918F0010F4FEA40171AD06B
:10270000D6F81038DB0716D505EB8003D9684B697E
:102710001868DA68904230D2121A4FF000091A6035
:10272000C3F80490302383F3118821462846FFF72D
:1027300091FF89F3118818F0800F1CD0D6F8343837
:102740000126A640334216D005EB84036D6DD3F805
:102750000CC0DCF814200134E4B2D2F800E005EB40
:1027600004342F445168714515D3D5F8343823EA21
:102770000606C5F83468BDE8F883012303FA04F2BD
:102780002B8923EA02032B818B68002BD3D02146AF
:1027900028469847CFE7BCF81000AEEB0103834210
:1027A00028BF0346D7F8180980B2B3EB800FE2D8F0
:1027B0009068A0F1040959F8048FC4F80080A0EBD8
:1027C00009089844B8F1040FF5D818440B449060F8
:1027D0005360C7E7682D00202DE9F74FA24C656DC7
:1027E0006E69AB691E4016F480586E6107D02046B2
:1027F000FEF750FD03B0BDE8F04F00F047BC002EDF
:1028000012DAD5F8003E98489B071EBFD5F8003E67
:1028100023F00303C5F8003ED5F8043823F0010384
:10282000C5F80438FEF760FD370505D58E48FFF77B
:10283000BDFC8D48FEF746FDB0040CD5D5F8083830
:1028400013F0060FEB6823F470530CBF43F41053DE
:1028500043F4A053EB6031071BD56368DB681BB9F9
:10286000AB6923F00803AB612378052B0CD1D5F8B5
:10287000003E7D489A071EBFD5F8003E23F00303B3
:10288000C5F8003EFEF730FD6368DB680BB17648A3
:102890009847F30274D4B70227D5D4F85490DFF8E0
:1028A000C8B100274FF0010A09EB4712D2F8003BEC
:1028B00003F44023B3F5802F11D1D2F8003B002B55
:1028C0000DDA62890AFA07F322EA0303638104EB53
:1028D0008703DB68DB6813B1394658469847A36D18
:1028E00001379B68FFB29F42DED9F00617D5676DAE
:1028F0003A6AC2F30A1002F00F0302F4F012B2F5C2
:10290000802F00F08580B2F5402F08D104EB8303BF
:102910000022DB681B6A07F5805790426AD13003BA
:10292000D5F8184813D5E10302D50020FFF744FE7F
:10293000A20302D50120FFF73FFE630302D5022068
:10294000FFF73AFE270302D50320FFF735FE750394
:102950007FF550AFE00702D50020FFF7C1FEA107C9
:1029600002D50120FFF7BCFE620702D50220FFF767
:10297000B7FE23077FF53EAF0320FFF7B1FE39E72F
:10298000636DDFF8E4A0019300274FF00109A36D08
:102990009B685FFA87FB9B453FF67DAF019B03EB8E
:1029A0004B13D3F8001901F44021B1F5802F1FD14A
:1029B000D3F8001900291BDAD3F8001941F090412F
:1029C000C3F80019D3F800190029FBDB5946606DE4
:1029D000FFF718FC218909FA0BF321EA030323818D
:1029E00004EB8B03DB689B6813B15946504698474C
:1029F0000137CCE7910708BFD7F80080072A98BFB6
:102A000003F8018B02F1010298BF4FEA182884E70E
:102A1000023304EB830207F580575268D2F818C0DE
:102A2000DCF80820DCE9001CA1EB0C0C002188423A
:102A30000AD104EB830463689B699A6802449A6034
:102A40005A6802445A606AE711F0030F08BFD7F8CA
:102A500000808C4588BF02F8018B01F1010188BF1D
:102A60004FEA1828E3E700BF682D0020436D03EB11
:102A70004111D1F8003B43F40013C1F8003B70470B
:102A8000436D03EB4111D1F8003943F40013C1F851
:102A900000397047436D03EB4111D1F8003B23F43B
:102AA0000013C1F8003B7047436D03EB4111D1F8AF
:102AB000003923F40013C1F80039704700F1604376
:102AC00003F561430901C9B283F80013012200F044
:102AD0001F039A4043099B0003F1604303F56143E0
:102AE000C3F880211A60704730B5039C017204332B
:102AF00004FB0325C0E90653049B03630021059BE7
:102B0000C160C0E90000C0E90422C0E90842C0E990
:102B10000A11436330BD0000416A0022C0E904117C
:102B2000C0E90A22C2606FF00101FEF7F7BE0000A3
:102B3000D0E90432934201D1C2680AB9181D704726
:102B40000020704703691960C2680132C260C2691F
:102B5000134482690361934224BF436A03610021E5
:102B6000FEF7D0BE38B504460D46E3683BB1626956
:102B7000131D1268A3621344E362002007E0237A66
:102B800033B929462046FEF7ADFE0028EDDA38BD00
:102B90006FF00100FBE70000C368C269013BC3603E
:102BA0004369134482694361934224BF436A43618A
:102BB00000238362036B03B11847704770B530235D
:102BC000044683F31188866A3EB9FFF7CBFF0546BA
:102BD00018B186F31188284670BDA36AE26A13F81B
:102BE000015BA362934202D32046FFF7D5FF002387
:102BF00083F31188EFE700002DE9F84F04460E46F5
:102C0000174698464FF0300989F311880025AA46E7
:102C1000D4F828B0BBF1000F09D141462046FFF798
:102C2000A1FF20B18BF311882846BDE8F88FD4E9C5
:102C30000A12A7EB050B521A934528BF9346BBF126
:102C4000400F1BD9334601F1400251F8040B43F801
:102C5000040B9142F9D1A36A40334036A362403558
:102C6000D4E90A239A4202D32046FFF795FF8AF35C
:102C70001188BD42D8D289F31188C9E730465A4637
:102C8000FEF744F8A36A5B445E44A3625D44E7E751
:102C900010B5029C0172043303FB0421C0E9061342
:102CA0000023C0E90A33039B0363049BC460C0E9AB
:102CB0000000C0E90422C0E90842436310BD0000DF
:102CC000026AC260426AC0E904220022C0E90A2204
:102CD0006FF00101FEF722BED0E904239A4201D130
:102CE000C26822B9184650F8043B0B6070470023B5
:102CF0001846FAE7C368C2690133C36043691344E5
:102D000082694361934224BF436A43610021FEF715
:102D1000F9BD000038B504460D46E3683BB12369B0
:102D20001A1DA262E2691344E362002007E0237ADD
:102D300033B929462046FEF7D5FD0028EDDA38BD27
:102D40006FF00100FBE7000003691960C268013AF7
:102D5000C260C269134482690361934224BF436A1B
:102D6000036100238362036B03B1184770470000BF
:102D700070B530230D460446114683F31188866AE8
:102D80002EB9FFF7C7FF10B186F3118870BDA36A93
:102D90001D70A36AE26A01339342A36204D3E1691E
:102DA00020460439FFF7D0FF002080F31188EDE7BB
:102DB0002DE9F84F04460D46904699464FF0300AEB
:102DC0008AF311880026B346A76A4FB949462046C0
:102DD000FFF7A0FF20B187F311883046BDE8F88FD8
:102DE000D4E90A073A1AA8EB0607974228BF174604
:102DF000402F1BD905F1400355F8042B40F8042B54
:102E00009D42F9D1A36A4033A3624036D4E90A2334
:102E10009A4204D3E16920460439FFF795FF8BF30A
:102E200011884645D9D28AF31188CDE729463A461A
:102E3000FDF76CFFA36A3B443D44A3623E44E5E7D3
:102E4000D0E904239A4217D1C3689BB1836A8BB13E
:102E5000043B9B1A0ED01360C368013BC360C36977
:102E60001A44836902619A4224BF436A03610023C2
:102E700083620123184670470023FBE700F030B956
:102E80004FF08043586A70474FF0804300225863E8
:102E90001A610222DA6070474FF080430022DA6044
:102EA000704700004FF0804358637047FEE7000012
:102EB00070B51B4B01630025044686B058608562DF
:102EC0000E4600F0BFF804F11003C4E904334FF0DC
:102ED000FF33C4E90635C4E90044A560E562FFF7A5
:102EE000CFFF2B460246C4E9082304F134010D4A02
:102EF000256580232046FEF7ABFC0123E0600A4AEB
:102F00000375009272680192B268CDE90223074B03
:102F10006846CDE90435FEF7C3FC06B070BD00BFBE
:102F200000260020283500082D350008AD2E0008A9
:102F3000024AD36A1843D062704700BF982300202A
:102F40004B6843608B688360CB68C3600B694361E7
:102F50004B6903628B6943620B6803607047000032
:102F600008B5264B26481A6940F2FF110A431A6138
:102F70001A6922F4FF7222F001021A611A691A6BAF
:102F80000A431A631A6D0A431A651E4A1B6D1146DD
:102F9000FFF7D6FF02F11C0100F58060FFF7D0FFBC
:102FA00002F1380100F58060FFF7CAFF02F1540119
:102FB00000F58060FFF7C4FF02F1700100F580604A
:102FC000FFF7BEFF02F18C0100F58060FFF7B8FF4C
:102FD00002F1A80100F58060FFF7B2FF02F1C40121
:102FE00000F58060FFF7ACFF02F1E00100F58060C2
:102FF000FFF7A6FFBDE8084000F0EEB80038024039
:10300000000002403435000808B500F06BF9FEF707
:10301000FDFBFFF78FF8BDE80840FEF76BBE000030
:1030200070470000EFF3098305494A6B22F0010263
:103030004A63683383F30988002383F31188704758
:1030400000EF00E0302080F3118862B60C4B0D4A8F
:10305000D96821F4E0610904090C0A43DA60D3F865
:10306000FC20094942F08072C3F8FC200A6842F053
:1030700001020A602022DA7783F82200704700BF3D
:1030800000ED00E00003FA05001000E010B5302369
:1030900083F311880E4B5B6813F4006314D0F1EED8
:1030A000103AEFF30984683C4FF08073E361094BF9
:1030B000DB6B236684F30988FEF782FB10B1064BB5
:1030C000A36110BD054BFBE783F31188F9E700BF4F
:1030D00000ED00E000EF00E02F03000832030008DD
:1030E0000F4B1A6C42F001021A641A6E42F0010290
:1030F0001A660C4A1B6E936843F0010393604FF00D
:10310000804353229A624FF0FF32DA6200229A61C2
:103110005A63DA605A6001225A611A60704700BF30
:1031200000380240002004E04FF0804208B51169E9
:10313000D3680B40D9B2C9439B07116107D530232F
:1031400083F31188FEF778FB002383F3118808BD11
:103150001F4B1A696FEAC2526FEAD2521A611A699A
:10316000C2F308021A614FF0FF301A695A695861B8
:1031700000215A6959615A691A6A62F080521A62CA
:103180001A6A02F080521A621A6A5A6A58625A6AB5
:1031900059625A6A1A6C42F080521A641A6E42F0EE
:1031A00080521A661A6E0B4A106840F480701060E4
:1031B000186F00F44070B0F5007F1EBF4FF48030F0
:1031C00018671967536823F40073536000F086B8DA
:1031D0000038024000700040334B4FF080521A64B8
:1031E000324A4FF4404111601A6842F001021A60FD
:1031F0001A689107FCD59A6822F003029A602A4B5C
:103200009A6812F00C02FBD1196801F0F9011960FB
:103210009A601A6842F480321A601A689203FCD5E8
:103220005A6F42F001025A671F4B5A6F9007FCD544
:103230001F4A5A601A6842F080721A601B4A53682B
:103240005904FCD5184B1A689201FCD5194A9A60AA
:10325000194B1A68194B9A42194B21D1194A116816
:10326000194A91421CD140F205121A60144A13689F
:1032700003F00F03052BFAD10B4B9A6842F00202C0
:103280009A609A6802F00C02082AFAD15A6C42F449
:1032900080425A645A6E42F480425A665B6E7047AE
:1032A00040F20572E1E700BF0038024000700040C4
:1032B0000854400700948838002004E0116400207E
:1032C000003C024000ED00E041C20F4108B5FFF7AD
:1032D0002BFFBDE80840FFF7D9BE000007211C20E6
:1032E000FFF7ECBB08B5FFF733FF00F00BF8FDF775
:1032F00067FFFDF73FFEFFF793FEBDE80840FFF7CD
:10330000BDBD000070470000121000001211000047
:103310001213000053544D3332463F3F3F00535485
:103320004D3332463430780053544D3332463432C4
:10333000780053544D333246343436585800000028
:10334000012033000010410001105A000310590001
:1033500007103100000000001433000813040000BF
:103360001E3300081904000028330008210400005F
:103370003233000800000000F10E0008DD0E0008E6
:10338000190F0008050F0008110F0008FD0E0008B6
:10339000E90E0008D50E0008250F00080000000007
:1033A000010000000000000063300000A8330008A6
:1033B000F0230020002600204172647550696C6F74
:1033C000740025424F415244252D424C002553455F
:1033D0005249414C2500000002000000000000009E
:1033E0000D1100087911000840004000A02A0020BB
:1033F000B02A0020020000000000000003000000CE
:1034000000000000BD1100080000000010000000D6
:10341000C02A0020000000000100000000000000A1
:10342000682D002001010200911C0008A11B00086A
:103430003D1C0008211C0008430000004034000827
:1034400009024300020100C0320904000001020227
:1034500001000524001001052401000104240202DA
:103460000524060001070582030800FF0904010086
:10347000020A000000070501024000000705810262
:1034800040000000120000008C34000812011001FE
:10349000020000400912415700020102030100002E
:1034A0000403090425424F415244250049726F6EBE
:1034B000436F726546340030313233343536373835
:1034C00039414243444546000040000000400000AE
:1034D0000040000000400000000001000000020069
:1034E00000000200000002000000020000000200D4
:1034F00000000200000002000000000001130008AC
:10350000B91500086516000840004000C82D0020CD
:10351000C82D002001000000D82D002080000000F0
:1035200040010000030000006D61696E0069646C79
:10353000650000000001802A00000000AAAAAAAAD3
:1035400000010024FFFF00000000000000A00A00AE
:103550000000000100000000AAAAAAAA00000001C1
:10356000FFFF000000000000000000000000005409
:1035700000000000AAAAAAAA00000010FFDF0000B5
:10358000000000000000000000000000000000003B
:10359000AAAAAAAA00000000FFFF00000000000085
:1035A000000000000000000000000000AAAAAAAA73
:1035B00000000000FFFF000000000000000000000D
:1035C0000000000000000000AAAAAAAA0000000053
:1035D000FFFF0000000000000000000000000000ED
:1035E00000000000AAAAAAAA00000000FFFF000035
:1035F00000000000000000000000000000000000CB
:103600000A000000000000000300000000000000AD
:1036100000000000000000000000000000000000AA
:10362000000000000000000000000000000000009A
:10363000DA1B00000000000000400F000000000046
:10364000FF0096000000000800960000000008003F
:1036500004000000A034000800000000000000008A
:10366000000000000000000000000000000000005A
:10367000FFFFFFFFFFFFFFFFFFFFFFFFFFFFFFFF5A
:10368000FFFFFFFFFFFFFFFFFFFFFFFFFFFFFFFF4A
:10369000FFFFFFFFFFFFFFFFFFFFFFFFFFFFFFFF3A
:10C0000000060020D9D20008750D0A08D10C0A08D4
:10C010003D0D0A08D10C0A08090D0A08DBD20008F8
:10C02000DBD20008DBD20008DBD20008D14A0C08C2
:10C03000DBD20008DBD20008DBD20008DBD200082C
:10C04000DBD20008DBD20008DBD20008DBD200081C
:10C05000DBD20008DBD2000869560C0891560C08A8
:10C06000B9560C08E1560C0809570C08E1FC0B08FE
:10C0700009FD0B0835FD0B0861FD0B088DFD0B0854
:10C08000B5FD0B08E1FD0B0865FC0B08DBD20008D1
:10C09000DBD20008DBD20008DBD2000831570C08E5
:10C0A0007D580C0881580C0895580C0899580C08B4
:10C0B0009D580C08B1580C08C5580C086D030C08A5
:10C0C00015050C08DBD20008DBD20008DBD2000823
:10C0D000DBD2000805580C0819580C082D580C081C
:10C0E00095570C08DBD20008DBD20008E9580C0891
:10C0F000ED580C0801590C0805590C080DFE0B08E9
:10C10000DBD20008DBD20008D9580C08DBD20008CB
:10C1100041580C0855580C08DBD20008DBD2000847
:10C1200039FE0B0861FE0B088DFE0B08B9FE0B08EB
:10C13000E5FE0B08DBD20008DBD20008DBD20008EA
:10C14000DBD20008DBD20008DBD20008FD510C086E
:10C150000DFF0B0839FF0B0865FF0B0869580C0829
:10C16000DBD20008DBD20008DBD20008DBD20008FB
:10C17000DBD20008DBD20008DBD20008DBD20008EB
:10C18000DBD20008DBD20008DBD20008DBD20008DB
:10C19000DBD20008DBD20008DBD20008DBD20008CB
:10C1A000DBD20008DBD20008DBD20008DBD20008BB
:10C1B000DBD20008DBD20008DBD20008DBD20008AB
:10C1C000DBD20008DBD20008DBD20008DBD200089B
:10C1D000DBD20008DBD20008DBD20008DBD200088B
:10C1E00089830108F9B10108C13B0208F98F0208EF
:10C1F000911A03086D9204083D1E0608452406089E
:10C20000A15E0608C1B80608F1C1060839C50608CE
:10C21000952D070879320708D54D0708ADE20708C4
:10C220008D530808496008089DFE090801040A08A2
:10C23000593E0B0811650B08B97B0B0851A90B0877
:10C2400019AF0B0800000000000000000000000013
:10C2500000000000000000000000000000000000DE
:10C2600000000000000000000000000000000000CE
:10C2700000000000000000000000000000000000BE
:10C2800081F0004102E000BF83F0004330B54FEA87
:10C2900041044FEA430594EA050F08BF90EA020FF4
:10C2A0001FBF54EA000C55EA020C7FEA645C7FEA87
:10C2B000655C00F0E2804FEA5454D4EB5555B8BFAA
:10C2C0006D420CDD2C4480EA020281EA030382EA1B
:10C2D000000083EA010180EA020281EA0303362DAD
:10C2E00088BF30BD11F0004F4FEA01314FF4801C80
:10C2F0004CEA113102D0404261EB410113F0004F92
:10C300004FEA03334CEA133302D0524263EB430348
:10C3100094EA050F00F0A780A4F10104D5F1200EE6
:10C320000DDB02FA0EFC22FA05F2801841F1000141
:10C3300003FA0EF2801843FA05F359410EE0A5F115
:10C3400020050EF1200E012A03FA0EFC28BF4CF046
:10C35000020C43FA05F3C01851EBE37101F00045FC
:10C3600007D54FF0000EDCF1000C7EEB00006EEB09
:10C370000101B1F5801F1BD3B1F5001F0CD3490893
:10C380005FEA30004FEA3C0C04F101044FEA4452EA
:10C3900012F5800F80F09A80BCF1004F08BF5FEA71
:10C3A000500C50F1000041EB045141EA050130BD51
:10C3B0005FEA4C0C404141EB0101013C28BFB1F563
:10C3C000801FE9D291F0000F04BF01460020B1FAAE
:10C3D00081F308BF2033A3F10B03B3F120020CDA81
:10C3E0000C3208DD02F1140CC2F10C0201FA0CF05F
:10C3F00021FA02F10CE002F11402D8BFC2F1200CC4
:10C4000001FA02F120FA0CFCDCBF41EA0C01904079
:10C41000E41AA2BF01EB0451294330BD6FEA0404C2
:10C420001F3C1CDA0C340EDC04F11404C4F12002AD
:10C4300020FA04F001FA02F340EA030021FA04F3BF
:10C4400045EA030130BDC4F10C04C4F1200220FA16
:10C4500002F001FA04F340EA0300294630BD21FA54
:10C4600004F0294630BD94F0000F83F4801306BF1A
:10C4700081F480110134013D4EE77FEA645C18BF0E
:10C480007FEA655C29D094EA050F08BF90EA020FA5
:10C4900005D054EA000C04BF1946104630BD91EA9D
:10C4A000030F1EBF0021002030BD5FEA545C05D1A0
:10C4B0004000494128BF41F0004130BD14F58004DF
:10C4C0003CBF01F5801130BD01F0004545F0FE4153
:10C4D00041F470014FF0000030BD7FEA645C1ABF88
:10C4E000194610467FEA655C1CBF0B46024650EABF
:10C4F000013406BF52EA033591EA030F41F40021EB
:10C5000030BD00BF90F0000F04BF0021704730B570
:10C510004FF4806404F132044FF000054FF0000145
:10C5200050E700BF90F0000F04BF0021704730B506
:10C530004FF4806404F1320410F0004548BF4042DB
:10C540004FF000013EE700BF42004FEAE2014FEA30
:10C5500031014FEA02701FBF12F07F4393F07F4F0B
:10C5600081F06051704732F07F4208BF704793F00E
:10C570007F4F04BF41F40021704730B54FF4607421
:10C5800001F0004521F000411CE700BF50EA010224
:10C5900008BF704730B54FF000050AE050EA0102CD
:10C5A00008BF704730B511F0004502D5404261EB3D
:10C5B00041014FF4806404F132045FEA915C3FF47E
:10C5C000D8AE4FF003025FEADC0C18BF03325FEA1B
:10C5D000DC0C18BF033202EBDC02C2F1200300FACC
:10C5E00003FC20FA02F001FA03FE40EA0E0021FAF1
:10C5F00002F11444BDE600BF70B54FF0FF0C4CF4DF
:10C60000E06C1CEA11541DBF1CEA135594EA0C0F90
:10C6100095EA0C0F00F0DEF82C4481EA030621EACB
:10C620004C5123EA4C5350EA013518BF52EA033506
:10C6300041F4801143F4801338D0A0FB02CE4FF0B8
:10C640000005E1FB02E506F00042E0FB03E54FF0E8
:10C650000006E1FB03569CF0000F18BF4EF0010EE0
:10C66000A4F1FF04B6F5007F64F5407404D25FEADC
:10C670004E0E6D4146EB060642EAC62141EA55518F
:10C680004FEAC52040EA5E504FEACE2EB4F1FD0CD1
:10C6900088BFBCF5E06F1ED8BEF1004F08BF5FEA4F
:10C6A000500E50F1000041EB045170BD06F0004601
:10C6B00046EA010140EA020081EA0301B4EB5C04AE
:10C6C000C2BFD4EB0C0541EA045170BD41F48011A6
:10C6D0004FF0000E013C00F3AB8014F1360FDEBFCB
:10C6E000002001F0004170BDC4F10004203C35DAA7
:10C6F0000C341BDC04F11404C4F1200500FA05F32A
:10C7000020FA04F001FA05F240EA020001F00042CA
:10C7100021F0004110EBD37021FA04F642EB060140
:10C720005EEA430E08BF20EAD37070BDC4F10C046A
:10C73000C4F1200500FA04F320FA05F001FA04F22E
:10C7400040EA020001F0004110EBD37041F100011A
:10C750005EEA430E08BF20EAD37070BDC4F1200525
:10C7600000FA05F24EEA020E20FA04F301FA05F28D
:10C7700043EA020321FA04F001F0004121FA04F235
:10C7800020EA020000EBD3705EEA430E08BF20EA05
:10C79000D37070BD94F0000F0FD101F0004640003F
:10C7A00041EB010111F4801F08BF013CF7D041EAC1
:10C7B000060195F0000F18BF704703F000465200C5
:10C7C00043EB030313F4801F08BF013DF7D043EA96
:10C7D0000603704794EA0C0F0CEA135518BF95EA4C
:10C7E0000C0F0CD050EA410618BF52EA4306D1D1D3
:10C7F00081EA030101F000414FF0000070BD50EAF2
:10C80000410606BF1046194652EA430619D094EA7B
:10C810000C0F02D150EA013613D195EA0C0F05D165
:10C8200052EA03361CBF104619460AD181EA0301B9
:10C8300001F0004141F0FE4141F470014FF0000071
:10C8400070BD41F0FE4141F4780170BD70B54FF00C
:10C85000FF0C4CF4E06C1CEA11541DBF1CEA13558C
:10C8600094EA0C0F95EA0C0F00F0A7F8A4EB05046E
:10C8700081EA030E52EA03354FEA013100F0888065
:10C880004FEA03334FF0805545EA131343EA12632E
:10C890004FEA022245EA111545EA10654FEA0026E3
:10C8A0000EF000419D4208BF964244F1FD0404F59C
:10C8B000407402D25B084FEA3202B61A65EB0305F8
:10C8C0005B084FEA32024FF480104FF4002CB6EBB5
:10C8D000020E75EB030E22BFB61A754640EA0C0035
:10C8E0005B084FEA3202B6EB020E75EB030E22BF75
:10C8F000B61A754640EA5C005B084FEA3202B6EBB6
:10C90000020E75EB030E22BFB61A754640EA9C0074
:10C910005B084FEA3202B6EB020E75EB030E22BF44
:10C92000B61A754640EADC0055EA060E18D04FEA02
:10C93000051545EA16754FEA06164FEAC30343EAA2
:10C9400052734FEAC2025FEA1C1CC0D111F4801F6F
:10C950000BD141EA00014FF000004FF0004CB6E768
:10C9600011F4801F04BF01430020B4F1FD0C88BF07
:10C97000BCF5E06F3FF6AFAEB5EB030C04BFB6EB12
:10C98000020C5FEA500C50F1000041EB045170BD05
:10C990000EF0004E4EEA113114EB5C04C2BFD4EB32
:10C9A0000C0541EA045170BD41F480114FF0000EB6
:10C9B000013C90E645EA060E8DE60CEA135594EA32
:10C9C0000C0F08BF95EA0C0F3FF43BAF94EA0C0F35
:10C9D0000AD150EA01347FF434AF95EA0C0F7FF4AA
:10C9E00025AF104619462CE795EA0C0F06D152EAFE
:10C9F00003353FF4FDAE1046194622E750EA4106E2
:10CA000018BF52EA43067FF4C5AE50EA41047FF4F2
:10CA10000DAF52EA43057FF4EBAE12E74FF0FF3C57
:10CA200006E000BF4FF0010C02E000BF4FF0010C28
:10CA30004DF804CD4FEA410C7FEA6C5C4FEA430CA1
:10CA400018BF7FEA6C5C1BD001B050EA410C0CBFF0
:10CA500052EA430C91EA030F02BF90EA020F002052
:10CA6000704710F1000F91EA030F58BF994208BFB9
:10CA700090422CBFD8176FEAE37040F00100704776
:10CA80004FEA410C7FEA6C5C02D150EA013C07D1CD
:10CA90004FEA430C7FEA6C5CD6D152EA033CD3D018
:10CAA0005DF8040B704700BF8446104662468C4612
:10CAB0001946634600E000BF01B5FFF7B7FF002845
:10CAC00048BF10F1000F01BD4DF808EDFFF7F4FF6E
:10CAD0000CBF012000205DF808FB00BF4DF808EDF9
:10CAE000FFF7EAFF34BF012000205DF808FB00BF1C
:10CAF0004DF808EDFFF7E0FF94BF012000205DF83E
:10CB000008FB00BF4DF808EDFFF7CEFF94BF0120F2
:10CB100000205DF808FB00BF4DF808EDFFF7C4FFEB
:10CB200034BF012000205DF808FB00BF4FEA410C34
:10CB30007FEA6C5C02D150EA013C0AD14FEA430C17
:10CB40007FEA6C5C02D152EA033C02D14FF0000054
:10CB500070474FF0010070474FEA410212F5001292
:10CB600015D211D56FF47873B3EB625212D94FEA34
:10CB7000C12343F0004343EA505311F0004F23FA1E
:10CB800002F018BF404270474FF00000704750EA73
:10CB9000013005D111F0004008BF6FF00040704730
:10CBA0004FF00000704700BF4A0011D212F500128A
:10CBB00011D20DD56FF47873B3EB62520ED44FEAF5
:10CBC000C12343F0004343EA505323FA02F0704775
:10CBD0004FF00000704750EA013002D14FF0FF30B3
:10CBE00070474FF0000070474FEA4102B2F1E04356
:10CBF00024BFB3F5001CDCF1FE5C0DD901F0004C44
:10CC00004FEAC0024CEA5070B2F1004F40EB830093
:10CC100008BF20F00100704711F0804F21D113F1BF
:10CC20003872BCBF01F00040704741F480114FEAF8
:10CC30005252C2F11802C2F1200C10FA0CF320FA81
:10CC400002F018BF40F001004FEAC1234FEAD3239E
:10CC500003FA0CFC40EA0C0023FA02F34FEA430308
:10CC6000CCE77FEA625307D150EA01331EBF4FF091
:10CC7000FE4040F44000704701F0004040F0FE40AC
:10CC800040F40000704700BF80F0004002E000BFA9
:10CC900081F0004142001FBF5FEA410392EA030FA7
:10CCA0007FEA226C7FEA236C6AD04FEA1262D2EBF1
:10CCB0001363C1BFD218414048404140B8BF5B42F6
:10CCC000192B88BF704710F0004F40F4000020F08F
:10CCD0007F4018BF404211F0004F41F4000121F0A5
:10CCE0007F4118BF494292EA030F3FD0A2F10102EF
:10CCF00041FA03FC10EB0C00C3F1200301FA03F12D
:10CD000000F0004302D5494260EB4000B0F5000F4F
:10CD100013D3B0F1807F06D340084FEA310102F10E
:10CD20000102FE2A51D2B1F1004F40EBC25008BFC0
:10CD300020F0010040EA03007047490040EB00008A
:10CD4000013A28BFB0F5000FEDD2B0FA80FCACF18B
:10CD5000080CB2EB0C0200FA0CF0AABF00EBC250B8
:10CD600052421843BCBFD0401843704792F0000FA6
:10CD700081F4000106BF80F400000132013BB5E7F9
:10CD80004FEA41037FEA226C18BF7FEA236C21D06F
:10CD900092EA030F04D092F0000F08BF08467047D4
:10CDA00090EA010F1CBF0020704712F07F4F04D1A2
:10CDB000400028BF40F00040704712F100723CBFB5
:10CDC00000F50000704700F0004343F0FE4040F4DF
:10CDD000000070477FEA226216BF08467FEA23639D
:10CDE0000146420206BF5FEA412390EA010F40F488
:10CDF000800070474FF0000304E000BF10F00043D4
:10CE000048BF40425FEA000C08BF704743F09643BA
:10CE100001464FF000001CE050EA010208BF7047D5
:10CE20004FF000030AE000BF50EA010208BF70475C
:10CE300011F0004302D5404261EB41015FEA010C71
:10CE400002BF84460146002043F0B64308BFA3F169
:10CE50008053A3F50003BCFA8CF2083AA3EBC2534B
:10CE600010DB01FA02FC634400FA02FCC2F120026A
:10CE7000BCF1004F20FA02F243EB020008BF20F0A1
:10CE80000100704702F1200201FA02FCC2F1200207
:10CE900050EA4C0021FA02F243EB020008BF20EAFC
:10CEA000DC7070477BB972B90029BEBF00204FF01B
:10CEB000004106E008BF00281CBF6FF000414FF0A2
:10CEC000FF3000F007BAADF1080C6DE904CE00297F
:10CED00009DB002B1ADB00F095F8DDF804E0DDE952
:10CEE000022304B07047404261EB4101002B1BDB81
:10CEF00000F088F8DDF804E0DDE9022304B04042E8
:10CF000061EB4101524263EB43037047524263EBD2
:10CF1000430300F077F8DDF804E0DDE9022304B014
:10CF2000404261EB41017047524263EB430300F022
:10CF300069F8DDF804E0DDE9022304B0524263EB56
:10CF40004303704753B94AB9002908BF00281CBFE2
:10CF50004FF0FF314FF0FF3000F0BCB9ADF1080CDD
:10CF60006DE904CE00F04EF8DDF804E0DDE90223BF
:10CF700004B07047430803F05533C01A830803F028
:10CF8000333300F03330184400EB101000F00F3052
:10CF900000EB002000EB0040000E704707EE900A07
:10CFA000F5EEC07AF1EE10FA01D400F00BB8F1EE14
:10CFB000677A08B517EE900A00F004F8404261EB7A
:10CFC000410108BDD0B5FFF7BFFA0C4B0022064661
:10CFD0000F46FFF711FBFFF7E7FD0446FFF792FA54
:10CFE000074B0022FFF708FB02460B463046394646
:10CFF000FFF74AF9FFF7D8FD2146D0BD0000F03D0C
:10D000000000F0412DE9F047089D04468E46002BB4
:10D010004DD18A42944669D9B2FA82F252B101FAEC
:10D0200002F3C2F1200120FA01F10CFA02FC41EAFC
:10D03000030E94404FEA1C48210CBEFBF8F61FFA81
:10D040008CF708FB16E341EA034306FB07F199421C
:10D050000AD91CEB030306F1FF3080F01F819942CF
:10D0600040F21C81023E63445B1AA4B2B3FBF8F0A9
:10D0700008FB103344EA034400FB07F7A7420AD930
:10D080001CEB040400F1FF3380F00A81A74240F258
:10D0900007816444023840EA0640E41B00261DB1C3
:10D0A000D4400023C5E900433146BDE8F0878B42F8
:10D0B00009D9002D00F0EF800026C5E900013046B7
:10D0C0003146BDE8F087B3FA83F6002E4AD18B4291
:10D0D00002D3824200F2F980841A61EB030301203B
:10D0E0009E46002DE0D0C5E9004EDDE702B9FFDE27
:10D0F000B2FA82F2002A40F09280A1EB0C014FEAD2
:10D100001C471FFA8CFE0126200CB1FBF7F307FB2E
:10D11000131140EA01410EFB03F0884208D91CEBD1
:10D12000010103F1FF3802D2884200F2CB8043466E
:10D13000091AA4B2B1FBF7F007FB101144EA01444D
:10D140000EFB00FEA64508D91CEB040400F1FF31DC
:10D1500002D2A64500F2BB800846A4EB0E0440EACA
:10D1600003409CE7C6F12007B34022FA07FC4CEAD3
:10D17000030C20FA07F401FA06F31C43F9404FEAC6
:10D180001C4900FA06F3B1FBF9F8200C1FFA8CFEDB
:10D1900009FB181140EA014108FB0EF0884202FA2F
:10D1A00006F20BD91CEB010108F1FF3A80F08880F0
:10D1B000884240F28580A8F102086144091AA4B2AD
:10D1C000B1FBF9F009FB101144EA014100FB0EFE2E
:10D1D0008E4508D91CEB010100F1FF346CD28E455D
:10D1E0006AD90238614440EA0840A0FB0294A1EBEE
:10D1F0000E01A142C846A64656D353D05DB1B3EB4B
:10D20000080261EB0E0101FA07F722FA06F3F1407A
:10D210001F43C5E9007100263146BDE8F087C2F121
:10D220002003D8400CFA02FC21FA03F39140014399
:10D230004FEA1C471FFA8CFEB3FBF7F007FB1036D2
:10D240000B0C43EA064300FB0EF69E4204FA02F47E
:10D2500008D91CEB030300F1FF382FD29E422DD9D1
:10D26000023863449B1B89B2B3FBF7F607FB163306
:10D2700041EA034106FB0EF38B4208D91CEB010186
:10D2800006F1FF3816D28B4214D9023E6144C91A06
:10D2900046EA004638E72E46284605E70646E3E616
:10D2A0001846F8E64B45A9D2B9EB020864EB0C0E20
:10D2B0000138A3E74646EAE7204694E74046D1E72F
:10D2C000D0467BE7023B614432E7304609E76444DD
:10D2D000023842E7704700BF02E000F000F8FEE7C6
:10D2E00072B6374880F30888364880F30988364894
:10D2F0003649086040F20000CCF200004EF634716E
:10D30000CEF200010860BFF34F8FBFF36F8F40F282
:10D310000000C0F2F0004EF68851CEF20001086025
:10D32000BFF34F8FBFF36F8F4FF00000E1EE100A95
:10D330004EF63C71CEF200010860062080F314889E
:10D34000BFF36F8FB7F022FCB6F070FC4FF0553092
:10D350001F491B4A91423CBF41F8040BFAE71D49A3
:10D36000184A91423CBF41F8040BFAE71A491B4A9C
:10D370001B4B9A423EBF51F8040B42F8040BF8E7EE
:10D3800000201849184A91423CBF41F8040BFAE7C3
:10D39000B7F000FCB6F09EFC144C154DAC4203DA1D
:10D3A00054F8041B8847F9E70AF0DEFF114C124DD0
:10D3B000AC4203DA54F8041B8847F9E7B7F0E8BB3E
:10D3C000000600200022002000C0000808ED00E058
:10D3D000000000200006002048850E0800220020E2
:10D3E000E82B0020E82B002070660120E0C1000837
:10D3F00044C2000844C2000844C200082DE9F04FAE
:10D400002DED108AC1F80CD0C3689D46BDEC108A82
:10D41000BDE8F08F002383F311882846A047002041
:10D42000B6F08AF9FEE7B5F0F1FF00DFFEE7000095
:10D4300038B510EE105A25F00044B4F1A14FF0EECB
:10D44000407A0BDBB4F1FF4F58DCDFED517A9FEDF2
:10D45000510A002DC8BFB0EE670A38BD4E4B9C4242
:10D460005BDCB4F1445F4CDB4FF0FF3267EEA76A40
:10D47000DFED4A4ADFED4A5A9FED4A5A9FED4A4A8C
:10D4800026EEA67AB0EE666AE7EE245A531CDFED6C
:10D49000474ADFED476AA5EE875AE7EE246ADFEDDB
:10D4A000455ADFED454AE6EE875AA5EE074A9FED5D
:10D4B000435ADFED436AA5EE875AE4EE074ADFEDF3
:10D4C000415AE4EE876AE5EE075A66EE866A25EE73
:10D4D000877A37D03C4B03EB820376EE876A93ED75
:10D4E000000A93ED047A96EEA70A002D70EE677A93
:10D4F00037EE670AB1DAB1EE400A38BD30EE000A05
:10D5000038BD9FED327A30EE077AF7EE006AB4EE5E
:10D51000E67AF1EE10FAA7DD38BD00F0DBF82C4B0F
:10D520009C4216DCA3F5D0039C4227DCF0EE007A87
:10D53000BFEE007AA0EE277A002230EE270AC7EE6F
:10D54000007A93E776EE876AE6EEE77AB0EE670A4E
:10D5500038BD204B9C420BDCF7EE087AB7EE007A20
:10D56000A0EE277A022230EE670AC0EE077A7DE746
:10D57000BFEE007AC7EE007A032277E7F7EE007A73
:10D5800030EE677A30EE270A0122C7EE007A6DE7A7
:10D59000DB0FC93FDB0FC9BFFFFFDF3ED769853C0B
:10D5A00059DA4B3D356B883D6E2EBA3D21A215BD33
:10D5B0006BF16EBD95879DBD2549123E388EE3BD4A
:10D5C000ABAAAA3ECDCC4CBE5C620C08CAF2497133
:10D5D000FFFF973FFFFF1B4010EE102AC2F3C75317
:10D5E0007F3B162B22F000412FDC002B18DB1A4961
:10D5F00019410A4228D0DFED197A70EE277AF5EE4C
:10D60000C07AF1EE10FA1FDD002A04DD4FF40000AD
:10D6100040FA03F31A4422EA010300EE103A70477D
:10D62000DFED0E7A70EE277AF5EEC07AF1EE10FAA1
:10D630000ADD002A06DBF7EE007A002918BFB0EEFB
:10D64000670A70479FED060A7047B1F1FF4FFBD3A1
:10D6500030EE000A704700BFFFFF7F00CAF2497139
:10D660000000008010EE103A184A23F00043934265
:10D670001BDDB3F1FF4F02DB30EE400A704700B50F
:10D6800083B0684601F0A2FB00F003000128DDED45
:10D69000010A9DED000A0CD0022812D070B10120C1
:10D6A00002F086F803B05DF804FBDFED090A01F033
:10D6B000C3BC02F07DF8B1EE400AF3E701F0BCFC18
:10D6C000F0E701F0B9FCB1EE400AEBE7D80F493FB3
:10D6D0000000000010EE103A23F0004300EE103A74
:10D6E000704700BF10EE102AC2F3C7537F3B162BC2
:10D6F00022F0004128DC002B18DB1A4919410A42AC
:10D7000021D0DFED197A70EE277AF5EEC07AF1EECE
:10D7100010FA18DD002A04DA4FF4000040FA03F38F
:10D720001A4422EA010300EE103A7047DFED0E7A48
:10D7300070EE277AF5EEC07AF1EE10FA03DD002ADA
:10D7400008DB9FED0A0A7047B1F1FF4FFBD330EEC3
:10D75000000A7047FFEE007A002918BFB0EE670A92
:10D76000704700BFFFFF7F00CAF249710000000050
:10D7700008B52DED028BF0EE408AB0EE608A00F025
:10D7800033F820B9B0EE480ABDEC028B08BDB0EE0C
:10D79000480A00F029F820B1F4EEC88AF1EE10FA38
:10D7A000F0DDB0EE680ABDEC028B08BD08B52DEDCA
:10D7B000028BF0EE408AB0EE608A00F015F820B9D6
:10D7C000B0EE480ABDEC028B08BDB0EE480A00F08E
:10D7D0000BF820B1F4EEC88AF1EE10FAF0D5B0EEF5
:10D7E000680ABDEC028B08BD10EE103A33F0004021
:10D7F0000ED0A0F50003B3F1FE4F0DD3074B421E30
:10D800009A4207D9A0F1FF40B0FA80F04009704772
:10D81000022070470320704704207047FEFF7F00FE
:10D8200010B485B08DED010A019BC3F3C751A1F17E
:10D830007F021E2A2ADC501C23DB162A4FEAD374EF
:10D840000BDDC3F3160040F400009639884004B1A4
:10D85000404205B05DF8044B7047164BDDED017A90
:10D8600003EB840393ED007A77EE277ACDED037A0C
:10D87000DDED037A77EEC77A17EE903A33F0004287
:10D880000ED1002005B05DF8044B7047DDED017A44
:10D89000FDEEE77A17EE900A05B05DF8044B70478D
:10D8A000C3F31600C3F3C75340F40000C3F196035B
:10D8B000D840CCE77C620C089FED010A704700BF9E
:10D8C0000000C07F10EE103AC3F3C7527F3A162A09
:10D8D00010EE101A15DC002A0CDB0C481041034234
:10D8E00005D04FF4800313410B4423EA000300EEFC
:10D8F000103A7047013203F00043F8D143F07E53F1
:10D90000F5E7802AF3D130EE000A7047FFFF7F0071
:10D9100010EE103A194A23F0004393421CDDB3F194
:10D92000FF4F02DB30EE400A704700B583B0684617
:10D9300001F04CFA00F003000128DDED010A9DED35
:10D94000000A0ED0022813D070B101F075FBB1EEC1
:10D95000400A03B05DF804FBDFED090A002001F086
:10D9600027BF01F069FBF4E7012001F021FFF0E798
:10D97000012001F01DFFB1EE400AEAE7D80F493F50
:10D980000000000010EE103A114A23F000439342C9
:10D9900018DDB3F1FF4F02DB30EE400A704700B5EF
:10D9A00083B0684601F012FA400000F00200DDED9D
:10D9B000010A9DED000AC0F1010001F041FF03B032
:10D9C0005DF804FBDFED030A012001F039BF00BF61
:10D9D000DA0F493F0000000008B52DED028BB0EED4
:10D9E000408A00F0ABF9144B93F900300133F0EEAC
:10D9F000408A0FD0B4EE488AF1EE10FA0AD6B0EEA3
:10DA0000480AFFF767FEF7EE007AB4EEE70AF1EE98
:10DA100010FA04DCB0EE680ABDEC028B08BD02F01F
:10DA2000E7F8BDEC028B034621221A600348BDE8EB
:10DA30000840FFF741BF00BF00220020F8840E0815
:10DA400008B52DED028BB0EE408A00F09BFA144B26
:10DA500093F900300133F0EE408A0FD0B4EE488ADB
:10DA6000F1EE10FA0AD6B0EE480AFFF733FEF7EEF1
:10DA7000007AB4EEE70AF1EE10FA04DCB0EE680AC0
:10DA8000BDEC028B08BD02F0B3F8BDEC028B03467F
:10DA900021221A600348BDE80840FFF70DBF00BF10
:10DAA00000220020F8840E0800F072BB08B52DEDAE
:10DAB000028BB0EE408A00F011FC164B93F9003057
:10DAC0000133F0EE408A12D0B0EE480A01F098FF20
:10DAD00068B1DFED117AB4EEE78AF1EE10FA12DCEC
:10DAE000DFED0E7AB4EEE78AF1EE10FA04D4B0EE70
:10DAF000680ABDEC028B08BD02F07AF82223DFED44
:10DB0000088A0360F3E702F073F82223DFED058A49
:10DB10000360ECE7002200208071B142B5F1CFC272
:10DB2000000000000000807F08B52DED028BF0EEB4
:10DB3000408AB0EE608A00F0BFFC0E4B93F90030D3
:10DB400001330BD0F4EE488AF1EE10FA06D6DFED81
:10DB50000A8AB4EE688AF1EE10FA02D0BDEC028BAC
:10DB600008BD02F045F888EEA80ABDEC028B21231F
:10DB7000036008BD002200200000000008B52DED64
:10DB8000028BB0EE408A00F027FD144B93F9003071
:10DB9000013314D0B4EE488AF1EE10FA0FD6B5EE88
:10DBA000C08AF1EE10FA0ADCB5EE408AF1EE10FA06
:10DBB00008D102F01DF822239FED090A0360BDEC95
:10DBC000028B08BD02F014F8BDEC028B0346212243
:10DBD0001A600448BDE80840FFF76EBE002200202E
:10DBE000000080FFF8840E0808B5FFF7C7FFDFEDDF
:10DBF000027A80EE270A08BD1872313F08B52DED74
:10DC0000048BF0EE408AB0EE608A00F0E5FD474BF1
:10DC100093F900300133B0EE409A1FD0B4EE488A39
:10DC2000F1EE10FA1AD6F4EE688AF1EE10FA59D62F
:10DC3000DFED3F9AF4EE698AF1EE10FA13D1B4EEFB
:10DC4000698AF1EE10FA29D0B0EE480A01F0D8FE48
:10DC500020B1B4EEE98AF1EE10FA4DD4B0EE490AE3
:10DC6000BDEC048B08BD01F0CBFEF0B1B5EE409ADF
:10DC7000F1EE10FAF2D1B0EE680A01F0C1FE002810
:10DC8000ECD0B0EE480A01F0BBFE0028E6D001F06F
:10DC9000AFFF22239FED269A0360DFE7B7EE009ADD
:10DCA000B0EE490ABDEC048B08BDB0EE680A01F085
:10DCB000A7FE0028DAD0B0EE480A01F0A1FE002845
:10DCC000D4D0B4EE499AF1EE10FA28D601F090FFC4
:10DCD000F5EEC08A2223F1EE10FA036013D49FED13
:10DCE000159ABBE7B5EE408AF7EE007AF1EE10FA2E
:10DCF00008BFB0EE679AB1E701F07AFF21239FEDEC
:10DD00000E9A0360AAE7B0EE480A01F087FEB4EE6F
:10DD1000480AF1EE10FAE2D09FED079A9EE701F073
:10DD200067FF212389EEA99A036097E7002200206C
:10DD3000000000000000807F000080FF08B510EEAA
:10DD4000102A22F00043B3F17E5F2DED028B12D03A
:10DD50000ADCB3F17C5F19DAB3F10C5F6CDCBDEC6B
:10DD6000028B9FED770A08BD70EE407A87EEA70A16
:10DD7000BDEC028B08BDBDEC028B9FED720ADFED9E
:10DD8000727A002AD8BFB0EE670A08BD002AC0F236
:10DD90009080F7EE008A38EEC00AB6EE008A20EED8
:10DDA000088AB0EE480A01F043F9DFED687A9FED8A
:10DDB000687A9FED686ADFED685ADFED686AA8EE61
:10DDC000277ADFED677AA7EE086AE8EE257AE6EEB5
:10DDD000086ADFED645A9FED647AE7EE885AA6EE92
:10DDE000887ADFED627A10EE103AE5EE887A23F455
:10DDF0007F6323F00F03B0EE476A9FED5D7AF0EE8C
:10DE0000676AA6EE087A07EE903AB0EE486AE6EE48
:10DE1000888AA7EEE76A70EE276A27EE088A86EE00
:10DE2000267AC8EE286ABDEC028BA0EE267A37EE81
:10DE3000870A30EE000A08BD20EE007ADFED437A53
:10DE40009FED436ADFED436A9FED435ADFED435A8E
:10DE5000A7EE276ABDEC028BE6EE076ADFED407A9B
:10DE60009FED406AE7EE057AE6EE875AA7EE876AED
:10DE70009FED3D5ADFED3D7ADFED3D6AA5EE875A15
:10DE8000E6EE077AE5EE076AF7EE005AE7EE875A04
:10DE900026EE877A9FED376ADFED377AC7EE256A7F
:10DEA000B0EE467AA0EE667A30EE470A37EEC00A48
:10DEB00008BDB7EE007A30EE070AF6EE007A60EEA3
:10DEC000277ADFED226A9FED226ADFED224ADFED3D
:10DED000225A9FED225A9FED268AA7EEA66ADFED11
:10DEE000206AE6EE274AE7EEA56ADFED1E5A9FEDAF
:10DEF0001E6AA4EEA75AE6EEA75ADFED1C6AA5EE4D
:10DF0000276AE5EEA76AA6EE278AA6EEA77A28EE8C
:10DF1000278AF0EE478AB0EE670A01F089F888EEAA
:10DF2000286ADFED167AB0EE407AE7EE067A9FEDCA
:10DF3000140A77EE877AF0EE006AA7EEE60A17E792
:10DF4000DB0FC93F00000000DB0F494008EF11382C
:10DF5000047F4F3A461124BD2EC69D3DA80A4E3E71
:10DF6000613330BF2D57014090B0A6BE39D119C0E2
:10DF7000ABAA2A3E6821A233DA0FC93F6821A2B3B7
:10DF8000DA0F494038B510EE105A25F00044B4F1CC
:10DF90007E5F2DED048B00F085807ADCB4F17C5F30
:10DFA0000FDAB4F1485F80F29C80DFED697A70EEA1
:10DFB000277AB7EE007AF4EEC77AF1EE10FA00F3A2
:10DFC0008D80FFF787FBF7EE007A37EEC00AB6EEDA
:10DFD000008A20EE088A9FED5F7ADFED5F6A9FED91
:10DFE0005F6A9FED5F5ADFED5F5ADFED5F8AE8EE13
:10DFF000076A9FED5E7AA8EE067A9FED5D6AA6EE4F
:10E00000885AA7EE086A9FED5B7ADFED5B6AE5EE62
:10E01000085AA6EE087AE5EE886AE7EE087AE6EE98
:10E02000888AB0EE480AB0EE679A01F001F8534BC7
:10E030009C4268EE888A42DC10EE103A23F47F633B
:10E0400023F00F0306EE903AA6EEE68A70EE267AEB
:10E0500088EE895AC8EE274A9FED497ADFED497A62
:10E06000B0EE006AA4EEC67A30EE000AF0EE675A0F
:10E07000E6EEC65A90EE057A37EE657A37EEC77A45
:10E08000002D0ADCBDEC048BB1EE477AB0EE470AF6
:10E0900038BD70EE407A87EEA77ABDEC048BB0EE07
:10E0A000470A38BD9FED367ADFED377A20EE077AE2
:10E0B000BDEC048BA0EE277AB0EE470A38BD88EE9F
:10E0C000896A9FED327ADFED307AA0EE060AF0EE33
:10E0D000006AA0EE267A37EEC77AD1E7B0EE407A32
:10E0E000DBE760EE007A9FED1B7ADFED1B6A9FEDA8
:10E0F0001C6ADFED1A5A9FED1B5AE7EE876ABDECEA
:10E10000048BA6EEA76A9FED197ADFED196AA7EED8
:10E11000A57AA6EE275AE7EE276ADFED175A9FED9C
:10E12000156A9FED117AE5EE275AA6EEA76AA5EECD
:10E13000A77AF7EE006AE6EE276A67EE277AB0EE76
:10E14000407A87EEA66AA0EE067AB0EE470A38BD9E
:10E15000CAF2497108EF1138047F4F3A2EC69D3D2F
:10E16000461124BDA80A4E3EABAA2A3E613330BFF9
:10E170002D57014039D119C090B0A6BE9999793F69
:10E180002EBD3BB3DB0F493FDB0FC93F2EBD3B33F9
:10E1900010B582B0CDED010A019B23F00042B2F12F
:10E1A000FF4FF0EE407A30DC10EE100A20F0004114
:10E1B000B1F1FF4F29DCB3F17E5F42D09C1704F030
:10E1C000020444EAD07431B37AB3B2F1FF4F40D0C5
:10E1D000B1F1FF4F29D08A1AB2F1F45F4FEAE25150
:10E1E00034DA002B42DA3C3140DA9FED340A012C5C
:10E1F0004ED0022C43D064B19FED317ADFED317AFD
:10E2000030EE070A30EE670A03E09DED017A37EE43
:10E21000270A02B010BD022C10D09FED2B0A032C50
:10E2200018BFB0EE670A02B010BD9FED280ADFEDFF
:10E23000287A0028B8BFB0EE670AEAE79FED210A06
:10E24000E7E702B0BDE81040FFF7F2B89FED1F0A04
:10E25000CDE7B1F1FF4F04F1FF3420D0022C26D8D6
:10E260001C4B03EB840494ED030AD2E79DED017A85
:10E2700087EE870AFFF72EFAFFF7DAF8B7E79FED88
:10E28000107ADFED107A30EE070A37EEC00AC0E7E9
:10E2900010EE103A03F1004300EE103AB9E7022CF9
:10E2A00008D80C4B03EB840494ED000AB1E79FED12
:10E2B000030AAEE79FED080AABE700BF00000000CD
:10E2C0002EBDBB33DB0F4940DB0F49C0DB0FC93F1D
:10E2D000DB0FC9BF84620C08DB0F493F10EE103A18
:10E2E00023F00042B2F1FF4F52D84FEAD37100F051
:10E2F0009380614883424EDC002BC0F286805F4BE6
:10E300009A424DD95E4B9A4200F299805D4A02EBE7
:10E31000810292ED004A92ED027AC1F1010330EEE2
:10E32000444A5B1A34EE470ADFED577ADFED574A6D
:10E330009FED575A9FED576ADFED575A60EE006A1E
:10E34000E6EEA74AA4EEA65AA5EE266AE6EE265AFF
:10E35000B0EE406AA5EEE66A002B47D0F0EE006A08
:10E3600060EE065A36EEC66AF7EE007A85EE860A49
:10E3700013F17D0F37EE400A30EE440A37EEC00A43
:10E3800051DB10EE102A02EBC35300EE103A704737
:10E3900030EE000A70479FED410A20EE000A7047F8
:10E3A000B2F1465F0AD2DFED3D7A70EE277AB7EE22
:10E3B000007AF4EEC77AF1EE10FA5ADC60EE007AD9
:10E3C0009FED317ADFED315A9FED316ADFED316A31
:10E3D000E7EE875A9FED307AA7EEA56AE7EE866AE8
:10E3E000B0EE406AA7EEA67AA7EEC76AF0EE007A12
:10E3F00060EE066A36EE676AB7EE007AC6EE867A97
:10E4000037EEC00A37EE400A7047254B9A427FF636
:10E4100076AF9FED240A7047DFED227A002918BFFE
:10E42000B0EE670A704710EE102A643302EBC35354
:10E43000DFED1D7A00EE103A20EE270A7047114BEF
:10E440009FED1A7A9FED1A6ADFED1A6A03EB8103DA
:10E45000D3ED047AE0EE077AB0EE404AFDEEE77ABB
:10E46000B8EEE77A17EE903AA7EE464A27EE267AFC
:10E4700058E730EE070A70471772B1421872B13E82
:10E480009115853F9C620C084CBB31330EEADDB51B
:10E4900055B38A38610B36BBABAA2A3ECAF2497122
:10E4A000B5F1CF42000000000000800D3BAAB83F4C
:10E4B0008071313FD1F7173730B583B0CDED010A08
:10E4C000019D35F0004041D010EE10EA2EF00043DF
:10E4D000B3F1FF4F3ADAB0F1FF4F37DC83423BDB59
:10E4E0000EF000443AD01EF0FF4F56D11902002919
:10E4F0006FF07D0204DD4900002902F1FF32FADCF1
:10E5000015F0FF4F57D101026FF07D0C03D4490085
:10E510000CF1FF3CFBD512F17E0F47DBCEF3160367
:10E5200043F400031CF17E0F3ADBC5F3160040F400
:10E530000000B2EB0C0204D117E00FD04B00013AFF
:10E5400013D0191A0029F8DA5B00F8E7DDED017A3B
:10E5500060EE277A87EEA70A03B030BD1D4B03EBB0
:10E56000547393ED000A03B030BD181A58BF034628
:10E570001BB9F3E75B000CF1FF3CB3F5000FF9DBCF
:10E580001CF17E0F1CDBA3F500030CF17F0C234371
:10E5900043EACC5300EE103ADEE7DA157F3AAFE7F4
:10E5A0006FF07D01A1EB0C018840C2E76FF07D01A7
:10E5B000891A8B40B6E74FEAE05CACF17F0CAAE722
:10E5C0006FF07D02A2EB0C0C43FA0CF3234300EE38
:10E5D000103AC1E7B4620C0810EE103A33F0004272
:10E5E0002ED0002B33DBB3F1FF4F40DAB3F5000F31
:10E5F00034DB4FF0000C6848C3F31601084400F404
:10E60000000282F07E520A43DB1500EE102A7F3BA7
:10E61000624A634401F10F0CF7EE007A0CEA020241
:10E6200030EE670A03EBD05322BBB5EE400AF1EEA1
:10E6300010FA60D1002B40F092809FED590A70478C
:10E640009FED587ADFED567A87EE270A704770EE15
:10E65000407A9FED537A87EE870A7047DFED527A52
:10E6600060EE277A6FF0180C17EE903AC3E730EEA1
:10E67000000A7047F0EE007A70EE277A07EE103A43
:10E6800080EE274A4948C1F55712084402F5227224
:10E690000243002A9FED463ADFED464ADFED465A37
:10E6A000DFED463A9FED465ADFED467ADFED466AEA
:10E6B00024EE046AF8EEC72A26EE067AE7EE034A4D
:10E6C000A7EE235AE4EE875AE5EE076AE5EE877A6D
:10E6D00067EE867AE6EE877A2ADDB6EE007A20EEDD
:10E6E000077A27EE007A4BBB77EE877AA7EEC47ADB
:10E6F00030EE470A7047B6EE007ADFED346AF0EE8E
:10E70000477AE0EE667A20EE007A27EE277A002B31
:10E71000EED007EE903A9FED2E6ADFED2E6AF8EE0E
:10E72000E77AA7EEC67A37EE400A97EEA60A704758
:10E7300013BB70EE677AA7EEC40A7047DFED246A58
:10E740009FED246A77EE877A62EEA66AE7EE846A26
:10E7500037EE667A37EE400A92EE860A704707EE89
:10E76000903A9FED1B0A9FED1B7AF8EEE77A27EEB1
:10E77000800AA7EE870A70479FED157ADFED156ACC
:10E7800070EE677A27EE627AA7EE847A37EE400A57
:10E7900092EEA60A704700BF20FB4A00F0FF7F0000
:10E7A00000000000000000CC0000004C305CCFFFF7
:10E7B0009788173E25333A3E2549923E4FD01C3E5E
:10E7C000298E633EABAA2A3FCDCCCC3EABAAAA3E53
:10E7D000D1F717378071313F2DE9F04710EE904A9D
:10E7E00034F000482DED028B15D010EE105A25F0B4
:10E7F0000047B7F1FF4F10EE109A06DDBDEC028B1B
:10E80000B948BDE8F047FFF757B8B8F1FF4F08DD4A
:10E81000B7F17E5FF2D1B7EE000ABDEC028BBDE826
:10E82000F087002D10EE906AC0F2F4804FF0000ADD
:10E83000B8F1FF4F00F00281B8F17E5F00F028814F
:10E84000B6F1804F00F03D81B6F17C5F00EE105ACA
:10E8500040F00181B9F1000F80F23881FEF73AFFF4
:10E86000B7F1FF4F00F00981002F00F00281B7F1EE
:10E870007E5F00F0F8804FEAD973013B5AEA030249
:10E8800000F02A81B8F19A4F40F35081974A97429D
:10E8900040F35982964A974200F3FF80F7EE007AE0
:10E8A00030EE670A9FED936ADFED935AF5EE007A3A
:10E8B000A0EE676AF6EE006AE6EE406A20EE007AA5
:10E8C000DFED8E7A9FED8E6A27EE267A67EEC77AA5
:10E8D000E0EE257AF0EE676AE0EE066A16EE902A20
:10E8E00022F47F6222F00F0207EE102AA0EE467A91
:10E8F00006EE902A77EEC77A26F47F6626F00F069A
:10E9000007EE104A06EE106A67EE877A37EE466A1F
:10E9100007EE106AE6EE267A0AF1FF3A5AEA030396
:10E9200026EE877AB7EE000A77EE876ABFEE006AB6
:10E9300016EE903A0CBFB0EE468AB0EE408A002B3D
:10E9400023F0004240F3B581B2F1864F00F3F48129
:10E9500000F0E781B2F17C5F00F3B781002210463E
:10E9600023F47F6323F00F0306EE103ADFED656AB0
:10E970009FED655A9FED652A9FED653ADFED653A9B
:10E980009FED654ADFED654A36EE477AF0EE002AE4
:10E9900077EEC77A26EE267ADFED616AA7EEA67AD1
:10E9A000F0EE476AE6EE056A66EEA65AF0EE667A83
:10E9B000A5EE823AE6EE457AB0EE636AA3EE256AEA
:10E9C00077EE677AB0EE447AA6EE257AB0EE646A06
:10E9D000A7EE256AB0EE667AA6EE657AE6EEA77A2D
:10E9E00066EE875A37EE626AB7EE005A85EE867A8F
:10E9F00077EE677A77EEE66A35EE660A10EE103A41
:10EA00001344B3F5000FC0F2B68100EE103A20EEC9
:10EA1000080A02E7B8F1974F1ADAB8F17E5F0ADB0D
:10EA20004FEAE853C3F1960348FA03F202FA03F3FC
:10EA3000434500F039814FF0000AFDE6B7F17E5FF3
:10EA40003FF4E9AE2FDD002E2ADB00EE104AE4E6AB
:10EA50004FF0020AECE6FEF73DFEB7F1FF4F02D0A1
:10EA6000002F7FF404AF002EBCBFF7EE007A87EED4
:10EA7000800AB9F1000FBFF6D0AEA7F17E5757EA72
:10EA80000A0340F00A8170EE407A87EEA70AC4E6D6
:10EA9000002E0FDB00EE105ABFE6002E00F3568169
:10EAA0009FED200AB9E6002EFADA07EE904AB1EEA1
:10EAB000670AB2E607EE105AF7EE007A87EE870A89
:10EAC000ABE607EE905A27EEA70AA6E6BDEC028B4E
:10EAD000BDE8F04700F0ACBA07EE905A77EEE77A5F
:10EAE00087EEA70A99E600BFF8840E08F7FF7F3F7C
:10EAF0000700803FABAAAA3E70A5EC363BAAB83F00
:10EB000000AAB83F8CBEBF350072313F4CBB3133D9
:10EB10000EEADDB555B38A38610B36BBABAA2A3E87
:10EB20001872313F000000000000804B19F0FF4FC9
:10EB300040F0F5805FED047A60EE277A6FF01702FF
:10EB400017EE907A8D48F915C7F316077F3987427B
:10EB5000114447F07E5240F3DA808948874240F3FF
:10EB6000FA809FED885A0131B0EE453AA2F50002D5
:10EB7000F7EE005A002006EE102A76EE257AB7EE60
:10EB8000007A87EE270A521042F0005202F58022E6
:10EB9000024476EE656A07EE901A66EE803AB8EEA9
:10EBA000E77A13EE901A07EE902A774ADFED770A9C
:10EBB0009FED778A9FED771ADFED772ADFED771AE1
:10EBC0009FED772A77EEE55A114004EE901A36EE63
:10EBD000656A63EEA35AE4EEE76AF0EE607AE5EE6A
:10EBE000887AE4EEC66AA7EEA51A66EE806AE1EEC0
:10EBF000252A73EEA47AE2EEA51A25EEA58AA1EEE7
:10EC0000A52A67EEA67AB0EE084AB0EE446AE8EEAE
:10EC1000027AA4EEA46ADFED630A9FED631ADFEDCA
:10EC2000632A36EE276A16EE101A114006EE101A05
:10EC300076EE445AE4EEE45A77EEE57A67EEA37A8C
:10EC4000E6EE867AF0EE675AE4EE865A15EE901AF2
:10EC5000114006EE901AE4EEC66A05EE901A77EEC1
:10EC6000E67A67EEA07AE5EE817A77EE837AF0EEC7
:10EC7000676AE5EEA26A76EE856A76EE876A16EE38
:10EC8000901A114006EE901A36EEC77A37EE457AA2
:10EC9000A5EEE27A77EEC77A2EE6BAF1010F7FF49D
:10ECA000BCADB1EE400AB8E502F00102C2F1020AC1
:10ECB000C2E53F498A4257DC7FF44CAE76EEC76A24
:10ECC000F4EEE76AF1EE10FA4EDAD2154FF40001D5
:10ECD0007E3A41FA02F21A44C2F3C751354C7F39E9
:10ECE0000C41C2F3160022EA040206EE902A37EE27
:10ECF000667A40F40000C1F117010841002B77EE5D
:10ED0000876AB8BF404216EE903AC20528E69FEDEA
:10ED10001D5AF7EE005AB0EE453A00202BE70022CC
:10ED200010E79FED256A76EEC76A37EE866AB4EE85
:10ED3000E66AF1EE10FAC8DDDFED207A28EE270A48
:10ED400020EE270A69E5002EBFF6AAAE9FED1B0A4A
:10ED500020EE000A61E59FED1A5A9FED1A3AF7EE90
:10ED6000085A4FF4001006E7DFED177A28EE270A5D
:10ED700020EE270A51E500F0AFFE48E671C41C0002
:10ED8000D6B35D000000000000F0FFFF55326C3E7E
:10ED900042F1533E05A38B3EABAAAA3EB76DDB3EC4
:10EDA0009A99193F4F38763FA0C39D360038763F79
:10EDB00000001643FFFF7F003CAA3833CAF24971B6
:10EDC00000C0153FDCCFD1356042A20D70B510EE0A
:10EDD000103A894A23F00044944286B0054670DD1B
:10EDE000864A944210EE106A22DC002BDFED847A12
:10EDF000844A24F00F04B0EE407A40F3E480944259
:10EE000070EE677A09BFDFED806A9FED807A9FED33
:10EE1000807A77EEE67A012077EEC76A77EEE67AB7
:10EE2000C5ED006A77EEC77AC5ED017A06B070BD10
:10EE3000784A944254DDB4F1FF4F49DAE215863A3C
:10EE4000A4EBC25307EE903ABDEEE77ADFED726AAB
:10EE5000B8EEC77A77EEC77A8DED037A67EEA67AB9
:10EE6000BDEEE77AB8EEC77A77EEC77A8DED047A11
:10EE700067EEA67AF5EE407AF1EE10FACDED057A5E
:10EE800040F09080B5EE407AF1EE10FA14BF022304
:10EE90000123624901910221009103A8294600F053
:10EEA0004DF9002EC2DA95ED007AD5ED017AB1EE7A
:10EEB000477AF1EE677A85ED007AC5ED017A404236
:10EEC000B4E7002285ED000A4260002006B070BD64
:10EED00070EE407A0020C5ED017AC5ED007AA5E715
:10EEE000FEF7F8FB9FED4E7A9FED456AF6EE007A4D
:10EEF000E0EE077A9FED457AFDEEE77A17EE900A8D
:10EF0000F8EEE76A1F28A6EEC60A66EE877AB1EE2B
:10EF1000666A1EDC434A411E24F0FF0352F821209A
:10EF2000934216D030EE677A85ED007A30EE470ACC
:10EF3000002E30EE670A85ED010ABFF677AFB1EE1D
:10EF4000477AB1EE400A85ED007A85ED010A40422C
:10EF50006CE730EE677AE21517EE103AC3F3C75349
:10EF6000C3EBD454082CDFDDDFED277A9FED287A40
:10EF7000F0EE405AE6EE275A30EE650AA6EE270A72
:10EF8000F0EE407AD6EE877A35EEE77A17EE103A51
:10EF9000C3F3C753D21A192A06DCB0EE650A85ED11
:10EFA000007AC3E7032374E79FED1F7A9FED1F5A92
:10EFB000B0EE650AA6EE070A75EEC07AE6EE077AAD
:10EFC000D6EE857AAEE7944270EE277A09BFDFED80
:10EFD0000E6A9FED0E7A9FED0E7A77EEA67A4FF0CD
:10EFE000FF3077EE876A77EEE67AC5ED006A77EE56
:10EFF000877AC5ED017A19E7D80F493FE3CB164070
:10F00000800FC93FD00FC93F0044353743443537DF
:10F0100008A3852E800F4943000080433C630C0801
:10F0200084F9223FBC620C0800A3852E32318D2466
:10F03000B1EEC00A704700BF10EE103A23F0004353
:10F04000B3F1485F2CDAFDEEC07A17EE903A002B50
:10F0500060D020EE007ADFED317A9FED315ADFED9E
:10F06000315A9FED316ADFED316AA7EE275ADFEDA5
:10F07000307AE7EE055AA7EE256AE7EE067AE7EE64
:10F08000276A67EE266A60EEC00AF6EE007AE7EEBF
:10F09000260AB7EE000AD7EE270A30EE600A70475C
:10F0A00020EE007ADFED1D7A9FED1D5ADFED1D5A2F
:10F0B0009FED1D6ADFED1D6A1E4AA7EE275A934297
:10F0C000DFED1B7AE5EE075AA5EE876AE6EE077AD2
:10F0D000E7EE876A66EE876AD5DD174A934214DC4D
:10F0E00003F17F4307EE903AB7EE006A36EE676AA7
:10F0F00060EEC00AF6EE005AD7EE257AE7EE260A51
:10F1000077EEE00A36EE600A7047B6EE076AF5EE73
:10F11000027AEDE7B7EE000A704700BF4ED747AD61
:10F12000F6740F317CF293B4010DD037ABAA2A3DAF
:10F13000610BB6BA9999993E0000483F2DE9F04F0E
:10F140002DED048BDBB01C4603930691A24B68990E
:10F15000089253F82150111D824604F1FF38C0F285
:10F16000A382D31E48BF131DDB1002930133DB00C3
:10F170000793DDE907239B1A0593029B15EB080112
:10F18000A3EB080316D401319FED947A69981944D2
:10F190001EAA002BA4BF50F8234007EE904A03F1AB
:10F1A0000103ACBFF8EEE77AF0EE477A8B42E2EC6F
:10F1B000017AEED1002DC0F2E782039B1EAA02EB7A
:10F1C000830446AE4FEA830C4046EF180AEB8301F6
:10F1D000B8F1000FDFED817A09DB22465346F3ECEC
:10F1E000016A32ED017A8B42E6EE877AF7D101307F
:10F1F000B842E6EC017A04F10404E9D109AB0AAFA4
:10F2000003EB850907EB8503083B9FED769ADFED5D
:10F21000748A059804930AEB0C0446AE00955AAB29
:10F2200003EB8503002D13ED140A4FEA850B16DD61
:10F2300006EB85033A4660EE097AB0EE407AFDEEC1
:10F24000E77A73ED016AF8EEE77AB342A7EEE87A5F
:10F2500037EEA60ABDEEC77AA2EC017AEBD1019097
:10F2600000F03AFCB0EE408AB4EE000A28EE000A44
:10F27000FEF738FAF2EE007AA0EE678A01980028CD
:10F28000FDEEC89AF8EEE97A38EE678A79DD05F185
:10F29000FF3EC0F1080357F82E1041FA03FC0CFAA8
:10F2A00003F3CB1AC0F1070219EE901A43FA02F2E7
:10F2B0006144002A47F82E3009EE901A69DCB5EE59
:10F2C000408AF1EE10FA40F0C080009B05F1FF3B50
:10F2D0005B4510DC05F18043013B07EB8303002114
:10F2E000944653F804294B4541EA0201F9D162469C
:10F2F000002940F0F280009B013B57F82330002B9F
:10F3000040F0E780049B4FF0010C53F804290CF106
:10F31000010C002AF9D06B1CAC449E46039A51198B
:10F32000029A02EB030B0BF1804B699A0BF1FF3B46
:10F3300006EB83051EAB02EB8B0B03EB8101DBEDD0
:10F34000017A9FED267AF8EEE77AB8F1000F0BF11B
:10F35000040BC1ED007A0A4601F1040109DB5346B2
:10F3600001E072ED017AF3EC016AA342A6EEA77AFE
:10F37000F7D10EF1010EE645A5EC017ADFDD654619
:10F380004DE740F09C806B1E57F823201212002A94
:10F3900095DD19EE903A002D03F1010309EE903A44
:10F3A00040F39881396800297FD1012D26D03B4652
:10F3B0004FF0010C53F8041F00297AD00CF101031F
:10F3C000C1F580719D4247F82C1016DD57F82310C7
:10F3D000BB4407EB83030AE054660C0800000000FE
:10F3E000000080430000803B0000C93F1968C1F164
:10F3F000FF0143F8041B5B45F8D1012100280CDD17
:10F40000012800F04881022807D105F1FF3C57F898
:10F410002C3003F03F0347F82C30022A7FF44FAF23
:10F42000B7EE000A30EE488A00293FF448AF09924F
:10F43000019000F051FB38EE408A099A0198B5EE30
:10F44000408AF1EE10FA3FF440AF0292DDE9073254
:10F45000B0EE480A981A0195009D00F03DFB1FEDA3
:10F46000207AB4EEC70AF1EE10FADDE90132C0F2FB
:10F4700059815FED247A059960EE277A0831FDEE17
:10F48000E77A0591F8EEE77A03F1010BA7EEC70AD8
:10F49000FDEEE77ABDEEC00A10EE101A47F8231011
:10F4A00017EE903A47F82B302EE001234FF0000C76
:10F4B00086E70CF1010CAC457FF47CAF9EE7F6EEDD
:10F4C000007AB4EEE78AF1EE10FA80F2F2800022C0
:10F4D000F5E66B1C9E469C4620E70599A1F10800C5
:10F4E00057F82B1005902B46009D69B903F1804316
:10F4F000023B07EB8303014653F804090BF1FF3B82
:10F5000008390028F8D0059105980092B7EE000A56
:10F5100000F0E2FABBF1000F009AC0F228814FEA36
:10F520008B0E46AB03EB0E060EF1040C1FED537A67
:10F5300007EB0C03311D73ED017AF8EEE77ABB425D
:10F5400067EE807A20EE070A61ED017AF3D1002D93
:10F550001FED5B6A4FF0000420DB9348DFED937AE8
:10F56000B0EE467A3146002303E09C4208DBB0EC63
:10F57000017AF1EC016A01339D42E6EE877AF4DA12
:10F580005AAB03EB8403A34543ED287AA6F10406A6
:10F5900004F1010305D0002D1C46DEDADFED837A8D
:10F5A000EEE7689902291CDC002900F395800FD151
:10F5B00032ABDFED7E7A9C443CED017A634577EE19
:10F5C000877AF9D10AB1F1EE677A069BC3ED007A2A
:10F5D00019EE903A03F007005BB0BDEC048BBDE878
:10F5E000F08F689B032BF3D1BBF1000F00F0D480A8
:10F5F0000EF5B4736B4432A913ED287A01EB8B033B
:10F6000073ED017AF0EE476A37EE277A994277EE8A
:10F61000C77A83ED007A77EEA67AC3ED017AEFD14F
:10F62000BBF1010F40F3B8800BF1804B0EF5B473C2
:10F630000BF1FF3B0DEB030E4FEA8B0B0BF10403B9
:10F640001EED287A0B4433A873ED017AF0EE476A79
:10F6500037EE277A984277EEC77A83ED007A77EE15
:10F66000A67AC3ED017AEFD10BF1080BDFED4F7AEB
:10F6700001EB0B03083133ED017A994277EE877A7B
:10F68000F9D1002A56D10699329A339B0A604B6011
:10F69000C1ED027A9CE705F1FF3C57F82C3003F0EE
:10F6A0007F0347F82C30B8E6082307930023029322
:10F6B0005FE519EE903A002D03F1010309EE903A4F
:10F6C000C8BF02223FF76EAEF7EE007A37EEC88A67
:10F6D0000222F4E5002191E632A9DFED347A01EB54
:10F6E000830333ED017A994277EE877AF9D19DED64
:10F6F000327A8ABB069BBBF1000FC3ED007A77EE2E
:10F70000677A0BDD33A90123B1EC017A01339B4504
:10F7100077EE877AF8DA0AB1F1EE677A069BC3EDE5
:10F72000017A55E7BDEEC00A9B4610EE101A47F865
:10F730002310E9E6DDED326A9DED337A069BF1EEAA
:10F74000666AB1EE477AF1EE677AC3ED006A83ED3F
:10F75000017AC3ED027A3BE7069BF1EE676ABBF1E3
:10F76000000F77EE677AC3ED006ACBDCD4E7689BC5
:10F77000022B0DDC002B14DC7FF42AAFDFED0B7ABB
:10F78000002A3FF422AF1EE7039B4FEA830C35E5C6
:10F79000689B032B7FF41CAFDFED047A002AC9D1EC
:10F7A00071E7DFED027AA2E764660C080000000052
:10F7B00010EE103A23F00043B3F1485F04DAFDEE97
:10F7C000C07A17EE903A5BB360EE007A9FED157A3F
:10F7D000DFED155A9FED156ADFED156AE7EE875AE2
:10F7E0009FED147AA5EEA76A20EE275AE6EE276A67
:10F7F000A6EEA77A30B9DFED106AE7EE876AA6EECB
:10F80000850A704727EE457AF6EE006AA0EEA67AE2
:10F81000DFED0A6AD7EE270AE5EE260A30EE600A27
:10F82000704700BFD3C92E2F342FD7B21BEF383605
:10F83000010D50B98988083CABAA2ABEABAA2A3E62
:10F8400008B510EE103A23F00042B2F1465FF0EE38
:10F85000407A0FDABDEEC07A17EE101A01BB431CD6
:10F86000134300F0A080012803D0BFEE007A87EE9A
:10F87000270A08BD50498A4212DB002BB8BFF1EEBF
:10F88000407A9FED4E7A9FED4E0AB8BFF1EE600AC6
:10F8900070EE677A37EE600ADFED4A0A70EE277A7B
:10F8A00067EEA76ADFED484ADFED485A9FED485AF8
:10F8B0009FED486A404926EEA67A8A42E7EE245A2E
:10F8C000A7EE056ADFED444A9FED445AE5EE874A0C
:10F8D000A6EE075ADFED425A9FED426AE4EE875AE0
:10F8E000A5EE076ADFED404A9FED405AE5EE874AF4
:10F8F000A6EE075A9FED3E6ADFED3E5AA4EE876AF8
:10F90000E5EE075AB0EE467AA5EEA67A27EEA65A9D
:10F91000B0EE606AA7EE056ADFED374AE6EE260A2A
:10F92000E5EE240A37EEA00A1FDA0128A1D0BFEEC7
:10F93000007AC7EE006A314B10EE102A1A4006EE2C
:10F94000102A16EE902A76EE677A134000EE103AEF
:10F95000B7EE007A70EEE70AF0EE477AE6EE007A4C
:10F96000E0EE807AA7EEA60A08BD07EE100AB8EE10
:10F97000C77A60EE005A30EE070A9B17C5EE806A20
:10F9800003F00203C3F10103B0EE006A76EEE00A71
:10F9900000EE103A77EEE07AB8EEC00AA7EEC67A2B
:10F9A00020EE070A08BDFDF795FEB7EE007AF0EEEF
:10F9B000407A87EE270A08BD40A12C3F68212233F8
:10F9C000DA0F493F000000005FAE9BB745F4A33853
:10F9D0008453D9377AC09538C8261A3AB93781394D
:10F9E00016696B3B48DEBE3AA427B33C1F37113C77
:10F9F0008988083ED10D5D3DABAAAA3E00F0FFFF0D
:10FA000082B08DED010A019820F00040B0F1FF4F67
:10FA1000ACBF0020012002B0704700BF10EE101AEA
:10FA2000C1F3C753A3F17F02162A21F0004325DC5E
:10FA300053B3002A82B04FEAD17026DB244B134126
:10FA4000194219D04FEA530C11EA530307D04FF46F
:10FA5000001321EA0C0113410B4300EE103A1D4B39
:10FA600003EB8003D3ED007A37EE800A8DED010AB7
:10FA70009DED010A30EE670A02B07047B3F1FF4F07
:10FA800002D330EE000A70477047124AC1F31603E2
:10FA90005B4202EB80005B0A0A0D03F4800312054F
:10FAA000134307EE903AD0ED006A36EEA77A01F0E4
:10FAB00000418DED017ADDED017A77EEE67A17EE01
:10FAC000903A23F000430B4300EE103AD4E700BF16
:10FAD000FFFF7F008C660C0882B08DED010A019B50
:10FAE00033F000422AD0B2F1FF4F23D213F0FF4F80
:10FAF00028D19DED017ADFED2A7A2A4B67EE277A2D
:10FB00009842CDED017A37DB019BC3F3C752193A16
:10FB10000244FE2A1ADD9FED240A9FED247A019B00
:10FB2000002BF0EE407AB8BFB0EE470A20EE270A6D
:10FB300002B0704730EE000A02B070479DED010A36
:10FB400002B07047D20D0244FE2AE4DC002A0BDC2E
:10FB500012F1160F17DA4CF250339842DBDC9FEDAE
:10FB6000140A9FED147ADAE723F0FF4343EAC25305
:10FB700000EE103A02B070479FED0D0ADDED017AFC
:10FB800027EE800AD8E7193223F0FF4343EAC25335
:10FB9000DFED097A07EE103A27EE270ACCE700BF1F
:10FBA0000000004CB03CFFFFCAF24971CAF249F1B3
:10FBB0006042A20D6042A28D00000033002102F0DD
:10FBC00091BD00BF0A22002102F038BF0A230022A3
:10FBD00002F014BF10B5054C34B113460A46014675
:10FBE0000220AFF3008010BD204610BD00000000D1
:10FBF000014B1868704700BF04220020F8B5D0E917
:10FC00000067634A00230C4630463946FDF74AF93F
:10FC10005F4A0546394630460023FDF743F9002A7E
:10FC2000C0F2AC8005F52F2303F66C235948A0FBE6
:10FC30000250C00A4FF4616101FB10225649A060D6
:10FC4000A1FB0201490955486160C1EB0111A2EB1A
:10FC50008102D91C80FB015008442260CA17C2EB04
:10FC6000A002C2EBC2028A1A48BF0732002BA2616F
:10FC700079DB4B4AD91782FB0302C1EBE2314948D9
:10FC8000494A4A4E00FB01308508A2FB053200EBD1
:10FC9000D222A6FB0535464BA2EBD5120509A3FBE4
:10FCA0000535A2EB1512434DA5FB023CA2EB0C035C
:10FCB0000CEB530C404D9308A6FB03234FEA1C2288
:10FCC000A5FB0265DB09C3EB5513034440F26D103D
:10FCD00000FB123303EB830538480235A0FB050C0B
:10FCE0004FEADC1C40F2F9560CEBCC00B54200EBBD
:10FCF0000010334D00F10200A5FB00504FF4C87610
:10FD000094BF02256FF0090506FB01216544012D12
:10FD100098BF01315E1CB3F5997FA6EB90000BD321
:10FD2000A3F59973A1F26C71E3610023E060C4E96B
:10FD3000045123622046F8BD96070BD0214E06FBE6
:10FD400002F2214EB6EB321F2CBF012200223B33C0
:10FD50001344E7E71B4E1D4F02FB06F6B7EBB60F49
:10FD6000ECD20122F3E70E49A3F50E32A2F52C7274
:10FD700081FB0201D217C2EBE13180E702F5A83224
:10FD800005F52F2302F5C07203F66B234EE700BF83
:10FD900080510100C5B3A291898888889324499233
:10FDA000BD066B394FC5FDFF7F206B39D97CC65925
:10FDB00041D6720061F319671F85EB51D7802BD6AE
:10FDC000CDCCCCCC295C8FC20AD7A300285C8F0293
:10FDD000024B1844407800F008007047E8660C08B1
:10FDE00001F0FF01102A2BDB10F0070F08D010F8EC
:10FDF000013B013A8B422DD010F0070F42B3F6D1F0
:10FE0000F0B441EA012141EA014122F007047FF008
:10FE100000070023F0E80256083C85EA010586EA5F
:10FE2000010685FA47F5A3FA87F586FA47F6A5FA9B
:10FE300087F68EB9EED1F0BC01F0FF0102F00702A7
:10FE400032B110F8013B013A83EA010313B1F8D152
:10FE50000020704701387047002D06BF3546033833
:10FE6000073815F0010F07D1013015F4807F02BF6C
:10FE7000013015F4C03F0130F0BC0138704700BFBD
:10FE8000032A70B515D940EA010C1CF0030F044693
:10FE90000B4621D1194620460E680568B54204F18B
:10FEA000040403F1040317D1043A032A2046194637
:10FEB000F0D8541EA2B100F1FF3C013901E0C31893
:10FEC0000CD01CF801EF11F8012F9645A4EB0C03A0
:10FED000F5D0AEEB020070BD541EECE7184670BDC5
:10FEE000104670BD844641EA000313F003036DD150
:10FEF000403A41D351F8043B40F8043B51F8043BED
:10FF000040F8043B51F8043B40F8043B51F8043BF3
:10FF100040F8043B51F8043B40F8043B51F8043BE3
:10FF200040F8043B51F8043B40F8043B51F8043BD3
:10FF300040F8043B51F8043B40F8043B51F8043BC3
:10FF400040F8043B51F8043B40F8043B51F8043BB3
:10FF500040F8043B51F8043B40F8043B51F8043BA3
:10FF600040F8043B51F8043B40F8043B51F8043B93
:10FF700040F8043B403ABDD2303211D351F8043B33
:10FF800040F8043B51F8043B40F8043B51F8043B73
:10FF900040F8043B51F8043B40F8043B103AEDD2E2
:10FFA0000C3205D351F8043B40F8043B043AF9D233
:10FFB000043208D0D2071CBF11F8013B00F8013B06
:10FFC00001D30B8803806046704700BF082A13D313
:10FFD0008B078DD010F003038AD0C3F10403D21A2B
:10FFE000DB071CBF11F8013B00F8013B80D331F85F
:10FFF000023B20F8023B7BE7043AD9D3013A11F8DF
:020000040801F1
:10000000013B00F8013BF9D20B7803704B78437049
:100010008B788370604670472DE9F04F012BADF26D
:100020001C4D07468A46154640F21F814FF00109D4
:10003000002448464FF0FF364A4606E0A2EB060988
:1000400014460120221893420FD9A91915F802C0AD
:10005000095C8C45F2D300F08C804FF001092646F4
:1000600048464C4422189342EFD84FF0010E00242A
:1000700070464FF0FF3C724606E0A2EB0C0E1446B1
:100080000120221893420FD905EB0C0115F80280CC
:10009000095C8845F1D872D04FF0010EA446704635
:1000A000744422189342EFD80CF1010C01366645D6
:1000B00001D8F146664605AA0DF2144142F8043F04
:1000C0008A42FBD1002B00F0CB805C1E691E05EB41
:1000D000040C0DF1180811F8010FCA431A442A4400
:1000E000614548F82020F6D1324605EB0901284643
:1000F0000193FFF7C5FE019B002868D1AAEB03011D
:10010000A3EB0903024602930346701E0590C6F155
:100110000100CDE903908A4601950AE022B1039AD5
:100120009142029A38BF11460B4453454FF00002EA
:1001300048D807EB030B1BF8041058F821100029CE
:10014000ECD1B242114638BF3146A1421DD20198CE
:100150004D1E05445818384402E00131A14214D222
:1001600010F801CB15F801EFE645F6D0049A1344D8
:10017000DAE7814512BF01304C44012062E7704547
:100180000ABF2418013001207BE7B242059972D2E0
:10019000019D98193844354402E08A425ED0614698
:1001A00010F801CD15F801EDE64501F1010901F165
:1001B000FF3CF2D001324A455BD8039A13445345C1
:1001C000029AB6D900200DF21C4DBDE8F08FAAEBC3
:1001D000030A9B1BB34238BF33464FF0000901337B
:1001E00007EB09000293C6F101030193035D58F880
:1001F000233006F1FF3B4BB19944D145E2D807EBE0
:100200000900035D58F82330002BF5D1A64213D224
:1002100006EB09023A4405EB0B01334602E00133D9
:10022000A34209D212F801CB11F801EFE645F6D04E
:10023000019A91449944E0E7002EC4D006EB0901ED
:100240003944AA1901E0AB42BDD012F801ED11F812
:1002500001CDE6451346F6D0029BCDE79146A9E7CE
:100260004FF0FF340DF118083EE74FF0010900266A
:1002700021E75846A7E7B1469CE700BF2DE9F047C4
:100280000446C0B0002B69D0012B0D4690461F4696
:1002900000F087808B425DD8CD1A022B00EB05065B
:1002A00060D0B3F5807F00F2838000214FF480722C
:1002B00068465D1E00F0FEF8404601210246437884
:1002C0001278A3EBC203DBB201300DF80310013149
:1002D0008D42F3D808EB07034FF0000A13F8022C05
:1002E00018F80530A3EBC203DBB21DF803900DF83C
:1002F0000350A5EB0909B44201D92BE063B92C44A2
:10030000A64214F8013C94F800C0ACEBC30C5FFAB1
:100310008CFC1DF80C30F1D29D42A4EB0304EAD80A
:100320000F2D07D9042208EB0A0104EB0A00FFF79E
:10033000A7FD60B92A4641462046FFF7A1FD68B1F6
:10034000BAF1030F8CBFAAF1040AA7F1050A4C44C5
:10035000B442D4D9002040B0BDE8F087204640B078
:10036000BDE8F08713785578017845EA03450346E0
:1003700013F8012F9E4242EA01421DD39542EDD06F
:10038000013601E09542E6D0184613F8011FB3424A
:1003900041EA0242F6D1954208BF06F1FF30D9D1B9
:1003A000D9E711782A4640B0BDE8F047FFF718BDFD
:1003B00040B0BDE8F0472FE61E46ECE788420DD975
:1003C0008B1883420AD900EB020CBAB1624613F8CB
:1003D00001CD02F801CD9942F9D170470F2A0ED80C
:1003E000034602F1FF3C4AB10CF1010C013B8C4485
:1003F00011F8012B03F8012F6145F9D1704740EA4C
:1004000001039B0750D1A2F1100370B501F1200C3C
:1004100023F00F0501F1100E00F11004AC441B098C
:100420005EF8105C44F8105C5EF80C5C44F80C5C00
:100430005EF8085C44F8085C5EF8045C44F8045C10
:100440000EF1100EE64504F11004E9D1013312F06B
:100450000C0F01EB031102F00F0400EB031327D084
:10046000043C24F003064FEA940C1E441C1F8E46E5
:100470005EF8045B44F8045FB442F9D10CF1010466
:1004800002F0030203EB840301EB840102F1FF3C61
:100490004AB10CF1010C013B8C4411F8012B03F81B
:1004A000012F6145F9D170BD02F1FF3C03469BE786
:1004B0002246EBE7830730B548D0541E002A3FD0D0
:1004C000CAB2034601E0013C3AD303F8012B9D0771
:1004D000F9D1032C2DD9CDB245EA05250F2C45EADB
:1004E000054536D9A4F1100222F00F0C03F1200EBD
:1004F000E6444FEA121C03F1100242E9045542E9B6
:10050000025510327245F8D10CF1010214F00C0FB3
:1005100003EB021204F00F0C13D0ACF1040323F030
:1005200003030433134442F8045B9342FBD10CF001
:1005300003042CB1CAB21C4403F8012B9C42FBD12A
:1005400030BD64461346002CF4D1F9E70346144647
:10055000BFE71A46A446E0E72DE9F04757EC106BD9
:1005600084B0002F0C46DDE90CA9904619465FDBEC
:100570000025B9F1660F0D701AD0B9F1460F17D0EA
:1005800029F02003452B36D003AA019202AA00923B
:1005900047EC106B53462246022102F0C3FBB9F12F
:1005A000670F054634D118F0010F34D1039B1BE0CF
:1005B00003AB019302AB009347EC106B534622460A
:1005C000032102F0AFFB054600EB04082B78302B2B
:1005D00033D0DAF800404444304639460022002344
:1005E000FCF772FAC8B123460E9A5B1B28461360CB
:1005F00004B0BDE8F08703AA0192013402AA009278
:1006000047EC106B53462246022102F08BFB054655
:10061000B9F1470FC7D02C44DEE7039B9C42E3D9D6
:1006200030215A1C03921970039BA342F9D3DBE7D4
:1006300007F100432D251F469BE70022002330468B
:100640003946FCF741FA0028C3D1C4F10104CAF8C5
:100650000040C0E7F0B5002983B002703FDB841C86
:100660002B230929437030DD0DF107051F4FAC46E0
:1006700087FB0132CB17C3EBA20303EB8302A1EB91
:1006800042020E463032632EE6460CF8012C194623
:100690000CF1FF3CECDC3031AEF10203C9B29D42FB
:1006A0000CF8011C1FD96346224601E013F8011B18
:1006B00002F8011BAB42F9D10DF10903A3EB0E0EB9
:1006C000A644AEEB000003B0F0BD3023A6461944AB
:1006D0000EF8023B6170AEEB000003B0F0BD494282
:1006E000841C2D23BDE7A646F5E700BF6766666656
:1006F0002DE9F04F2DED028B8DB00C46DDF86080BA
:1007000016461F46054603F0FDFE0368184608EE30
:10071000103A00F0CDFE00230A93D8F8003007907D
:10072000073323F0070303F10802D4F800B094F86C
:1007300018A0C8F80020D3E9008929F000430593E8
:10074000CDF81080C4E91289DDE90401A74B4FF010
:10075000FF32FCF7EBF948B9DDE90401A34B4FF098
:10076000FF32FCF7C5F9002800F0928042464B4664
:1007700040464946FCF7DAF9002840F034826168C7
:100780004B1C2DD0BAF1670F68D0BAF1470F65D076
:100790004BF480620023226003930AAB029309ABFF
:1007A00049EC108B0093CDF804A00DF123032846EB
:1007B000FFF7D2FE8046BAF1650F099934D80139A6
:1007C000524604F150000991FFF744FF0A9A1318AA
:1007D000012A8146236140F37E810133236135E0A4
:1007E000062161604BF480620023226003930AAB10
:1007F000029309AB49EC108B0093CDF804A00DF1E6
:1008000023032846FFF7A8FE0AF0DF03472B8046A4
:10081000D1D10999C81C80F2FE80AAF1020A5FFAC0
:100820008AFABAF1650FCAD9BAF1660F00F0FA80F8
:100830000A9B8B4240F301810029D4BFC1F102021F
:10084000012213442361A1654FF000099DF8233074
:10085000002B35D02D2384F8433031E0002900F0FF
:1008600023814BF480620023226003930AAB02933E
:1008700009AB49EC108B0093CDF804A00DF12303D4
:100880002846FFF769FE09998046C81CC5DBC2E00F
:100890004046494600220023FCF720F910B12D23E1
:1008A00084F84330524B53482BF00402BAF1470FFF
:1008B00094BF984680460323226023614FF00009CD
:1008C000009733460BAA2146284600F0ABF90130C9
:1008D00025D02368580531D423694246314628463D
:1008E000B84701301BD02368E06813F0020F0B9B60
:1008F0001CD0C21A002A19DD04F119094FF00008B2
:1009000004E0E0680B9BC21A42450FDD01234A4612
:1009100031462846B847013008F10108F1D14FF0BF
:10092000FF300DB0BDEC028BBDE8F08F9842B8BF30
:1009300018460DB0BDEC028BBDE8F08FBAF1650F23
:1009400032D9D4E9120100220023FCF7BDF80028B7
:100950007BD0294A012331462846B8470130DED0F2
:10096000DDE909239A4202DB2368D907BCD5079B3E
:1009700018EE102A31462846B8470130CFD00A9BDE
:10098000012BB0DD04F11A094FF0000803E00A9BC7
:10099000013B4345A7DD01234A463146284698449A
:1009A000B8470130F3D1BAE70A9A012A7FDD012363
:1009B000424631462846B8470130B0D0079B18EE72
:1009C000102A31462846B8470130A8D0D4E9120190
:1009D00000220023FCF778F8002877D00A9B012B2F
:1009E00070DD04F11A0A4FF000080BE0FFFFEF7F03
:1009F000B0830E08B4830E08C0830E080A9B013B27
:100A000043455FDD01235246314628469844B847A6
:100A10000130F3D183E7636899423FF7FEAE4FF0B0
:100A2000670A05E700295BDD63682161002B00F0A0
:100A3000898001330B44236105E723682161DB07CB
:100A40007FF501AF4B1C2361FDE6099B002B4FDDB9
:100A50000A9BD4F858A05345A8BF5346002B9B4689
:100A600008DD424631462846B84701303FF457AFCB
:100A7000D4F858A02BEAEB7BAAEB0B03002B6EDD1E
:100A800004F11A024FF00009924604E0A36DA3EBB3
:100A90000B024A4562DD01235246314628469944FD
:100AA000B8470130F2D13AE7012161609AE6DB07ED
:100AB0003FF57DAF4246012331462846B847013015
:100AC0003FF42DAF4B4604F1500207E70A9B08F1B3
:100AD0000102013BF0E72268D2077FF5B7AE7CE662
:100AE0006368002B33D12268D20730D40123A9E6F2
:100AF000494A012331462846B84701303FF40FAF39
:100B0000DDE90923134324D0079B18EE102A314650
:100B10002846B84701303FF402AF099B002B77DA33
:100B200004F11A0A4FF0000903E0099B5B424B45B0
:100B30006EDD01235246314628469944B8470130BC
:100B4000F3D1ECE62268D0077FF57DAE71E7023382
:100B500078E62368DA077FF5C7AED5E79A46DDE980
:100B600009218A4202DB2368D8070AD5079B18EEC1
:100B7000102A31462846B84701303FF4D0AEDDE9AF
:100B80000921A1EB0A098A1A9145A8BF9146B9F13A
:100B9000000F0BDD08EB0A024B4631462846B847EA
:100BA00001303FF4BCAEDDE90932D21A29EAE97915
:100BB000A2EB0903002B7FF796AE04F11A0A4FF05F
:100BC000000807E0DDE909239B1AA3EB090343456D
:100BD0007FF789AE01235246314628469844B847EC
:100BE0000130EFD19BE64B46002BBCBF2D2384F890
:100BF00043302BF00403094A2360094BBAF1470F35
:100C000094BF90469846032323614FF0000957E6AE
:100C10000A9B424662E600BFC0830E08B8830E08F6
:100C2000BC830E082DE9F84F92461F460A698B686F
:100C3000DDF828909A42B8BF1A46CAF8002091F809
:100C400043300C46064613B10132CAF80020226830
:100C500091065DD5DAF800300233CAF80030226818
:100C600012F0060F11461ED1E168CB1A002BD8BF37
:100C7000114618DD04F1190B4FF0000805E0E56896
:100C8000DAF80030ED1A45450CDD01235A463946A5
:100C90003046C847013008F10108F0D14FF0FF306D
:100CA000BDE8F88F216894F84330003B18BF01235A
:100CB0008A060AD5E1185A1C302081F843002244E4
:100CC00094F8451082F84310023304F14302394688
:100CD0003046C8470130E1D0236803F00603042BF7
:100CE0001DD0A3682269934225DD4FF000089B1AAE
:100CF00098441A34002501E045451CDA01232246B8
:100D000039463046C847013005F10105F4D1C5E741
:100D100012F0060F12D0003B18BF0123D5E7DAF816
:100D20000030E1682269C91AA368934221EAE17898
:100D3000DDDC0029DDDC0020BDE8F88FE168DAF8B1
:100D40000030CB1A002BD8BF114693DCABE700BFB5
:100D50002DE9F0470C4684B09046227E0C99074658
:100D6000994604F14300002A33D0A2F15803DDB2C2
:100D7000202D67D8202B65D8DFE813F0DE00640053
:100D80006400640064006400640064006400640043
:100D90006400A3006E0064006400640064006E00E0
:100DA000640064006400640021007F00C0006400EF
:100DB0006400AE0064007F0064006400E500236806
:100DC0001A0640F104810B6862691D1D0D601B68E5
:100DD0001A60002382462361CDF80090434603AA9F
:100DE00021463846FFF71EFF013020D023695246C6
:100DF00041463846C847013019D02368E068039E51
:100E00009B0719D5831B002B16DD04F1190A002559
:100E100004E0E068039E831BAB420DDD01235246D4
:100E200041463846C847013005F10105F1D14FF080
:100E3000FF3004B0BDE8F087B042B8BF304604B020
:100E4000BDE8F087012384F84220236104F1420ABF
:100E5000002384F84330BFE723681A0602D45E06F5
:100E600000F1C1800D682A6804350D601546002A1E
:100E70006BDBDFF884C10A2610E023681D0640F111
:100E80009C800B681D1D0D601D68DFF86CC16F2A0A
:100E90000CBF08260A26002384F843306268A2604B
:100EA000002A7FDB236823F004032360002D5BD13D
:100EB000002A79D18246082E65D0A0EB0A00206175
:100EC0008AE70B680122186804330B6004F1420AB8
:100ED00084F842002261BBE70B686268181D086055
:100EE000D3F800A000215046FEF77AFF002800F05A
:100EF0008180A0EB0A0060602061A9E7236843F0CD
:100F0000200323607822DFF8F4C084F845200A68C3
:100F1000151D0D601D0643D4590641D51588DE0701
:100F200044BF43F020032360002D44D1236823F005
:100F3000200323601026AEE7582384F84530DFF8FD
:100F4000B8C02368E3E72368DCE76268A2602D216C
:100F5000002AC5F1000584F8431002DB23F00403E6
:100F60002360DFF894C00A268246B5FBF6F306FB41
:100F700013512A461CF801100AF8011DB2421D4601
:100F8000F3D2082E99D12368D90796D562682369D0
:100F90009A4292DC30230AF8013C0AF1FF3A8CE7CE
:100FA0001568BCE7002DDFD19CF8003084F8423092
:100FB00004F1420A7FE710266DE713F0400F0B683B
:100FC00003F104050D600CBF1D681D885DE713F07B
:100FD000400F0B68626903F104050D601B6814BFC4
:100FE0001A801A60F5E60A68B2F9005004320A6005
:100FF0002A463CE760687FE7C4830E08D8830E0862
:1010000010B5114C86461EF801CB14F80C3003F0D5
:101010000303012B11F8013B624608BF0CF12002CB
:1010200014F803C00CF0030CBCF1010F184604D0F7
:10103000D21A06D1002BE6D110BD2033D01AE2D04F
:1010400010BD104610BD00BFE9660C0811F0FF018D
:10105000034644D0820732D110B5046841EA012E1C
:101060004EEA0E4E8EEA0402A2F1013323EA020395
:10107000A4F1013222EA0402134313F0803F0FD19E
:1010800050F8044F84EA0E0CA4F10133ACF10132A4
:1010900023EA040322EA0C02134313F0803FEFD04B
:1010A000037823B936E010F8013F002B32D0994283
:1010B000F9D110BD8A4211D09A071846CCD01846F3
:1010C00013F8012B002AF5D11046704799071846EE
:1010D00007D0184601330278002AF7D170478207FB
:1010E000F7D10268A2F1013323EA020313F0803F33
:1010F00008D150F8042FA2F1013323EA020313F0C0
:10110000803FF6D00378002BE8D010F8013F002B89
:10111000FBD17047184610BDA2EB0300704700BF1B
:1011200002780B78012A28BF9A42F5D16DE904456F
:1011300040EA0104CDE902676FF0000C4FEA447207
:1011400012B380EA010414F0070F6AD100F007041B
:1011500020F0070004F0030521F007014FEAC50560
:10116000F0E8042314F0040FF1E804670CFA05F426
:1011700062EA040266EA04060AD063EA04036246ED
:1011800067EA0407664603E0F0E80423F1E8046731
:1011900082FA4CF582EA0604A4FA8CF46CBB83FA5A
:1011A0004CF583EA0705A5FA8CF595B950E90223B9
:1011B00051E9026782FA4CF582EA0604A4FA8CF43B
:1011C00083FA4CF583EA0705A5FA8CF52543DBD0B5
:1011D0009CB92DBAB5FA85F424F0070427FA04F176
:1011E000DDE9026723FA04F303F0FF0001F0FF01D9
:1011F000FDE80445A0EB0100704724BAB4FA84F47A
:1012000024F0070426FA04F1DDE9026722FA04F269
:1012100002F0FF0001F0FF01FDE80445A0EB010032
:10122000704714F0030F3CD110F0030428D150F89C
:10123000082B51F8083B82FA4CF582EA0305A5FA1F
:101240008CF55DB950F8042C51F8043C82FA4CF549
:1012500082EA0305A5FA8CF5002DE8D02DBAB5FA7F
:1012600085F424F0070423FA04F122FA04F202F0D0
:10127000FF0001F0FF01FDE80445A0EB010070470D
:101280004FEAC40420F0030050F8082B21F00301BA
:1012900051F8083B0CFA04F462EA040263EA04031E
:1012A000C9E710F003041AD0A1EB040120F00300F9
:1012B000E40750F8042B06D00FD28B785FFAA2F423
:1012C000E41A06D12BB1CB785FFAB2F4E41A00D15C
:1012D0001BB920465DF8104B704701F1040150F82E
:1012E000042BCC0721F0030151F8043B48D824D249
:1012F00022F07F4482FA4CF594EA1325A5FA8CF586
:101300000AD165B951F8043B84EA0204B4EB036FD7
:101310000ED150F8042BEBE74FEA132355E035F0DC
:101320007F454DD10878FDE80445C0F100007047C5
:101330004FEA126203F0FF0347E002EA1C4482FA1C
:101340004CF594EA1345A5FA8CF50AD165B951F824
:10135000043B84EA0204B4EB034F0CD150F8042B95
:10136000EBE74FEA134330E015EA1C4528D10B8820
:101370004FEA124229E04FEA124203EA1C4324E0FA
:1013800002F0FF0482FA4CF594EA1365A5FA8CF595
:101390000AD165B951F8043B84EA0204B4EB032F87
:1013A00009D150F8042BEBE74FEA13630DE015F079
:1013B000FF0F05D10B684FEA122223F07F4304E0B0
:1013C0004FF00000FDE80445704712BA1BBA82FADC
:1013D0004CF482EA0304A4FA8CF5B5FA85F402FA17
:1013E00004F203FA04F34FEA1260FDE80445A0EBAF
:1013F0001360704780EA0102844612F0030F4FD158
:1014000011F0030F32D14DF8044D11F0040F51F8D3
:10141000043B0BD0A3F101329A4312F0803F04BF8A
:101420004CF8043B51F8043B16D100BF51F8044B73
:10143000A3F101329A4312F0803FA4F101320BD1A3
:101440004CF8043BA24312F0803F04BF51F8043B28
:101450004CF8044BEAD023460CF8013B13F0FF0F85
:101460004FEA3323F8D15DF8044B704711F0010FB8
:1014700006D011F8012B0CF8012B002A08BF704789
:1014800011F0020FBFD031F8022B12F0FF0F16BF80
:101490002CF8022B8CF8002012F47F4FB3D1704748
:1014A00011F8012B0CF8012B002AF9D1704700BF6D
:1014B00090F800F06DE9024520F007016FF0000C94
:1014C00010F0070491F820F040F049804FF000043C
:1014D0006FF00700D1E9002391F840F000F1080017
:1014E00082FA4CF2A4FA8CF283FA4CF3A2FA8CF34F
:1014F0004BBBD1E9022382FA4CF200F10800A4FAB6
:101500008CF283FA4CF3A2FA8CF3E3B9D1E9042309
:1015100082FA4CF200F10800A4FA8CF283FA4CF340
:10152000A2FA8CF37BB9D1E9062301F1200182FAFA
:101530004CF200F10800A4FA8CF283FA4CF3A2FA00
:101540008CF3002BC6D0002A04BF04301A4612BA0E
:10155000B2FA82F2FDE8024500EBD2007047D1E911
:10156000002304F00305C4F100004FEAC50514F0A0
:10157000040F91F840F00CFA05F562EA05021CBF71
:1015800063EA050362464FF00004A9E72AB330B5C9
:10159000134C8646851804E0D21A1CD1C3B1AE455F
:1015A00017D01EF8010B235C03F00303012B11F885
:1015B000013B14F803C00CF0030C024608BF00F115
:1015C0002002BCF1010F1846E6D12033D01AE6D034
:1015D00030BD002030BD104630BD1046704700BF02
:1015E000E9660C08A2B330B540EA0104A4078446BA
:1015F0000B462AD09CF800000C7884422FD1012A97
:101600000DD0E64660B11EF8010F11F8014F6FEAE8
:101610000E03A042134422D11CEB0303F2D100209D
:1016200030BD0468194653F8045BA4F1013EAC4296
:1016300084462EEA040E00F104000BD1043A8446DD
:101640001946ECD01EF0803FE9D1032AE9D8D1E752
:10165000104670479CF800000C78A042D1D0001BC7
:1016600030BD00BF30B540EA0104A30701D1032A11
:101670000FD8844601F1FF3E07E01EF8011F03F872
:10168000011B541EC1B19C4622466346002AF4D178
:1016900030BD0B468446194653F8045BA5F101346E
:1016A00024EA050414F0803FE4D1043A032A4CF8FC
:1016B000045B1946EFD8DDE76244002CE8D003F85C
:1016C000011B9342FBD130BD10B4044C03460A46C3
:1016D00020685DF8044B194600F002B8042200208F
:1016E00070B50D461446012162B12B4605EB020C84
:1016F00001E0634512D01A4601331478002CF8D16A
:10170000541B611CB2F096FE064628B122462946BB
:10171000FEF7E8FB00233355304670BD5C1B611CAF
:10172000F0E700BF71B1034600EB010C01E0634537
:1017300006D01A46013311780029F8D1101A7047E3
:10174000181A70470846704771B138B503460C4601
:10175000002501E0431C054621461846FFF776FCAC
:101760000028F7D1284638BDFFF770BC2DE9F04FAF
:101770001C462DED048B9D4B1B689FB000258246B7
:101780001846884607921A950893FFF791FE0021A4
:1017900083460020CDE90401CDF864804246174617
:1017A00012F8013B2D2B2FD8DFE813F0A4002E00F8
:1017B0002E002E002E002E002E002E002E00B40033
:1017C000B400B400B400B4002E002E002E002E0091
:1017D0002E002E002E002E002E002E002E002E0099
:1017E0002E002E002E002E002E002E00B4002E0003
:1017F0002E002E002E002E002E002E002E002E0079
:101800002E000E042E00040400220992302B00F05A
:10181000838000220C922F2B1C4640F24D854FF006
:10182000000938464E464D4612E00130082D199009
:10183000C8BF09EB89090478C6BF03EB4903A3F1CC
:101840003009A2F130062F2C05F10105234674DD85
:1018500006EB8602392C03EB4202E6DD08995A4674
:10186000FFF7C0FE0346002835D1199A11465A44A5
:10187000199211F80B40002D40F0A985302C40F052
:101880006185C2F101015318013219921478302C8C
:10189000F9D0A4F13102082A00F24383A4F1300EFA
:1018A000199C03F1010B0023012527460A9306EB3F
:1018B00086060EEB46060023621C19926478A4F19A
:1018C0003001092900F2F18201338E46002940F0EF
:1018D000D284199CF0E70023652C0A959B469E460E
:1018E00001D0452C36D1002D40F085800C9A1A434A
:1018F00040F08080079B9FED3B8B13B1079BC3F8A3
:101900000080B0EE480AF0EE680A1FB0BDEC048B10
:10191000BDE8F08F199242E77B7803F0DF03582B84
:1019200000F08D84013719973B78302BFAD0002BCB
:1019300000F0D38001220C926DE708995A46FFF718
:1019400051FE0346002800F0DB800A954FF0000BA3
:101950005B46DE4600220D92002D00F098800A9A28
:101960001346002A08BF2B4630460A93FAF7CAFDF1
:101970000B460246CDE904230D9B102DA3EB0B0370
:101980002C46A8BF1024092D0C9314DD184B03EB33
:10199000C40353E91223FAF72FFE02464846904645
:1019A0008946FAF7AFFD02460B4640464946FAF72C
:1019B0006DFCCDE904010F2D00F3AB800C9B002BD7
:1019C00000F034840C9B40F38283162B40F3F184A7
:1019D0000C9AC5F12503934280F204850C9B2C1BC5
:1019E0001C449CE00000000000000000EC680C08B3
:1019F00008690C080025DDF8648008F101021992DD
:101A000098F801402B2C00F089822D2C00F01D82CB
:101A100000220892A4F13002092A00F21182302C2F
:101A200005D1199A013219921478302CFAD0A4F108
:101A30003102082A8ED819990D914A1C1992A4F1E5
:101A400030004C782F2C09DC00F044BC0132199294
:101A50009CF801402F2CA1F1300006DD00EB800145
:101A6000392C944604EB4101F0DD0D99521A082AF5
:101A700040F3308444F61F620D92089A002A3FF426
:101A80006BAF0D9A52420D92002D7FF468AF0C9A05
:101A9000134322D1BEF1000F7FF42CAF692C00F06C
:101AA000318400F35283492C00F02C844E2C7FF4B7
:101AB00021AFB84919A802F031FC00283FF41AAF51
:101AC000199B1B78282B00F07185B34803F0B8FAF6
:101AD000B0EE408AF0EE608A01E09FEDAA8B079A93
:101AE0000AB1199B1360099B002B3FF40AAF18EE53
:101AF000901A18EE102A01F1004343EC182B00E76E
:101B0000199A0A9502EB0B01199112F80B409B46AA
:101B1000D5E60C9B2C1B1C44002C40F31B8314F0BB
:101B20000F000AD09D4901EBC001DDE90423D1E992
:101B30000001FAF761FDCDE9040134F00F0340F034
:101B40007082002308930A9A00962B463946504625
:101B500002F0B6FD1190002800F06B830D9BABEBFB
:101B600003000C9B002BB4BF024600224FF000087C
:101B700023EAE3730D921093C346119C50466168AB
:101B800002F0E8FC8146002800F0478122699DEDC3
:101B9000048B0232920004F10C010C30FEF7A2F922
:101BA000B0EE480AF0EE680A1CAA1BA9504603F0E2
:101BB00031F91A90002800F01D810121504602F0F1
:101BC00029FE8346002800F028811B9B002BC0F2D1
:101BD00017810D9A109D9E18089A1C9C9B1A2344ED
:101BE0006F4A013B9342C4F1360480F2B080D21AAE
:101BF0001F2AA4EB020400F31C81012393400A93E3
:101C00000027089B25443444A6421D443346A8BF00
:101C10002346AB42A8BF2B46002B02DDE41AED1A87
:101C2000F61A0D9B002B00F3C580002C00F3D98021
:101C30000C9B002B00F3E880002D00F3F080002EB9
:101C400008DD59463246504602F018FF8346002808
:101C500000F0E3801A994A46504602F0A5FF8046FC
:101C6000002800F0DA800023C268C36059460E9253
:101C700002F078FF0028C0F2758400F0E583594631
:101C8000404603F02FF955EC104B10EE100A0022DD
:101C90004FF080432946FAF72BFF00285BD00E9BBC
:101CA000002B00F0DD80059B0F933E4B3D4D002245
:101CB000CDE90A2300243C4F0F9A3C4B02EA070669
:101CC0009E4200F0F880089B8BB1B6F1D46F0ED81D
:101CD0002EA3D3E9002320462946FAF709FF00285E
:101CE00040F087810B9B03F1D6639B1B0B93DDE9CF
:101CF0000A01B0EE480AF0EE680ACDE9040102F0EC
:101D0000F9FFDDE9040153EC102BFAF775FC53ECF5
:101D1000182BFAF7BBFACDE904010A91089B2BB9FD
:101D2000214B0A9A13409E4200F004811A995046B2
:101D300002F050FC4946504602F04CFC59465046D1
:101D400002F048FC4146504602F044FC15E70123EE
:101D500000270A9355E7164B204629460022FAF73A
:101D60004BFC0E9B04460D46002B76D101F100433F
:101D700012901393059B0F93DDE91223CDE90A23FB
:101D800099E700BF00000000000000000000C0FF55
:101D9000FFFFDF41F8830E08F8840E0808690C087D
:101DA00002FCFFFF0000F03F0000F07F0000E07F3A
:101DB0000000E03F59461A46504602F0EFFD8346C8
:101DC00058B301461A9A504602F03AFD28B30E90D5
:101DD0001A99504602F0FEFB0E9B1A93002C7FF7D7
:101DE00027AF1A992246504602F048FE1A90002862
:101DF0007FF41EAF22239FEDBF8BCAF80030C4E0F2
:101E0000109A0D9ED51AE7E64946109A504602F000
:101E1000C5FD814600287FF40FAF1A98EAE74946CE
:101E20002A46504602F02AFE814600287FF407AF7A
:101E3000F3E7B84FFF1A012303FA07F70A93E0E626
:101E40000022CDF864800D9286E50122089208F107
:101E50000202199298F80240DCE5CDE9124589E7C3
:101E6000DDE90412002940F0B280C2F313030F929F
:101E7000002B40F0B280A84B002220462946FAF7FA
:101E80002DFE002840F0A782A44B204629460022C0
:101E9000FAF7B2FB01F1004304460D461690179382
:101EA000DDE91623CDE90A2305E7652C4FF0010E85
:101EB0003FF4A1AD15E5A2F1547305939DED047BAC
:101EC000DDE90A01B0EE470AF0EE670AB0EE479A84
:101ED000F0EE679ACDE9040102F00CFFDDE90401A0
:101EE00053EC102BFAF788FB53EC192BFAF7CEF9C9
:101EF0008B4B0F409F42CDE9040175D918EE902A13
:101F000003F154739A4203D118EE103A013384D08E
:101F1000844A4FF0FF33CDE9043207E700220892EC
:101F200095E7652C00F00A81452C00F007814FF001
:101F3000010EACE52046294604F008FAFAF72EFB1C
:101F40000B46024629462046FAF79EF9049C0E9F4E
:101F500027430A9CC4F3130657EA060304460D46BA
:101F600000F0AC8065A3D3E90023FAF7B7FD48B9C8
:101F700064A3D3E9002320462946FAF7CDFD0028C3
:101F80003FF4D4AE9DED048B1A980146504602F002
:101F900021FB4946504602F01DFB5946504602F0CF
:101FA00019FB1199504602F015FB4146504602F0CC
:101FB00011FB94E5012309937A1C19927B78002B7D
:101FC0003FF498AC174621E400230993F4E7DDE9D8
:101FD0000412012900F086810F92534B4E4D0022CE
:101FE000CDE90A23002466E601F154730A930593B0
:101FF00094E629462046FAF7D7FD012838BF01208C
:10200000FAF780FA0E9B04460D46002B40F07781CC
:1020100001F1004314901593DDE91423CDE90A235F
:1020200060E6B3F59A7F00F304811C11102B3F4B3F
:10203000089340F3D7829846DDE904234FF0000C63
:10204000E14614F0010F104619464FEA640409F105
:10205000010907D0D8E90023FAF7CEFA4FF0010CB6
:1020600002460B46012C08F10808EAD1BCF1000F2A
:1020700001D0CDE90423089B03EBC909059BA3F11B
:1020800054730593DDE90423D9E90001FAF7B4FAA2
:10209000274BCDE904010B400A4626498B4200F24A
:1020A000C880A1F580118B4240F23B821D4A4FF05F
:1020B000FF33CDE904320023089344E513A3D3E9A9
:1020C0000023FAF70BFD00283FF430AE5AE7163331
:1020D000FFF61FAD0D9BABEB030A174B03EBCA03D7
:1020E000DDE90401D3E90023FAF7B0FB41EC180B5A
:1020F000F5E400BF000000000000F07F9535A094DB
:10210000FFFFDF3F35E5AF350000E03F9535A09498
:10211000FFFFCF3FE2FBFFFF0000F03F0000E03F8A
:10212000FFFF9F7CFFFFEF7F0000F0BFF8690C0806
:102130000000F07F0000A07C08690C0800220A92D1
:1021400093464FF0010EFFF7D1BB6E2C3FF4B1ACBC
:10215000FFF7D0BB3FF4F5AC644214F00F020AD095
:10216000B24B03EBC203DDE90401D3E90023FAF724
:102170006DFBCDE9040124113FF4E3AC1F2C3EDCE0
:1021800014F0100318BF6A230893DDE90423DFF875
:10219000B4824FF0000C14F0010F1046194607D01E
:1021A000D8E90023FAF728FA4FF0010C02460B4653
:1021B000641008F10808EED1BCF1000F01D0CDE9A0
:1021C0000423089B93B1DDE90401C1F30A52C2F173
:1021D0006B03002B0ADD1F2B40F330820020342BD1
:1021E000049040F336824FF05C730593DDE90401FF
:1021F00000220023FAF768FC00283FF4A4AC222355
:102200009FED848BCAF8003069E41C9B04931B9BF0
:1022100003F233421D9B23F4801343EA02530593D8
:10222000290742BF059B43F0004305939DED048BB6
:1022300055E422239FED798BCAF800304FE4099BC7
:1022400001931AAB02940093794A1BAB19A950462B
:1022500001F078FD10F0070405463FF43EAC062C73
:1022600073D1079B9FED6B8B0137002B3FF449AB7C
:102270001F60FFF746BB6A1C012B199C9B4410464C
:1022800015D02B4403F1FF3C03E0460094450DD0EC
:1022900001322B46082B154606EB8600F5D9102A8D
:1022A000DCBF09EB89094FEA4909EFE7981C082DC3
:1022B0003EDC0546FFF7FBBA08995A463846FFF759
:1022C00091F900286BD000231D460A9399461E46BB
:1022D000FFF73CBB44F61F629042A8BF10460D902A
:1022E000FFF7CBBBDDE904120F92002A7FF475AE35
:1022F00022239FED488B1A98CAF8003045E6CDE9B5
:10230000144589E64B4919A802F008F800283FF463
:10231000F1AA199B4849013B19A8199301F0FEFF46
:1023200010B9199B013319939FED3C8BFFF7D7BB75
:102330001028DCBF09EB890901EB49090546002398
:10234000FFF7BABA0023FFF7A4BA1A9A3AB13521B7
:102350001CA802F015FE1A99504602F03BF9013C08
:10236000042C3FF65DAF01A353F824F00B220108C3
:10237000952301088F230108812301080B220108FE
:102380004FF0FF336FF00040CDE9043048E72B4BAE
:10239000059345E71C9B04931D9B059340E7199A01
:1023A00013465A44199213F80B4006468146FFF72C
:1023B00065BA0C981D4901EBC001DDE90423D1E9A0
:1023C0000001FAF719F941EC180BFFF788BB0A95E1
:1023D0008346FFF774BA9FED137B194D8DED167B85
:1023E00000245DE5114CC5F10F0504EBC501DDE9E5
:1023F0000423D1E90001FAF7FFF80C9B5D1B04EB05
:10240000C504D4E90023FAF7F7F841EC180BFFF7FD
:1024100066BB00BF000000000000000000000000DC
:102420000000F07F000000000000E0BF08690C0819
:1024300098660C08EC830E08F0830E080000F07F0D
:102440000000E03FC0660C080E9B002B70D0DDE959
:102450000445954BC5F3130199422A463FD0002FFE
:1024600000F0B880DDE904231F421C4623D0B0EE03
:10247000480AF0EE680A0E9B002B00F0B68002F0CE
:1024800039FC089B51EC100B6BB1C4F30A54C4F136
:102490006B04002C07DD240504F17F53002203F5B3
:1024A0004013FAF7A9F802460B4651EC180BF9F75E
:1024B000EDFE41EC180B089B7BB151EC180B7B4BEC
:1024C0000022FAF799F841EC180B18EE902A03460F
:1024D000134304BF2223CAF800301A9855E5089B1D
:1024E0000499002B00F0B280714B2B40B3F1D46FF4
:1024F00000F2AC801B0DC3F16B034FF0FF3000FA0C
:1025000003F39942ABD16B4B9A4200F0C780684B02
:10251000134003F580130593002304939DED048B72
:10252000C9E702F15473059300230893FFF70BBB2F
:10253000DDE90412C2F313030B4314468FD1089B49
:10254000002B40F0A0805A4B2340A3F580136FEA84
:1025500013536FEA035305934FF0FF3304939DED3C
:10256000048BA8E7DDE904010E9B0343A3D1C1F36B
:1025700013030C46002B9ED121F000431B0D1B05BD
:10258000B3F1D66F97D9D8F814301BB9D8F81030FA
:10259000012B90DD41460122504602F06FFA594668
:1025A000804602F0DFFA002885DDC8E7424919A815
:1025B0001CAA01F0CFFE05287FF487AA1D9B43F0DB
:1025C000FF4343F4E00305931C9B04939DED048BB0
:1025D000FFF785BADDE904010A9B03423FF46BAFC4
:1025E0000C4644E74FF0000945E502F083FB0899EB
:1025F00053EC102BB9B3C4F30A54C4F16B04002C90
:102600000CDD2405194604F17F530E9A03F540139F
:1026100010EE100AF9F7F0FF02460B4651EC180BCA
:10262000F9F732FE02460B4643EC182B002200233A
:10263000FAF74AFA00283FF440AF59E64FF0FF326C
:1026400002FA03F3049A1A400492CFE54FF0FF33E5
:1026500057E74FF0FF33C2F14B0203FA02F202EAEE
:1026600001030593C2E551EC180BF9F70DFE024684
:102670000B4643EC182B00220023FAF725FA00281A
:102680003FF42BAF34E60A4B2340B3F1D66F3FF74C
:102690005CAFB3F15C7F3FF710AF29E601317FF407
:1026A00036AFFFF7BABB00BFFFFF0F000000503985
:1026B0000000F07FFFFFEF7FAC660C08014BFFF7D7
:1026C00055B800BF6C22002010B4054C8446134658
:1026D00020685DF8044B0A466146FFF747B800BF23
:1026E0000422002010B4054C054B84460A4620689D
:1026F0005DF8044B6146FFF739B800BF04220020A3
:102700006C2200202DE9F041DFF8A8800446134632
:102710002DED028B0A46D8F800002146FFF726F877
:1027200055EC104B10EE102A10EE100A2B462946DD
:10273000FAF7FCF950BB20462946FAF755FA08EE9D
:10274000100ADFED197AB0EEC87AB4EE677AF1EECE
:1027500010FA15DD25F00047144B4FF0FF322046EC
:102760003946FAF7E3F938B9104B4FF0FF322046FB
:102770003946FAF7BDF918B1D8F8003022221A60AC
:10278000B0EE480ABDEC028BBDE8F081002D084890
:1027900004DAFBF791F8B1EE408AF1E7BDEC028B69
:1027A000BDE8F041FBF788B8FFFF7F7FFFFFEF7FB9
:1027B000F8840E08042200202DE9F041DFF8AC80F7
:1027C000264B04460A462DED028B2146D8F8000020
:1027D000FEF7CCFF55EC104B10EE102A10EE100A4D
:1027E0002B462946FAF7A2F950BB20462946FAF7AC
:1027F000FBF908EE100ADFED1A7AB0EEC87AB4EEF3
:10280000677AF1EE10FA15DD25F00047154B4FF011
:10281000FF3220463946FAF789F938B9114B4FF0A3
:10282000FF3220463946FAF763F918B1D8F800307C
:1028300022221A60B0EE480ABDEC028BBDE8F0819E
:10284000002D094804DAFBF737F8B1EE408AF1E7CA
:10285000BDEC028BBDE8F041FBF72EB86C220020E6
:10286000FFFF7F7FFFFFEF7FF8840E080422002028
:10287000F0B4074610B33E468C4616F8010B01E053
:10288000A04216D01CF8014B002CF9D1D8B116F893
:10289000015B0C4601E0002BF9D014F8013B9D428E
:1028A000F9D14DB1002306F8013C16603846F0BC62
:1028B00070475BB13746DEE72E46F6E71768002F14
:1028C000D9D13846F3E7F0BC10607047166038463F
:1028D0003B70ECE70123FFF7CBBF00BF2DE9F04FC2
:1028E000814645488E4675461EF801CB10F80C40CF
:1028F00014F00804F7D1BCF12D0FE34654D0BCF11D
:102900002B0F08BF9EF800B06FF0004808BF05F11C
:10291000020E1BB1102B4FD01F4604E0BBF1300F4D
:1029200055D00A231F460025B8FBF7F6284607FBBB
:10293000168A07E0864215D329D007FB00C001257F
:102940001EF801BBABF1300CBCF1090F06D9ABF19D
:10295000410CBCF1190F08D8ABF1370C63450DDD04
:10296000002DE7DA4FF0FF35EAE7ABF1610CBCF17F
:10297000190F03D8ABF1570C6345F1DC002D0BDBCD
:1029800004B140420AB195BB1160BDE8F08FE24549
:10299000D3DA4FF0FF35D3E72223C9F800301AB35A
:1029A0000EF1FF314046EFE79EF800B04FF00048CF
:1029B00005F1020E0124ACE7BBF1300FACD19EF85B
:1029C000000000F0DF00582807D01F46ABE79EF854
:1029D000003003F0DF03582B0BD110279EF801B015
:1029E0003B460EF1020E9EE74046BDE8F08F804662
:1029F000D6E708231F4696E7E9660C08012B02D0AC
:102A0000242B00D86AE710B5FDF7F2F8162303600F
:102A1000002010BD012A08D0242A06D88446064882
:102A2000134600680A46614658E710B5FDF7E0F81E
:102A300016230360002010BD04220020012A08D0C4
:102A4000242A06D884460648134600680A4661468A
:102A500044E710B5FDF7CCF816230360002010BD45
:102A6000042200202DE9F04707464B480E46354624
:102A700016F801CB10F80C4014F00804F7D1BCF1A3
:102A80002D0FE64658D0BCF12B0F04BF96F800E09E
:102A9000AE1C5BB1102B54D04FF0FF38B8FBF3F8ED
:102AA00003FB08FA6FEA0A0A994608E0BEF1300F04
:102AB0005AD00A23DFF8E4804FF0050A9946002532
:102AC000284607E0404515D829D009FB00C001255C
:102AD00016F801EBAEF1300CBCF1090F06D9AEF1DE
:102AE000410CBCF1190F08D8AEF1370C63450DDD70
:102AF000002DE7DA4FF0FF35EAE7AEF1610CBCF1EB
:102B0000190F03D8AEF1570C6345F1DC002D0BDB38
:102B100004B140420AB16DB91160BDE8F087D445F7
:102B2000D3DD4FF0FF35D3E722233B604FF0FF307A
:102B3000002AF2D0711EEFE796F800E00124AE1CE7
:102B4000A7E7BEF1300F21D1307800F0DF00582820
:102B500016D14FF0100996F801E04FF00F0A023637
:102B60006FF070484B46AAE7337803F0DF03582B29
:102B7000EFD008234FF0070A6FF0604899469EE7B0
:102B800099466FF070484FF00F0A98E74FF00F0A20
:102B90006FF07048994692E7E9660C08999999197F
:102BA00060E700BF10B4044C8446134620685DF80B
:102BB000044B0A46614655E70422002010B4044C39
:102BC0008446134620685DF8044B0A46614649E78F
:102BD00004220020034BC35C03F00303012B08BF56
:102BE00020307047E9660C08034BC35C03F0030315
:102BF000022B08BF20387047E9660C082DE9F04F1A
:102C000003690C69A34283B0C0F28780013C01F1E3
:102C10001405A30000F11408009355F8243058F867
:102C20002420013381469A4208EB840005EB840797
:102C30000190B2FBF3F63BD30023AE4640469B46E1
:102C40005EF804AB02681FFA8AFC06FB0C334FEAFD
:102C5000134C4FEA1A4A06FB0ACA1FFA83FCABEB75
:102C60000C0C1FFA8AF31CFA82FCC3EB124202EB33
:102C70002C421FFA8CFC4CEA0243774540F8043B97
:102C80004FEA224B4FEA1A43DAD2009B58F803303E
:102C900073B9019B043B984504D307E0984504F1C0
:102CA000FF3403D253F80429002AF7D0C9F81040A2
:102CB000484601F057FF00282BDB01364046002331
:102CC00055F8041BD0F800C08AB29A1A0B0C12FAFD
:102CD0008CF2C3EB1C4303EB224392B242EA034261
:102CE000AF4240F8042B4FEA2343E9D258F824209E
:102CF00008EB84036AB9043B984504D307E0984580
:102D000004F1FF3403D253F80429002AF7D0C9F89C
:102D10001040304603B0BDE8F08F002003B0BDE89E
:102D2000F08F00BF2DE9F04F2DED068B466A95B070
:102D30008DED020B249C019159EC108B05460992F4
:102D40000693002E00F00683316849B172684A602C
:102D5000012393408B6001F03DFC6B6A00221A60F6
:102D6000B9F1000AB4BF0123002323607B4BBCBF31
:102D70002AF0004ACDF80CA033EA0A0300F0B28032
:102D80009DED027B002251EC170BB0EE479AF0EE5E
:102D9000679A0023F9F798FE074680B1069A012347
:102DA0001360259B002B00F0EF826D481860431ED6
:102DB0000093009815B0BDEC068BBDE8F08F12AA09
:102DC00013A92846B0EE490AF0EE690A02F022F88B
:102DD000B0EE498AF0EE698A5FEA1A56044640F07E
:102DE0009980DDE912763E4406F23240202840F315
:102DF000BF83C0F140000AFA00FA06F2124028FA36
:102E000000F04AEA0000F9F77DFB0123013E0D9333
:102E1000A1F1F871534B0022F9F736FA49A3D3E92F
:102E20000023F9F7E9FB49A3D3E90023F9F72EFAC8
:102E3000804630468946F9F775FB46A3D3E900235F
:102E4000F9F7DAFB02460B4640464946F9F71EFA07
:102E500080468946F9F780FE0022834600234046DB
:102E60004946F9F73BFE002840F08182BBF1160F7E
:102E700000F263823C4B03EBCB03D3E9002351EC1C
:102E8000190BF9F72BFE002874D00023BE1B0C93FE
:102E9000731E0BF1FF3B049300F15682002308934D
:102EA000BBF1000F6DDA089BCDF814B0A3EB0B0358
:102EB0000893CBF100030B93019B092B4FF0000B00
:102EC00068D8052B40F35283043B01930026019BF5
:102ED000023B032B00F2AC86DFE813F065046204CA
:102EE0005A043C04069A42F20F73CAF3130A1360A1
:102EF0005AEA08031DD1259B002B00F095861B4B39
:102F000000930833259A0098136015B0BDEC068B2A
:102F1000BDE8F08F18EE903AC3F3130351EC190B90
:102F200043F07F510D97A6F2FF36129F41F44011F6
:102F300070E7259B002B40F0F0830D4B009338E7A2
:102F4000AFF3008061436F63A787D23FB3C8608B44
:102F5000288AC63FFB799F501344D33F0000F07F7F
:102F6000C1830E080000F83F08690C08FC830E08B6
:102F700008840E08BE1B731E049300F1D9840C90C4
:102F80000890049B5B44CDE9043B00230B93019B19
:102F9000092B96D9002301264FF0FF3201930A96A0
:102FA000079209936B6A00215960079B0F9328468B
:102FB00001F0D0FA0090002800F043866B6A009A76
:102FC0001A60079B0E2B00F2F980002E00F0F680AD
:102FD0000599002940F38084BD4B01F00F0203EBFB
:102FE000C2034FEA2118C905D3E9006740F11384F1
:102FF000B84B51EC190BD3E90823F9F727FC41EC46
:10300000180B08F00F084FF0030AB8F1000F13D0A7
:10301000DFF8C09218F0010F09D030463946D9E9DF
:103020000023F9F7E9FA0AF1010A06460F465FEABA
:10303000680809F10809EDD151EC180B32463B46FE
:10304000F9F704FC41EC1A0B0C9B5BB157EC1A6BC3
:10305000A14B1AEE100A00223946F9F73FFD00286D
:1030600040F06C855046F9F75DFA53EC1A2BF9F7EE
:10307000C3FA9A4B0022F9F709F9079B8046A1F1A0
:103080005079002B00F00484059B1093079B0E934E
:103090000A9B002B00F0D6840E9A8D4B9049DDF8E8
:1030A00000A003EBC20353E902230020F9F7CEFB93
:1030B00042464B46F9F7E8F859EC1A8B41EC180BED
:1030C00049461AEE100AF9F747FD0746F9F72AFABA
:1030D00002460B461AEE100A4946F9F7D5F8303782
:1030E0000AF8017B53EC182B06460F46F9F7F6FC5D
:1030F000002840F067854FF000080AEE104A0AEEFB
:10310000905ACDF844B0554644465BEC18AB2AE0E3
:103110000E9B01349C424BDA724B504659460022BA
:10312000F9F76AFA6F4B002282468B4630463946E1
:10313000F9F762FA89468046F9F70EFD0746F9F776
:10314000F1F902460B4640464946F9F79DF83037FB
:1031500005F8017B52465B4606460F46F9F7BEFC72
:10316000002840F02A8532463B465B490020F9F7AB
:103170008BF852465B46F9F7B1FC0028C8D0109B8B
:10318000009A0593AA461AEE104A1AEE905A02E0E7
:10319000524500F0FC84D1461AF8013D392BF7D096
:1031A0000133DBB28AF80030059B01330593BEE1A1
:1031B000DDF844B01AEE104A1AEE905A139B002B19
:1031C000C0F29480059A0E2A00F39080404B03EBE6
:1031D000C203D3E90089099B002B1BDA079B002B54
:1031E00018DC40F06E83404B002240464946F9F718
:1031F00003FA02460B4651EC190BF9F779FCDDF89E
:103200001CA05646002800F0E682099BDDF80080ED
:10321000DF43E8E242464B4651EC190BF9F716FB47
:10322000F9F79AFC06468346F9F77CF942464B4685
:10323000F9F7E2F90B46024651EC190BF9F724F8BD
:10324000DDF800A0334630330AF8013B079B012B21
:1032500000F09F834FF0010B08EE104A08EE905AE1
:1032600054461D46DA461DE042464B463046394636
:10327000F9F7ECFAF9F770FC8346F9F753F942468F
:103280004B46F9F7B9F90AF1010A0B4602463946ED
:103290003046F8F7F9FF0BF13003AA4504F8013B7B
:1032A00000F072830F4B0022F9F7A6F900220023E9
:1032B00006460F46F9F708FC0028D5D0A24618EEBE
:1032C000905A18EE104A059B01330593D1462EE122
:1032D00008690C08F8690C080000F03F00001C4069
:1032E0000000E03F00002440000014400A9A002A39
:1032F00052D0019A012A40F3A682079B03F1FF38BE
:103300000B9B434580F284820B9BCDF82C80A8EB6D
:1033100003039B444FF00008079B002BC0F271830E
:10332000049A1A440492089A17461A4408920121F2
:10333000284601F06FFA064632E00123BE1B0C93CB
:10334000731E04937FF5AAADC6F101030893002311
:103350000493A5E51020B0F0CFFF02466862002874
:1033600000F05D84C0E901660660C660F8E4584676
:10337000F9F7D8F842464B46F9F7A6FB00287FF448
:1033800075AD0BF1FF3B71E5874B0093009815B0CD
:10339000BDEC068BBDE8F08FDDF82C80089F0A9EFF
:1033A000002F0CDD049A002A09DD0899BA42134661
:1033B000A8BF3B46C91AFF1AD31A089104930B9B66
:1033C000DBB10A9B002B00F08082B8F1000F0FDD0B
:1033D00031464246284601F0E1FA224601460646B9
:1033E000284601F02DFA21460446284601F0F2F85D
:1033F0000B9BB3EB080240F0FE820121284601F04E
:1034000009FABBF1000F824600F3B780019B012B44
:1034100040F388814FF000080120BBF1000F40F01D
:10342000B880049A104410F01F0000F09680C0F19C
:103430002003042B40F30C84089BC0F11C000344C0
:103440000244089307440492089B002B05DD2146A3
:103450001A46284601F012FB0446049B002B05DDAA
:1034600051461A46284601F009FB82460C9B002B68
:1034700040F03881079B002B40F31F810A9B002BF3
:1034800040F0A280059B01330593DDF80080DDF854
:103490001C90012707E0214600230A22284601F05C
:1034A000BDF80137044651462046FFF7A7FB4F45BC
:1034B00000F1300008F8010BEDDB079A002AC8BFC5
:1034C0009346009AD8BF4FF0010B03469344002760
:1034D000214601222846019301F0D0FA51460446C4
:1034E00001F040FB002840F3A3811BF8013C009A47
:1034F0000BF1FF3B04E05A4500F0B5811BF8013D9C
:10350000392B0BF10109F6D001338BF8003051460D
:10351000284601F05FF856B12FB1B74203D03946C3
:10352000284601F057F83146284601F053F8214665
:10353000284601F04FF8002389F80030DDE9052323
:103540001A60259B002B3FF434AC0098C3F8009020
:1035500015B0BDEC068BBDE8F08F1C20089B034422
:103560000893049B0344074404936DE70126AEE4EB
:10357000C0F1200008FA00F045E401465A4628460A
:1035800001F00CFA019B012B824640F3D3814FF0EE
:103590000008DAF810300AEB8303186901F0EAF842
:1035A000C0F120003DE700BFC0830E083146002374
:1035B0000A22284601F032F80F9B002B064640F302
:1035C0001F83CDF814900793002F00F31A81B8F1F0
:1035D000000F40F0F981B046029B009F079903F06D
:1035E00001027B1E1944019B0A921343089109931F
:1035F00051462046FFF702FB31468346204601F044
:10360000B1FA424651468146284601F0CDFAC268D9
:1036100001460BF13003002A42D104902046079363
:1036200001F0A0FA04990290284600F0D3FF029A14
:10363000079B1AB90999002900F0D482B9F1000F4B
:10364000C0F28481019949EA01090A9951EA090104
:1036500000F07C81002A00F3D881089A3B7007F1C2
:1036600001099742CB4600F0E381214600230A225C
:10367000284600F0D3FF4645044631464FF000038C
:103680004FF00A02284612D000F0C8FF4146064615
:1036900000230A22284600F0C1FF4F468046A7E7D4
:1036A0002846029300F096FF029B0122C6E700F035
:1036B000B5FF4F46064680469AE7019B022B79DC10
:1036C0000A9B002B80D1059B514601332046059370
:1036D000FFF794FADDF800B000F130030BF8013B7E
:1036E0000027F5E65146204601F03CFA0028BFF6D7
:1036F000C1AE214600230A22284600F08FFF059B19
:1037000003F1FF390A9B0446002B7FF44FAF0F9B58
:10371000002B40F36E820793B7E6BF4B0093033351
:10372000FFF7F0BBDDE9021200297FF473AEC2F3AC
:103730001303002B7FF46EAEB84B1340002B00F048
:103740003A82089B01330893049B013304934FF0A2
:10375000010861E601230A93099B059A13440F931C
:103760000133012B18460793B8BF01206F6A00216F
:10377000172879607FF71BAC012204235B0003F15B
:10378000140C8445114602F10102F7D979600EE468
:1037900001230A930998002845DD0F900790E5E77B
:1037A00000230A93D8E700230A93F3E70F9BCDF891
:1037B00014900793079B002B7FF427AD51460522F9
:1037C000284600F02BFF01468246204601F0CAF948
:1037D00000287FF71AAD0098059F3123804600F836
:1037E000013B013700905146284600F0F3FE7B1C58
:1037F000DDF800900593CDF80080002E7FF493AEA5
:1038000095E631463A46284601F038F90646DEE6A6
:10381000A3EB080880E54FF0020AB0EE498AF0EE0B
:10382000698AFFF7F2BB012309930793FFF7BABB3D
:1038300003D1019BDB073FF558AED9461BF8013D8C
:10384000302BFAD063E60D9A002A00F0F78003F2DD
:103850003343049ADDF82C801A440492089A1746E0
:103860001A44089263E5059B009A013305933123BE
:1038700013704CE65046F8F755FE53EC1A2BF8F748
:10388000BBFE674B0022F8F701FD8046A1F150799D
:10389000644B002251EC1A0BF8F7F6FC42464B46FB
:1038A00006460F46F9F738F9002840F08081304687
:1038B0003946424609F10043F9F710F900283FF470
:1038C0007DAC4FF0000A56469FE421460B9A2846ED
:1038D00001F064F8044690E500F02881059A524B07
:1038E000564206F00F0203EBC203D3E9002351EC6A
:1038F000190BF8F781FE361141EC1A0B00F08B81A1
:103900004A4F00234FF0020AF20706D5D7E90023F9
:10391000F8F772FE0AF1010A0123761007F1080791
:10392000F2D1002B3FF490AB41EC1A0BFFF78CBBAC
:103930000C9009E5029B002B7FF429AEDDE9021211
:10394000C2F31303002B3FF4F7AE20E6002A12DD8A
:10395000214601222846019301F090F85146044681
:1039600001F000F90028019B40F33681392B00F06B
:1039700014810BF13103B94609F8013B059B013372
:10398000374605934646C2E5A24618EE905A18EE11
:10399000104A02460B46F8F779FC42464B4606466B
:1039A0000F46F9F7B9F860B942464B4630463946FA
:1039B000F9F78AF800283FF486AC5FEACB717FF50F
:1039C00082AC009AFFF7E7BB7168284600F0C2FDA1
:1039D0000746002800F04181336902339A0006F15E
:1039E0000C010C30FCF77EFA39460122284601F022
:1039F00045F88046F0E52146284600F0CFFF044612
:103A0000FBE4DDE907239F1A91E4392B00F0C58020
:103A1000B9460133B0E700BF08840E080000F07F0C
:103A200000001C400000144008690C08F8690C08EC
:103A3000059A013237460592464649E5129BC3F185
:103A4000360306E70E988E4901EBC00142464B460D
:103A500051E90201F8F7D0FD5AEC1A9B41EC180B22
:103A600051461AEE100AF9F777F80746F8F75AFDAB
:103A700002460B461AEE100A5146F8F705FC0646B8
:103A80000E98DDF800803037012808F8017B0F46DA
:103A900000F0BF800E9B009ACDF838B013449B46CF
:103AA000C246784B002230463946F8F7A5FD8946D4
:103AB0008046F9F751F80746F8F734FD30370246EB
:103AC0000B4640464946F8F7DFFB0AF8017BDA452A
:103AD00006460F46E5D1DA46DDF838B06A4B59ECB8
:103AE000188B002218EE100A4946F8F7CFFB324631
:103AF0003B46F8F7F3FF002869D118EE102A4B4631
:103B000061490020F8F7C0FB32463B46F9F704F85C
:103B100000283FF453ABD1460AF1FF3A19F8013CB3
:103B2000302BF8D0109B0133059300E54FF0020ACB
:103B3000B0EE49AAF0EE69AAFFF786BA079B002B00
:103B40003FF498AE0F9B002B7FF738AB059A0E938E
:103B5000013A4C4B10921AEE100A39460022F8F73F
:103B60004BFD024616460F460AF10100F8F7DAFC53
:103B700032463B46F8F740FD444B0022F8F786FBFF
:103B800047EC1A6B8046A1F15079FFF781BA059B8B
:103B9000013305933123FFF705BB059BBB4601337A
:103BA0000593392337460BF8013B46469FE44FF017
:103BB000000A56460FE698462EE4AA461AEE104A28
:103BC0001AEE905A109B01330593D146AFE4109B37
:103BD000009A0593FFF7DFBA7FF4CDAEDA077FF5E1
:103BE000CAAEC3E6392BD8D0B9F1000F3FF7C1AE4A
:103BF000C1E6019B022B3FF7D9ADCDF8149062E5E9
:103C0000019B022B3FF7D2AD0F9BCDF81490079389
:103C1000DAE4C24662E74FF0020AFFF715BA1C4B1E
:103C20001C48EA2101F02CFA1B4B0093FFF7C1B8A6
:103C30006B6A00265E603146284600F08BFC0090DF
:103C400090B9164B134800224FF4D57101F018FAC1
:103C50003FF4FAABC0F13C0080E4104B0D483A460B
:103C600040F2EA2101F00CFA6B6A009A1A604FF0F8
:103C7000FF33012209960F930A920793FFF79EBA2A
:103C800008690C08000024400000E03F00001C40D0
:103C90000C840E0824840E08FC830E0858840E0839
:103CA0002DE9F0410469B4EB611F2FDD00F1140E22
:103CB0004E1111F01F0C0EEB84050EEB86032BD07A
:103CC0005EF8262004339D4222FA0CF1CCF1200844
:103CD00018D977461A6802FA08F20A4347F8042B03
:103CE00053F8041B9D4221FA0CF1F3D8A41BA30046
:103CF000053B9B0801330EEB83044EF82310C9B13A
:103D0000043417E0416174460029F9D100230361AE
:103D100000234361BDE8F0819D4288BF00F110029D
:103D2000F4D953F8041B42F8041F9D42F9D8A41B90
:103D30000EEB8404A4EB0E039B1074450361E7D0E3
:103D4000BDE8F0812DE9F04FAE4C2DED028B2468DB
:103D50008BB008EE100A204689460392079304941C
:103D6000FDF7A6FBD9F800302118024611F801BC76
:103D70009978302940F0E5816FF00100C01A0333D3
:103D800000EB030A1C4613F8011B3029F8D0DFF8BA
:103D9000788218F80130002B00F0F7802378002794
:103DA00018F803303D4626462BB116F8013F18F8A7
:103DB0000330002BF9D1049902923046FDF712FC32
:103DC000029A0190002800F09680002D40F0968025
:103DD0003378019503F0DF03502B354600F09880CF
:103DE000C9F80060002F40F0B0802B1B013B072B6F
:103DF000394604DD5B10072B01F10101FADC18EEF6
:103E0000100A059200F0A6FB059A0290002800F027
:103E10007182029BAC4203F11406069680F0E781A2
:103E20000027C2F10103B946059310E0202F00F0EE
:103E300097803946043715F8013C18F80330554689
:103E400003F00F038B40A54249EA030916D915F880
:103E5000013C5B4505F1FF3AE8D1059B5344A34281
:103E6000E4D31846049909920893FDF7BBFBDDE9FA
:103E700008320028DAD11D46A542E8D846F8049B4E
:103E8000069BF61A029BB6101E61484600F072FCB3
:103E9000039B76011C68301AA04200F3B780C0F281
:103EA0002F810027039B019A9B689342C0F2938164
:103EB0000399019A4B68934240F384809D1AAC4267
:103EC00000F3C480CA68022A00F0C681032A00F009
:103ED000BE81012A00F0A28118EE100A029900F0BA
:103EE00079FB5025169A0023284613600BB0BDECD1
:103EF000028BBDE8F08F002D00F01181AD1BAB00EF
:103F00000193337803F0DF03502B35467FF468AF1D
:103F10006B782B2B00F0F2802D2B6ED06E1C0020C6
:103F200018F803104B1E182B65D8737818F8033057
:103F30001039013633BB00B14942019BC9F800601A
:103F40000B440193002F3FF450AFBAF1000F14BFA0
:103F50000025062528460BB0BDEC028BBDE8F08F8E
:103F6000002146F8049B0427894664E701EB8101A0
:103F700003EB4103A3F1100116F8013F18F80330D9
:103F8000002BD8D0192BF1DDD5E7049901922046FA
:103F9000FDF728FB019A002876D1A15C18F80130C2
:103FA000A518002B72D030292C4605D114F8013FFA
:103FB000302BFBD018F80330B3FA83F77F094FF0AA
:103FC000010AF0E6012557B1039BDB68022B65D09F
:103FD000032B67D0012B00F0888045F01005169B5D
:103FE000029A1A60079B019A1A6028460BB0BDEC32
:103FF000028BBDE8F08F2E46F2E60120AB78AE1CB6
:104000008EE700BFEC680C08EC670C08029D061BED
:104010003146284600F0E2FF074678B1721E531180
:104020000699012751F8231002F01F0307FA03F342
:104030000B4203D0BA4200F3E4800227019B0298AE
:10404000334431460193FFF72BFE2BE76E1E002F02
:1040500040F0CB80002E40F0CE807311069A02987B
:1040600052F8232006F01F06012303FA06F6164233
:10407000294618BF47F00207FFF712FE039B5B6853
:104080000193641B02259EE72178254601F0DF019C
:10409000502900F0BF80C9F8005056E7179BC3F1C4
:1040A00001031793179B002B97D0029BDDF8189004
:1040B0001E6900214B464FEA860809EB860003E0A3
:1040C000984243F8041C40D91F4653F8042BB2F120
:1040D000FF3FF5D00132022D3A6000F0C28014F0AB
:1040E0001F0440F0E180212579E7BA077FF575AF1D
:1040F000069B1B681F43FB07D7D46EE700207DE7B4
:10410000DDE90131221A9B1A18EE100A019300F022
:10411000B5FC03461433029006930027C2E6B35C55
:1041200018F80310B018064600293FF453AE16F8ED
:10413000013F18F803100029F9D1801B810001917B
:1041400048E69C1C4FF0000A21E6029B9B689E42B9
:1041500080F28E803346029901EB830201330B61BA
:10416000022D4FF0010151617BD09E42B7DA002B46
:1041700040F3A780029A09EB8303516902F118000A
:1041800083424FEA510140F2AF804C46026841EA57
:10419000C27144F8041B50F8041B83424FEA5101DA
:1041A000F4D8029A9B1A193B9B08013349F8231053
:1041B00009EB8303002940F09B800299A3EB0902DD
:1041C00092104B450A617FD0039B019A9B68013294
:1041D0009342019287DA029918EE100A00F0FAF978
:1041E000169A00231360A325B4E6012735E7069E3F
:1041F0004FF0000942E60298314600F0EFFE074614
:104200002BE7B11E284600F0E9FE00283FF415AF69
:10421000032713E700230193012779E6AC427FF4DB
:104220005BAE012C08D00298611E00F0D7FE00287A
:104230003FF452AE039B5B6807990B60029B0699A3
:1042400001221A610A60169A6225136082E6179AA3
:10425000002A3FF441AEEFE7179A002A7FF43CAE04
:10426000EAE7039B1B68013BA34231D02225B6E657
:10427000029B596818EE100A013100F06BF90746ED
:1042800000283DD002990B6902339A000C310C30A2
:10429000FBF728FE029918EE100A00F09BF907F1CF
:1042A00014093B69029756E7C844C4F1200458F842
:1042B000040C00F05FFAA042BFF615AF029B1B6929
:1042C00055E7029A00231361029A002353617BE7AA
:1042D000631104F01F0459F823200123A340134263
:1042E0000CBF222521257AE6C9F800104B4669B19A
:1042F000043362E7074B0848029ADE2100F0C0FE53
:10430000044B05483A46842100F0BAFE029B19612D
:10431000DAE700BF58840E086C840E0810B40468F5
:1043200009E014F8013FA3F1410CBCF1190F98BF4B
:104330002033934209D111F8012B002AF1D1013425
:10434000046001205DF8044B704700205DF8044BC9
:10435000704700BF2DE9F04F096885B04B1111F08F
:104360001F01029002EB8303039140F08E801D1F1A
:104370000193029B01991C68002341F8043C617879
:104380000134002900F09780DFF87091A846AC4610
:104390009A461E460EE0202900F28B80B24506DACE
:1043A000C44501D2072B5BDD624551D3082314F8C5
:1043B000011FA1B119F801000028ECD00133082B2E
:1043C00006F101063ADCDCF80010090100F00F00EC
:1043D0000843CCF8000014F8011F0029EAD1002E90
:1043E00069D0E04501D9072B73DD624551D2111F19
:1043F000634653F8040B41F8040F9D42F9D2A5EB34
:104400000C0323F00303691C04330CF1010C614518
:1044100038BF04231344002143F8041B9D42FBD200
:10442000019B53F8043C2BB9AA4248D055F8043DEF
:10443000002BF9D0052005B0BDE8F08F6245B6D25B
:1044400000234CF8043C1946ACF1040C0123BDE7F1
:104450000023ACF104084CF8043CB246C446A6E77D
:10446000C3F108018900DCF80030C1F1200E60467C
:104470008B46416801FA0EF73B43036021FA0BF3C8
:1044800040F8043F4045F4D38EE7191D01911D46C5
:104490006FE7039B002BC3D0039B0198C3F120015E
:1044A0004FF0FF33CB4050F8041C0B4040F8043C65
:1044B000B9E7292909D0042005B0BDE8F08F012310
:1044C00005202B6005B0BDE8F08F029901340C6027
:1044D00085E7C3F108039B00DCF80010C3F1200757
:1044E0006446666806FA07F00143216026FA03F184
:1044F00044F8041FA045F4D877E700BFEC670C0828
:10450000F0307047004870475C2300200048704737
:104510005C23002010B4034CD4F8E440A4465DF8BA
:10452000044B60476C22002082B049B15AB16BB194
:1045300013780B601278101E18BF012002B070476C
:1045400001A9002AF3D1104602B070476FF00100B4
:10455000F4E700BF70B5466A05460C465EB1F368E5
:10456000A3B153F82400E8B1026843F824200023E3
:10457000C0E9033370BD1020AFF0BEFE064668628E
:10458000E8B10023C0E901330360C36021220421A4
:104590002846AFF04BFF6B6AF060DB68002BE0D180
:1045A000002070BD012101FA04F6721D9200284618
:1045B000AFF03CFF0028F3D0C0E90146D7E7034B3A
:1045C00003483246662100F05BFD00BF0C840E08F4
:1045D000B8840E0870B5456A04460E464DB13EB12A
:1045E000636A7268DB6853F82200306043F8226027
:1045F00070BD1020AFF080FE0246606220B1C0E9BD
:1046000001550560C560EAE7024B03488A2100F0C6
:1046100037FD00BF0C840E08B8840E08F0B50C6995
:10462000064683B00D4601F1140E0020DEF800109E
:104630001FFA81FC02FB0C334FEA134C090C02FBFE
:1046400001CC01309BB203EB0C4384424EF8043B97
:104650004FEA1C43EADC3BB1AA68A24207DD05EB46
:104660008402013453612C61284603B0F0BD6968AF
:10467000019301313046FFF76DFF019B0746A0B162
:104680002A6901930232920005F10C010C30FBF70C
:1046900029FC294630463D46FFF79CFF05EB840286
:1046A000019B536101342C61DEE7034B03483A461A
:1046B000B52100F0E5FC00BF58840E08B8840E0850
:1046C0002DE9F8430C4628491F46164603F1080217
:1046D00081FB0231092F4FEAE2730546C3EB610308
:1046E00039DD4FF0010C00214FEA4C0C634501F11C
:1046F0000101F9DC2846FFF72DFF014668B3089B4E
:104700004361092E4FF00103036112DC0A340926CC
:10471000B7420BDDBE1B264414F8013B0A22303B96
:104720002846FFF77BFFA6420146F5D10846BDE8C3
:10473000F88304F10909C846344418F8013B0A22F9
:10474000303B2846FFF76AFFA0450146F5D1A6F1A8
:1047500008044C44DCE70021CCE70A46034B04483C
:10476000CE2100F08DFC00BF398EE33858840E084E
:10477000B8840E08030C1B04D3B90004102310F0F6
:104780007F4F04BF0002083310F0704F04BF0001D8
:10479000043310F0404F04BF80000233002805DBD3
:1047A00010F0804F03F1010308BF20231846704723
:1047B0000023E4E7036813F00702014607D0DA0795
:1047C0001FD4980721D55B080B600120704798B271
:1047D000A0B11046DAB20AB908301B0A1A0704BFA2
:1047E0001B0904309A0704BF9B080230DA0703D480
:1047F0005B0800F1010006D00B6070471B0C102015
:10480000E8E700207047202070479B080B600220DB
:10481000704700BF10B50C460121FFF79BFE024612
:1048200018B10123C0E9043410BD034B03484FF411
:10483000A07100F025FC00BF58840E08B8840E0853
:104840002DE9F04F0E691569AE4285B088461446D1
:1048500005DB2A46234635460C4616469846A3688D
:104860006168AF19BB42B8BF0131FFF773FE019019
:10487000002800F08780019B03F1140909EB870AE7
:10488000D14505D24B46002243F8042B9A45FBD86C
:1048900008F1140808EB860B04F11403D8451A46F6
:1048A00003EB85055FD22B1B153B23F00303043379
:1048B0001534A54238BF0423CDE902A7AC461F46F4
:1048C000924605E0000C29D1C34509F1040948D9F5
:1048D00058F8040B85B2002DF4D056464C46002300
:1048E00056F8040B216882B21FFA81FE05FB02EE26
:1048F000000C0A0C734405FB002202EB13429BB22E
:1049000043EA0243B44544F8043B4FEA1243E7D874
:1049100049F8073058F8040C000CD5D0D9F800300D
:10492000544619464D4600222688090C00FB061104
:104930000A449BB243EA024345F8043B54F8046B33
:104940002968360C8BB200FB063303EB1243A445F7
:104950004FEA1342E8D8C34549F8073009F1040982
:10496000B6D8DDE902A7002F02DC05E0013F03D045
:104970005AF8043D002BF9D0019B18461F6105B081
:10498000BDE8F08F034B0448019A40F25D1100F03E
:1049900077FB00BF58840E08B8840E082DE9F0415B
:1049A00012F0030382B0144607462DD10E46A41020
:1049B0001CD07A6A8AB39568002D39D0E3074FF08E
:1049C000000806D4641011D0286898B10546E307A2
:1049D000F8D531462A463846FFF732FF31460346BE
:1049E00038461E46FFF7F6FD6410EDD1304602B0A2
:1049F000BDE8F0812A4629463846FFF721FF2860A6
:104A0000C0F800800546E2E7013B184A52F823202F
:104A10000023FFF703FE0646C9E71020AFF06CFC49
:104A200002467862E0B10023C0E901330360C3604D
:104A3000012138460192FFF78DFD019A054640B1EC
:104A4000012340F27121C0E904310023906003602A
:104A5000B4E7074B07482A464FF4A07100F010FB5B
:104A6000054B04484FF4D77100F00AFBF8680C08B6
:104A700058840E08B8840E080C840E082DE9F047FF
:104A80000D4691462F69AB68496807EB62177C1C9D
:104A90009C4280464FEA621A04DD5B009C4201F1B1
:104AA0000101FADC4046FFF755FD064600284DD0CF
:104AB000BAF1000F00F114000EDD0AF105024FEA11
:104AC000820C034606EB8202002143F8041B93424A
:104AD000FBD1ACF114031844296905F1140319F052
:104AE0001F0903EB810129D0C9F1200E84464FF044
:104AF000000A1A6802FA09F242EA0A024CF8042B88
:104B000053F8042B994222FA0EFAF2D84B1B153BAC
:104B100023F00303043305F11502914238BF042347
:104B2000BAF1000F18BF274640F803A0404637618E
:104B30002946FFF74FFD3046BDE8F087043853F8AB
:104B4000042B40F8042F9942F9D8EFE7034B0448AF
:104B5000324640F2D91100F093FA00BF58840E0893
:104B6000B8840E080B6984460069C01A16D10CF18E
:104B7000140C14310CEB830210B401EB830301E03D
:104B8000944508D252F8044D53F8041D8C42F7D0D6
:104B900005D24FF0FF305DF8044B7047704701209D
:104BA0005DF8044B704700BF2DE9F84F0F6913699A
:104BB000FF1A002F0E4690467AD101F114051432E7
:104BC00002EB830205EB830301E09D4273D253F8AD
:104BD000041D52F8044DA142F7D064D37168FFF769
:104BE000B9FC8146002872D03569D8F81020C7601A
:104BF00008F1140E06F1140009F1140A06F1100C64
:104C00000EEB820200EB8507564600215EF8044B4E
:104C10005CF804BFA3B211FA8BF1CB1A210CC1EBE3
:104C20001B4101EB23419BB243EA0143724546F825
:104C3000043B4FEA2141E9D8A2EB0804153C08F1F6
:104C40001508424524F0030606F1040638BF042681
:104C5000304424F0030238BF002287425244B24459
:104C600016D95646044654F8043B11FA83F10A1447
:104C700002EB134289B241EA0243A74246F8043BE1
:104C80004FEA2241EFD87A1E101A20F00302524454
:104C900023B952F8043D013D002BFAD0C9F8105059
:104CA0004846BDE8F88F334601274646984695E7C3
:104CB000F9DB002792E70021FFF74CFC814668B141
:104CC00001220023C9E904234846BDE8F88F074BB9
:104CD00007484A464FF4107100F0D2F9034B0448DC
:104CE0004A4640F2322100F0CBF900BF58840E084A
:104CF000B8840E0882B08DED000B154B019A13405D
:104D0000A3F15073002B05DD0020194641EC100B78
:104D100002B070475B42B3F1A07F4FEA235208DA3A
:104D20004FF40023002043FA02F141EC100B02B0D3
:104D30007047143A1E2ADABF4FF0004323FA02F2FA
:104D400001220021104641EC100B02B0704700BF59
:104D50000000F07FF8B5046900F1140606EB840446
:104D6000271F54F8045C2846FFF704FDC0F1200318
:104D70000A280B6031DDBE421BD20B3854F8081CE8
:104D800023D0C0F1200C854021FA0CF72F43A4F169
:104D9000080547F07F53AE4243F4401336D28140BA
:104DA00054F80C0C20FA0CF00843024643EC102B8C
:104DB000F8BD0B3808D005FA00F040F07F53002012
:104DC00043F440130246F1E7014645F07F5343F4B4
:104DD00040130A4643EC102BF8BDC0F10B0C25FA2A
:104DE0000CF1BE4241F07F5338BF54F8081C00F16B
:104DF000150034BF21FA0CF1002105FA00F043F44C
:104E0000401340EA010243EC102BF8BD01FA00F018
:104E10000246CBE72DE9F043884683B0012157ECE9
:104E2000106B1546FFF796FB044600284FD0C7F3DA
:104E30000A59C7F31303B9F1000F01D043F48013EB
:104E4000002E019324D068460096FFF7B3FC00289B
:104E500039D0DDE90013C0F1200203FA02F20A435F
:104E6000C34062610193002B14BF02220122A3619F
:104E70002261B9F1000F16D0A9F233430344C0F107
:104E80003500C8F800302860204603B0BDE8F08344
:104E900001A8FFF78FFC019B636101222030226192
:104EA000B9F1000FE8D104EB8203A0F23240C8F858
:104EB00000001869FFF75EFCC0EB42102860204636
:104EC00003B0BDE8F083009B6361019BCBE7034B1C
:104ED0000348224640F20A3100F0D2F858840E0806
:104EE000B8840E082DE9F04383B00E4669460746A4
:104EF000FFF730FF01A9304655EC104BFFF72AFFB2
:104F00003B693169591ADDE90023D31A03EB4113D8
:104F1000002B51EC100B0DDD05EB03594D460246FD
:104F20000B4620462946F7F791FC41EC100B03B0E5
:104F3000BDE8F083C3EB033301EB03573946EEE7DB
:104F4000172870B506460CDD0A490B4D00200024D9
:104F500022462B46F7F750FB013EF9D141EC100BEE
:104F600070BD064B03EBC006D6E9040141EC100B03
:104F700070BD00BF0000F03F00002440F8680C083E
:104F80000139491101F1010C116902F1140303EB1C
:104F900081018B4200EB8C0C16D210B5A0F1040EEF
:104FA00053F8044B4EF8044F9942F9D88B1A153B2D
:104FB00023F0030304331844844504D9002340F844
:104FC000043B8445FBD810BD844505D9002340F837
:104FD000043B8445FBD87047704700BF03694A1102
:104FE000934200F1140009DA00EB830302E053F866
:104FF000042DCAB98342FAD80020704711DD11F0A0
:105000001F010ED010B450F8224000EB820324FAA6
:1050100001F202FA01F18C420CD001205DF8044B40
:10502000704700EB8203E5E70120704753F8042D39
:10503000002AF2D18342F9D800205DF8044B704772
:105040009FED010B704700BF000000000000F87FDB
:1050500010B4034CD4F8E040A4465DF8044B60471C
:105060006C22002049B1FF2A02D80A700120704743
:105070008A2303604FF0FF3070470846704700BF37
:1050800000B50B4C25681446EE681A4685B00346F9
:105090000D464CB107490095CDE90114304606494B
:1050A00000F022F800F0AEFA04490C46F3E700BF26
:1050B00004220020EC840E08FC840E08F8840E08FC
:1050C00008B513460022FFF7DBFF00BF0CB400B5A4
:1050D00083B004AB53F8042B019300F05DF803B0E8
:1050E0005DF804EB02B070470EB410B583B005ABA9
:1050F000064C53F8042B01930146206800F04CF84D
:1051000003B0BDE8104003B0704700BF0422002088
:105110009368013B002B936011DA10B49469A342A9
:1051200009DB0A2907D01368581C1060197008465B
:105130005DF8044B70475DF8044B00F07DB91368CF
:10514000581C106019700846704700BF9BB1F8B535
:10515000134406460F46541E5D1E01E0AC4208D0C3
:1051600014F8011F3A463046FFF7D2FF431CF5D131
:10517000F8BD0020F8BD0020704700BF936810B54F
:10518000144613B95360184610BD00F053FC0023B9
:10519000C4E9013310BD00BF2DE9F04F88469FB030
:1051A00015461C46814618B18369002B00F0A28089
:1051B000924B984500F0A480914B984500F0B18047
:1051C000904B984508BFD9F80C80B8F80C301807F8
:1051D00040F19D80D8F81030002B00F0988000231B
:1051E0000B932978884E059420238DF83130302395
:1051F0008DF832300127002974D02C460B4604E08C
:1052000014F8013F002B00F08F80252BF8D1B4EB70
:10521000050B40F08C802378002B63D000234FF0E7
:10522000FF32CDE90723069309938DF85B301C9379
:10523000013404E0069A07FA03F313430693254664
:10524000052214F8011B3046FAF7CAFD831B00281B
:10525000F0D1069BD90644BF20228DF85B20297827
:105260001A0744BF2B228DF85B202A2970D1059A9A
:105270001168043200290592C0F29B800991697877
:1052800001352E2976D0614C03222046FAF7A8FD7D
:1052900038B1069B001B402404FA00F00343069338
:1052A000013515F8011B5A488DF830100622FAF71F
:1052B00097FD002800F08380564B002B6DD005AA87
:1052C0000092554B424606A94846FBF711FA039057
:1052D000039B013306D00B9B039A297813440B934D
:1052E00000298AD1B8F80C305B0617D40B981FB090
:1052F000BDE8F08F00F07EFB404B98457FF45CAF3B
:10530000D9F80480B8F80C3018073FF563AF414670
:10531000484600F0F5F800283FF461AF4FF0FF3049
:10532000E5E7D9F8088050E7B4EB050BDAD0AA46D8
:10533000C5F1010503E0934536D91AF8011F42462D
:105340004846FFF7E5FE013005EB0A02F3D1C9E755
:10535000A1F13002092A94D8099B15F8011F03EB2B
:10536000830302EB4303A1F13002092AF5D92E2968
:10537000099388D169782A292BD1059BA9781A68C5
:1053800007920433002A05F102000593B8BF4FF0DD
:10539000FF330546B8BF079375E7059B073323F036
:1053A00007030833059396E70B9A23785A440B9228
:1053B00032E7494243F00203099106935FE705AAE9
:1053C0000092154B424606A94846FBF7C1FC0390E4
:1053D0007EE7A1F130020023092A079305F10105B8
:1053E0003FF651AF15F8011F03EB830302EB4303B4
:1053F000A1F13002092AF5D9079344E7606A0C0845
:10540000406A0C08206A0C082C850E0834850E08AA
:1054100038850E08F10601084D51010810B4054CFD
:105420008446134620685DF8044B0A466146FFF740
:10543000B3BE00BF04220020F8B50D461446064650
:1054400008B1836943B3254B9C422AD0244B9C422C
:1054500029D0244B9C4208BFF468A389A269A260AA
:105460001A0722D5236903B322686169D31AEDB202
:1054700099422F4629DD0133A1680139A160511CF1
:105480002160157062699A4216D0A389DB0701D5A5
:105490000A2D11D03846F8BD00F0ACFA0F4B9C42F3
:1054A000D4D17468D9E7B468D7E72146304600F014
:1054B00027F838B92369D7E72146304600F034F998
:1054C0000028E7D04FF0FF37E4E72146304600F0F0
:1054D0002BF90028F6D122680123CDE7606A0C0879
:1054E000406A0C08206A0C0810B4044C03460A46B3
:1054F00020685DF8044B1946FFF79EBF0422002088
:105500003C4B70B51D6806460C460DB1AB69E3B166
:10551000394B9C421FD0394B9C424DD0384B9C425A
:1055200008BFEC68B4F90C3018079AB219D5216994
:1055300011B312F001002FD00020A060606940423A
:10554000A06100292ED0002070BD284600F052FA3C
:10555000294B9C42DFD16C68B4F90C3018079AB221
:10556000E5D4D1063ED5520728D4216943F008037B
:10557000A3819AB20029DCD102F42070B0F5007F3B
:10558000D7D02146304600F011FCB4F90C30216927
:105590009AB212F00100CFD1950758BF6069A060A0
:1055A0000029D0D1120658BF0846CDD543F040039C
:1055B000A3814FF0FF3070BDAC68B3E7616B51B1B0
:1055C00004F14402914204D03046AEF037FFB4F902
:1055D0000C300022626321690022C4E9001223F02A
:1055E0002403C3E7092243F0400332604FF0FF3049
:1055F000A38170BD04220020606A0C08406A0C0878
:10560000206A0C0808B5062000F01AFD0120AEF053
:10561000F5FA00BF8B891A072DE9F0410C46804648
:105620003FD44A68002A58DDE66A002E52D0002294
:10563000D8F80050C8F8002013F4805251D101234B
:10564000216A4046B047431C5ED0A389E66A5F07E3
:1056500005D56368C01A636B0BB1236CC01A216A4D
:10566000024600234046B047411C3CD1D8F80030E8
:10567000002B38D01D2B01D0162B4DD123690022D1
:10568000C4E90032616BC8F8005019B304F1440357
:10569000994202D04046AEF0D1FE00206063BDE8E2
:1056A000F0810E69B6B10D680E609A070CBF4B69A8
:1056B0000023AD1B8B600BE02B463246216AA76AA4
:1056C0004046B847B0F1000CA5EB0C05664413DD6D
:1056D000002DF1DC0020BDE8F0810A6C002AA3DC7B
:1056E000F8E7606DB3E70023636023692360A38953
:1056F000DB04C7D56065C5E7A38943F040034FF0DD
:10570000FF30A381BDE8F081D8F80030002B9CD099
:105710001D2B06D0162B04D0A38943F04003A38190
:10572000D9E7C8F80050D5E738B50B69BBB10D46CD
:10573000044608B18369B3B10D4B9D4211D00D4BA6
:105740009D4213D00C4B9D4208BFE568B5F90C3063
:105750002BB129462046BDE83840FFF75BBF00204B
:1057600038BD6568F2E700F045F9E5E7A568EDE7C3
:10577000606A0C08406A0C08206A0C0838B540B30F
:1057800003690446E3B1174B1D680DB1AB69CBB19A
:10579000154B9C420FD0154B9C4221D0144B9C4280
:1057A00008BFEC68B4F90C3053B121462846BDE877
:1057B0003840FFF72FBF6C68B4F90C30002BF4D1E0
:1057C000002038BD284600F015F9074B9C42E2D175
:1057D000F1E7084B08491868BDE8384000F0C2BA44
:1057E000AC68DFE704220020606A0C08406A0C08FD
:1057F000206A0C0894660C0829570108002070479D
:10580000014900F0AFBA00BF2957010800207047D6
:1058100070B568224D1E02FB05F50E4605F17401B8
:10582000AEF008FE044640B100210C30C4E9001679
:10583000A06005F16802FAF73DFE204670BD00BF8A
:10584000274B2DE9F0411E68B369074653B348362C
:105850004FF00408D6E90134013B04D51EE05A1C80
:1058600004F168041AD0B4F90C50013B002DF6D1B4
:105870001C4B6566C4E90055C4E90253C4E90455EC
:10588000A5610822294604F15C00FAF713FEC4E979
:105890000D55C4E912552046BDE8F08135682DB19B
:1058A0002E46D7E7304600F01FF8D0E74FF4D67108
:1058B0003846AEF0BFFD044668B10560C0F804800C
:1058C0000C302946A06025464FF4D072FAF7F2FD5D
:1058D00034602E46BEE70C2330603B60DBE700BF40
:1058E00094660C080100FFFF2DE9F84F344B354951
:1058F0001A68816290424FF00003C0E912330365D9
:1059000004BF012383610546FFF79AFF68602846BC
:10591000FFF796FFA8602846FFF792FF6F68E860E0
:1059200000240423C7E9024308222146C7E90044B2
:10593000C7E904447C66BC6107F15C00FAF7BAFD74
:10594000DFF88CB0AE68DFF88CA0DFF88C90DFF861
:105950008C801D4BC7F828A0C7E9087BC7F82C909E
:10596000C7F830800822F360C6E90044C6E9044461
:105970007466B460B461214606F15C00FAF79AFDE2
:10598000C6E9086BC6E90AA9C6F83080EE680F4B75
:10599000F360C6E90044C6E904447466B460B461C7
:1059A0002146082206F15C00FAF784FD0123C6E9CE
:1059B000086BC6E90B98C6F828A0AB61BDE8F88F64
:1059C00094660C0801580108090001001200020049
:1059D000B1610108D9610108196201083962010841
:1059E000024B0349186800F0BDB900BF94660C086B
:1059F00029570108836903B976E77047704700BFEC
:105A0000704700BF704700BF704700BF024B03499B
:105A1000186800F087B900BF04220020FD57010874
:105A2000024B0349186800F07DB900BF0422002032
:105A30000D5801089368002B00F085802DE9F04F88
:105A4000B1F90C300C461907804683B0174698B25E
:105A500025D523691BB310F002033D682DD04FF00C
:105A6000000ADFF8BCB25646B9465E453346524698
:105A700028BF5B464046002E52D0216AA76AB8472D
:105A8000002856DDD9F808301B1A8244361AC9F8A6
:105A90000830002BE9D1002003B0BDE8F08F21468B
:105AA0004046FFF72DFD002840F03681B4F90C3058
:105AB0003D6898B210F00203D1D110F0010944D131
:105AC0004E46009746B38205D4F808B040F1838073
:105AD000B3455A4600F2B28010F4906F40F0BF8098
:105AE000206801924946FAF769FCA368019AA3EB82
:105AF0000B012368A1601344B24623600026009B7B
:105B00009868A0EB0A00D14498600028C3D0B4F98B
:105B10000C0080B2002ED6D1D5E900960835D1E729
:105B2000D5E900A60835A0E721464046FFF7FCFD71
:105B300080B3B4F90C3043F040034FF0FF30A38141
:105B400003B0BDE8F08F002070471E46AA46994674
:105B500018461D46009756B388B34A46D4E9041345
:105B60002068B24228BF3246884205D9A16803EBBB
:105B7000010B5A4500F3A680934263DC216AA76AB1
:105B80002A464046B847B0F1000BD2DDB9EB0B090D
:105B9000CAD00120009A9368A3EB0B035D44A6EBE7
:105BA0000B069360002B3FF476AF002ED4D10AF1A0
:105BB000080353E902569A460833002EF9D03246BC
:105BC0000A212846FAF70CF9002800F09C800130E1
:105BD000A0EB0509C1E720682369984216D86369DC
:105BE000B34213D86FF00042B24228BF3246216A56
:105BF00092FBF3F2A76A02FB03F340464A46B8471A
:105C0000B0F1000A95DDA6EB0A0678E7B345DA465F
:105C100028BFB24652464946FAF7D0FBA36822682D
:105C2000A3EB0A035244A3602260002BEBD1214670
:105C30004046FFF779FD0028E5D07AE72068B346B3
:105C400032464EE729460192FAF7B8FB019AA3685B
:105C50009B1AA360236813442360934696E7236846
:105C60002169A3EB010B636903EB430A0AEBDA7AC0
:105C70000BF101034FEA6A0A33445345524684BF8D
:105C80009A46524643052CD511464046AEF0D2FB0B
:105C900000283BD05A4621690190FAF723F9A289DE
:105CA000019B22F4906242F08002A28103EB0B0080
:105CB0002361AAEB0B03C4F814A0A3602060B346D1
:105CC00032460EE729465A46FAF778FB23685B44CA
:105CD000236021464046FFF727FD00283FF456AFDA
:105CE00027E7404600F0F0F803460028DED121699E
:105CF0004046AEF0A3FBB4F90C300C2223F0800335
:105D0000C8F8002017E7721C914627E70C22B4F967
:105D10000C30C8F800200EE74FF0FF30BCE600BFA3
:105D200000FCFF7F2DE9F041884600F1480700267E
:105D3000D7E90154013D0FD4A389012B05F1FF35AB
:105D400006D9B4F90E300133204601D0C0470643CE
:105D50006B1C04F16804EFD13F68002FE8D1304696
:105D6000BDE8F0812DE9F8430746884600F1480672
:105D70004FF00009D6E90154013D11D4A389012B4C
:105D800005F1FF3508D9B4F90E300133214603D0AF
:105D90003846C04749EA00096B1C04F16804EDD19C
:105DA0003668002EE6D14846BDE8F883F0B58B8909
:105DB0000C46990797B007D504F147030122C4E9BF
:105DC0000432236017B0F0BDB4F90E100029054667
:105DD0002DDB6A4600F05CFA002827DB019E06F402
:105DE00070464FF48067A6F50056B6FA86F6394637
:105DF00028467609AEF01EFB30B3A3891A4AAA6280
:105E000043F08003C4E90407A3812060002ED9D0A9
:105E1000B4F90E10284600F051FA0028D2D0A38918
:105E200023F0030343F00103A381CBE7A38913F01D
:105E3000800F14BF40274FF480673946284600265C
:105E4000AEF0F8FA0028D8D1B4F90C309A05B9D4DC
:105E500023F0030304F1470243F002030121C4E9E4
:105E60000421A3812260ADE70158010870B50C46FA
:105E7000B1F90E10002996B016461D4613DB6A468E
:105E800000F006FA00280EDB019901F47041A1F53B
:105E90000051B1FA81F14FF4806349090020296073
:105EA000336016B070BDB4F90C3000221B062A60B6
:105EB00004D540230020336016B070BD4FF48063DA
:105EC0000020336016B070BDF8B51446F9B1CAB100
:105ED00006460D4600F01AFAA04202D32F46384675
:105EE000F8BD21463046AEF0A5FA07460028F6D0A8
:105EF00022462946F9F7F6FF30462946AEF09EFACB
:105F00003846F8BD2746AEF099FA3846F8BDBDE8E8
:105F1000F8401146AEF08EBA38B5446C0CB1002092
:105F200038BD80210546AEF085FA0246686430B17E
:105F3000031F7C3243F8044F9342FBD1EFE74FF04D
:105F4000FF3038BD1F29F8B5054608D8466C0C4609
:105F500017464EB156F8240046F82470F8BD1623B3
:105F600003604FF0FF30F8BD8021AEF063FA0646C3
:105F7000686440B1031F00F17C05002143F8041F51
:105F80009D42FBD1E6E74FF0FF30F8BD1F2938B541
:105F9000054620D8426C0C466AB152F8213053B104
:105FA000012B16D0591C10D00025204642F8245051
:105FB0009847284638BD284600F0F8F822460146A2
:105FC0002846BDE8384000F0DBB816230360012006
:105FD00038BD002038BD162303604FF0FF3038BDB8
:105FE0001F292AD8426C38B50C46054682B152F8B2
:105FF000243002EB84024BB1591C19D0012B15D06F
:106000000025204615609847284638BD012038BD38
:106010008021AEF00FFA0246686458B1031F0021D8
:106020007C3043F8041F9842FBD1E0E7032038BDE1
:10603000022038BD4FF0FF3038BD4FF0FF307047C1
:1060400038B5144B1F281D681FD86A6C044662B10E
:1060500052F820304BB1012B15D0591C0FD0002520
:1060600042F820509847284638BD284600F09EF850
:10607000224601462846BDE8384000F081B8162384
:106080002B60012038BD002038BD16232B604FF057
:10609000FF3038BD04220020124B1F2870B51E6847
:1060A00008D80D46716C044649B151F8240041F8F6
:1060B000245070BD162333604FF0FF3070BD802137
:1060C0003046AEF0B7F90146706440B1031F00F1ED
:1060D0007C0C002243F8042F6345FBD1E5E74FF029
:1060E000FF3070BD0422002038B50B4B1D686C6C6E
:1060F0000CB1002038BD80212846AEF09BF96864C1
:1061000038B1031F00F17C0243F8044F9342FBD1E6
:10611000EFE74FF0FF3038BD0422002038B5174BB1
:106120001F281D6826D86A6C044682B152F82430B4
:1061300002EB84024BB1591C1AD0012B16D000255A
:10614000204615609847284638BD012038BD80217B
:106150002846AEF06FF90246686458B1031F00216B
:106160007C3043F8041F8342FBD1DFE7032038BDB6
:10617000022038BD4FF0FF3038BD00BF04220020A0
:1061800070B50C46084D03460026204611461C46B5
:106190002E60ADF037FD431C00D070BD2B68002B86
:1061A000FBD0236070BD00BFE82B0020ADF024BD04
:1061B00010B50C46B1F90E1000F0B2F8002803DB60
:1061C000636D0344636510BDA38923F48053A381E9
:1061D00010BD00BF002070472DE9F0410C46B1F919
:1061E0000C101F46CB05054616460BD421F48051F2
:1061F000A1813B46B4F90E1032462846BDE8F04175
:1062000000F01EB8B4F90E100223002200F068F866
:10621000B4F90C10EAE700BF10B50C46B1F90E1046
:1062200000F05EF8A389421C0EBF23F4805343F4B0
:1062300080536065A38110BDB1F90E1000F016B84F
:1062400038B50C46084D8446114620461A460023B0
:106250002B606446ADF0C4FC431C00D038BD2B68F5
:10626000002BFBD0236038BDE82B002038B5074D4C
:106270000022044608462A60ADF0B6FC431C00D05C
:1062800038BD2B68002BFBD0236038BDE82B0020E5
:1062900070B50C46084D03460026204611461C46A4
:1062A0002E60ADF0A3FC431C00D070BD2B68002B0A
:1062B000FBD0236070BD00BFE82B002038B5074D30
:1062C0000022044608462A60ADF094FC431C00D02E
:1062D00038BD2B68002BFBD0236038BDE82B002095
:1062E00038B50C46084D8446114620461A46002310
:1062F0002B606446ADF072FC431C00D038BD2B68A7
:10630000002BFBD0236038BDE82B002051F8040C93
:106310000028A0F10400BCBF0B58C018704700BF94
:1063200038B50C46084D8446114620461A460023CF
:106330002B606446ADF04EFC431C00D038BD2B688A
:10634000002BFBD0236038BDE82B002038B500229D
:10635000002304460D46F6F7C1FB28B9204629461E
:10636000BDE8384000F00AB8204605F1004100F0D1
:1063700005F8404261EB410138BD00BFD0B50C4B80
:10638000002206460F46F6F737F9F6F70DFC0446ED
:10639000F6F7B8F8074B0022F6F72EF902460B463F
:1063A00030463946F5F770FFF6F7FEFB2146D0BDC3
:1063B0000000F03D0000F041036800221B68184710
:1063C0007FB503914021054679F01EFD039A18B967
:1063D0000124204604B070BD134E039296F99E33FB
:1063E000002BF5D05CF042FF437A039A53B95CF07E
:1063F0003DFF847A039A2CB90C4B4021284679F052
:106400000BFDE6E7D6F8DC3CB6F9A013B3F908308B
:106410009942DDDD064B00934021064B284679F07A
:10642000FBFC0024D5E700BFF04B0020806A0C087D
:106430009F6A0C088D6A0C08F0B52DED028B0D4695
:106440009DB02021044679F0DFFC002800F0B480E4
:106450005A4E96F99E33ABB1D6F8DC2CB6F9A03380
:10646000B2F90C1003F10A02914203DD40F28D32C1
:10647000934207DC524B2A462021204679F0CCFC7F
:10648000002095E096F98D33022B05D14D4B2A461D
:106490002021204679F0C0FCB6F86433A3F57A7366
:1064A0009BB241F6583293420AD896EDF57ADFED69
:1064B000466AB4EEE67AF1EE10FA03D8434BDAE717
:1064C000434BD8E7D6EDF67AF4EEE67AF1EE10FA21
:1064D000F4D9404FD7F88C3AD3ED096AF4EEC76A85
:1064E000F1EE10FAEAD493ED0B7AB4EEE77AF1EE1E
:1064F00010FAE3D4B6F99A33002B01DC364BBAE735
:1065000096F834240D2A06D80123934013F4215F12
:1065100001D0324BAFE732480EF0DEFD012806D144
:10652000D7F8980A80F038FC98B101281AD00021D9
:10653000602204A80391F9F7BDFF2A49D7F8940A0D
:10654000642303AA7FF084FF48BB03AB0093264B70
:1065500002E0264B0093264B2A462021204679F064
:106560005BFC8DE796F8F43CBBB1224819214CF056
:10657000BBF890B11F4896EDDE8A19214CF0CAF89D
:10658000DFED1D7AB8EEC88A20EE270AB4EEC08A85
:10659000F1EE10FACBDD194BDCE7194BDAE71949BC
:1065A000D7F88C0A642303AA7CF022FF0028CCD001
:1065B0001DB0BDEC028BF0BD0120F9E7F04B0020CF
:1065C000A86A0C08BB6A0C08000000B4F36A0C0847
:1065D000E36A0C08F06B00200D6B0C08226B0C08B2
:1065E000F8860020B36B0C08B76B0C08676B0C08BF
:1065F000426B0C08003900200000C842866B0C0872
:10660000776B0C08C96B0C0808B514F065FDBDE884
:106610000840012113F06CBE2DE9F043DFF85091E2
:106620000546D9F804000368ADB01B690E469847CB
:10663000804614F051FD00210746602214A81391F2
:10664000F9F738FF642313AA4146384614F01CF8C2
:10665000044648B93C4A13AB3146284679F0E4FD7C
:1066600020462DB0BDE8F083A9F5656066F0E0F93D
:10667000B8F1000F03D195F91E30012B0AD1334830
:1066800011F08CFE80B9324A3146284679F0CCFDB3
:106690000024E5E710F0060FE2D0A9F5405011F014
:1066A0007DFE08B92B4AEFE703A9384613F012FE26
:1066B00028B19DF80D305B0601D5274AE4E7DFF8E5
:1066C000B480D8EDEF7AF5EEC07AF1EE10FA4FF023
:1066D0000003C5DD089309930A930DF1200907AB68
:1066E00005AA019304A906ABCDF80090384614F032
:1066F000E5F91A4B0B931A4B0D931A4B0F9348461F
:10670000194B11932FF02AFD059B0E93049B1093B8
:10671000D8EDEF7A069B12938DED0C0A0BAB042299
:1067200093ED017AB4EEE77AF1EE10FA04D5013A6E
:1067300003F10803F4D193E71B680C4A314628465D
:1067400079F072FDA4E700BFD06B0C08F02B00209D
:10675000D96B0C08F06B0C08166C0C08D7BB0C0836
:10676000904E0E08246C0C08FACE0C082D6C0C0808
:10677000F05B0020F04B002008B5054B5B7F9B07CA
:1067800004D5044A79F050FD002008BD0120FCE743
:10679000F05B0020406C0C0870B50C4C054660683E
:1067A00003685B690E46984710B10124204670BD0E
:1067B000A4F5405011F004FE04460028F5D1044A27
:1067C0003146284679F030FDF0E700BFF05B00204D
:1067D000506C0C082DE9F046454EB36A93F8CB5047
:1067E0009BB081468A4665B9424B1B68986A03682C
:1067F0005B6B9847044640B93F4A5146484679F09A
:1068000013FD28461BB0BDE8F0865CF02FFD20216B
:106810005DF060FD58B15CF029FD1F215DF05AFD6F
:1068200088B3364A5146484679F0FEFC0024344B82
:1068300093F8F22F42B193F8F43F2BB1314A51460D
:10684000484679F0F1FC0024514648467AF0BEFBF8
:10685000002188424FF0600202A808BF0C46019157
:10686000F9F728FEB06A036801AA1B6864219847FB
:10687000054680B9244A01AB5146484679F0D4FC1C
:106880002C462546BDE75CF0F1FCA5215DF022FD1C
:106890000028C6D1CBE7002CF3D0D9F808303BB99B
:1068A000D9F8003051465B6B484698470446E8E704
:1068B00051464846FFF7C0FD514607464846FFF798
:1068C0005BFF3840C4B251464846FFF779FD514658
:1068D00004404846FFF760FF51460440484679F0BF
:1068E000CBFC5146044048467AF088FB0440C8E798
:1068F000F05B002008890020646C0C087B6C0C089D
:10690000F04B0020956C0C08AD6C0C0808B5FFF737
:1069100061FF034A82F8E40F024A907108BD00BF8C
:10692000F04B0020D58A0020F7B506460F4679F0D7
:10693000A7FA0446A0B30221304679F065FA05466D
:1069400070B314F0C9FB4FF48071044613F0D0FC0F
:1069500048BB20464FF4007113F0CAFC04460023E4
:10696000019314F0B9FB01A913F05CFAECB1104BE0
:10697000DDED017A93ED007AF1EE677A77EEC77A72
:10698000B7EE007AF0EEE77AF4EEC77AF1EE10FA9D
:1069900006DD084B3A460221304679F03DFA0024E4
:1069A000204603B0F0BD0024D9E72C46F8E700BF2D
:1069B00048760020B86C0C08F8B504460F4679F00C
:1069C000F7FC10210546204679F01EFA58B1204602
:1069D000FFF71AFE064630B9044B3A46102120460E
:1069E00079F01AFA35462846F8BD00BFCC6C0C0881
:1069F00070B505460E4679F0ABF9044678B18021B2
:106A0000284679F001FA50B1074B93F87D3543B130
:106A1000064B32468021284679F0FEF900242046B4
:106A200070BD0446FBE700BFF05B0020E06C0C0883
:106A300038B50D4D0446D5F8980A80F0ADF9012817
:106A400010D0D5F8980A80F0A7F9022804D0204683
:106A5000BDE8384079F07EB904480EF03DFB0128CE
:106A6000F5D138BD0020FCE7F06B0020F88600204F
:106A7000F0B50F4D85B0D5F8D43C0093D5F8D83C8F
:106A80000193D5F8DC3C02936A46D5F8E03C0393C9
:106A900006460F467AF04CFA39460446304679F0FD
:106AA00015FA2040C0B285F8E30F05B0F0BD00BF75
:106AB000F04B00202DE9F84306462748DFF8A89060
:106AC000DFF8A8800F4665F0B3FF0446D9F804004C
:106AD00003681B699847054630B914F0060F03D1C7
:106AE000D9F83830022B09D13946304679F0C0FA4E
:106AF000054618B9002488F807400AE039463046B0
:106B0000FFF78AFD04460028F4D02DB9012388F848
:106B100007302046BDE8F8830821304679F074F943
:106B20000028F3D00D4823F02BF80028EED00C4BB2
:106B300093F8E423B02101FB023203F50053B2F8CD
:106B4000EE21B3F98E339A42E0DD064B3A46082136
:106B5000304679F061F9CDE7A04D0020102D0020DE
:106B6000F02B0020F46C0C08F05B0020D58A00208C
:106B70002DE9F3410E46054614F0AEFA804613F0B7
:106B80006BFB044640B94A4A0121284679F04CFB88
:106B9000204602B0BDE8F081464F78680368314670
:106BA0009B699847044650B978680368DB6C98473E
:106BB000414A03460121284679F036FBE8E7AB68F5
:106BC000002BE5D01021284679F01EF920B3D8ED2E
:106BD000967A98ED950A20EE270AF6F7FDFEDFED8E
:106BE000377AA7F5805320EE270AB3F96433DFED37
:106BF000347A20EE270A07EE903AF8EEE77AB4EE00
:106C0000E70AF1EE10FA07DD2E4B0122102128468B
:106C100079F002F90024BBE74021284679F0F4F826
:106C2000E0B1012E14D0232E12D0042E10D026480D
:106C300000F096FBB5EEC00AF1EE10FA1CDD234B16
:106C400000930122224B4021284679F0E5F8E1E744
:106C5000786803689B6C98470028E8D01D4B1B6838
:106C6000D86A0368DB6998470128014618D11A4A97
:106C7000284679F0D9FACDE7786803685B699847C8
:106C800038B1164BD3F8DC3CB3F90A30002BE5DD04
:106C9000D5E7786803681B6898470B28DED1F0E7D2
:106CA0003146284602B0BDE8F04179F049BE00BF48
:106CB000046D0C08F05B0020156D0C08E02E654299
:106CC0000000C842296D0C08F02B00209F6A0C08B8
:106CD000316D0C08088900203D6D0C08F04B002038
:106CE00070B505460E46FFF797FC084B0446D87171
:106CF00031462846FFF750FD31460028284608BF98
:106D0000002479F0EBFF204070BD00BFD58A002041
:106D1000F7B54C4F3B78002B40F091804A4DAC6A60
:106D200094F8CB4001263E701CB13B70204603B066
:106D3000F0BD7AF00BFA044630B9444A3870137843
:106D400043F001031370F1E751F032F8314650F08F
:106D500013F8A5F5405006F031FB3D4B1E710B2694
:106D600047F006FB013E47F0A1FA16F0FF06F7D107
:106D7000384800F071FF14F0AFF9D0F818222A65F6
:106D800090F88832DA0746D413F0F4FC51F010F88A
:106D90003C2150F0A5FD00232B6100212D4800F07F
:106DA000F1FF2C4811F0FAFA01462B4885F004FB5C
:106DB0002A4B1B68D86A036801211B689847A86A98
:106DC0000368DB6A98470121A86A82F0F3FA50F061
:106DD000EFFF06466868224D03681B68984795F8E0
:106DE00024230146304650F0A3F9A5F5005006F0E3
:106DF000D7FA00264CF002FF4CF028FA3E7089F0DA
:106E0000EFFF05F5005385F8F96FC3F8A40A0123D5
:106E100085F8F53F8AE79B07BFD431460D4804F05B
:106E2000ADFB0023019314F057F901A912F0FAFF0A
:106E3000DDED017AF1EE677AC5ED047AADE7002465
:106E400074E700BFEC2B0020F05B0020F48A0020E8
:106E5000D58A0020F02B00205C57002008890020F4
:106E6000F04B00202DE9F0433F4DAB6A93F8CB3057
:106E700087B007460C461646002B72D062B1012936
:106E800001D0232908D1394B93F8E73F23B90024D7
:106E9000204607B0BDE8F083002C56D0214632468C
:106EA00038467AF013FA04460028F0D014F014F9AA
:106EB00007461BF0F9FB8046384612F0B3FED8B106
:106EC00098F92430022B17D100264FF00009F1B2B7
:106ED00003AA38460191CDF80C90CDF81090CDF86A
:106EE000149013F06DFA019918B103AA40461BF0F3
:106EF0008BF80136032EEAD11D48012106F0BEFCB5
:106F00001B48012106F016FC0021A86A82F052FA03
:106F1000184831F0A3FE50F04BFF00214FF02CFF3A
:106F2000154B1B68D86A036800211B6898470F4BF4
:106F30006968002283F8F52F104BCA1A514251415B
:106F400003F1380085F06EFCA2E7686803685B69AE
:106F500098470028A2D1054B93F8E73F002B9DD11D
:106F600095E7012494E700BFF05B0020F04B002080
:106F7000F02B00203081002008890020D0820020E2
:106F80000020704710B5054C606803685B6A98473D
:106F900010B1A36A93F8CB0010BD00BFF05B0020D6
:106FA00030B52DED028B87B00C46B0EE408AFFF76E
:106FB000E9FF054600B3226863689FED120AD4ED2D
:106FC000027A0392B4EE488AF1EE10FA4FF0000212
:106FD00004934FF00103CDE90023F1EE677A0A48EC
:106FE000CDED057A6CBFF0EE400AF0EE480A68BFBE
:106FF000134603A90CF07CF9284607B0BDEC028BC0
:1070000030BD00BF00000000AC85002007B5019135
:10701000FFF7B8FF30B10199044803B05DF804EB05
:1070200000F0C8BA03B05DF804FB00BFF02B0020ED
:10703000014865F0BFBE00BFA04D002008B500F5B7
:10704000005090F8E53F8B4209D080F8E51F31B140
:1070500050F0AEFEBDE808400F2150F041BC08BD25
:1070600070B500F540560546B36B8B420C4611D007
:10707000012910D0022915D059B950F099FE1B21D1
:1070800050F02EFC0C4A05F5385006211C3055F006
:1070900069FCB46370BD50F08BFE1A2150F020FCE7
:1070A000064AF0E7012100F06DFE50F081FE1D213F
:1070B00050F016FC024AE6E7B46D0C08C96D0C08E6
:1070C000C46D0C0810B500F540520C46537F03F018
:1070D0000101A14208D064F300035377DB0704D415
:1070E00005F062FD024B9C7210BD05F033FFF9E71D
:1070F000D58A002000F54050437F61F34103437778
:10710000014B1973704700BFD58A002010B50446A3
:107110005CF0ACF820215DF0DDF804F50054003897
:1071200018BF012084F8F20F10BD000070B50446AE
:1071300004F580454CF062FDD5F8942A436FC2F8FF
:107140005C32D5F88C2A936604F5A04292F8112D92
:1071500042B904F54054A26AD360D5F88C0A03689A
:107160009B6D9847D5F88C0A0368BDE87040DB6DCD
:1071700018470000F0B52DED028B00F5405583B0A7
:10718000AB6A93F8CB300446002B00F0818000F509
:10719000005797F8E73F002B7AD100F5A04393F80A
:1071A0007034002B74D1686803685B6998470028C5
:1071B0006ED1394B586803681B6898470B2867D015
:1071C00004F580469FED357AD6F8943AD3EDB97A36
:1071D000F0EEE77AF4EEC77AF1EE10FA58D513F034
:1071E0007BFF97F8EC2D01A913F05EFD00284FD02E
:1071F000A86A443052F090FF0346DFED290A93ED70
:10720000000A9B20B7EE001A2BF004FAB5EEC00A74
:10721000F1EE10FA3CDDDDED017A9FED227AF0EE21
:10722000E77AF4EEC77AF1EE10FA31D5D6F88C0A87
:1072300004F5805404F5A66393ED008A0368D3F83F
:107240009C309847DFED187A9FED187AA0EE678A98
:10725000B0EEC88AB4EEC78AF1EE10FA18D504F27F
:107260003454D4ED007AFDEEE77A17EE903A002B15
:10727000B8BF5B4207EE903AF8EEE77AF4EEC77AD1
:10728000F1EE10FA04D59FED0A0AA86A83F0A0FB7C
:1072900003B0BDEC028BF0BDF05B002000000034B9
:1072A000000000009A99193FD4023739C2B8B23DA4
:1072B0000AD7233C08B500F54050806A03685B6933
:1072C0009847F6EE007A20EE270AB5EEC00AF1EEF6
:1072D00010FA48BF9FED010A08BD00BF0000000082
:1072E00038B52DED028B00F580450446D5F88C3A73
:1072F000DFED100A93ED370A04F540547C20B7EE19
:10730000001A2BF087F9A06AD5F8945A03685B69D4
:10731000B0EE408A984738EE400ABDEC028BDFEDB4
:10732000067A05F5BA75284620EE270ABDE83840EA
:1073300070F05CBD0000000000007A4400F50050D1
:10734000B0F91C3C33B9B0F99A030028B8BF4042E9
:1073500080B2704783EAE370A0EBE370F8E70000C7
:1073600038B52DED028B04465BF080FF0368DB68C7
:10737000984720B99FED310ABDEC028B38BD304BE8
:10738000DFED308AD3F8DC3CDFED2C0AB3F90A30AC
:1073900000EE103AB0EE681A5920B8EEC00A2BF091
:1073A00039F904F500554FF4C8720021B5F9A2036C
:1073B000B0EE408A2BF06CF9A5F8A203204610F03D
:1073C000EDF9B5F9A23307EE900AB8EEE77A07EEC9
:1073D000903AF8EEE77A77EE676AB4EEE68AF1EE75
:1073E00010FA11D52046FFF7A9FF07EE900AB8EE74
:1073F000E70ADFED157A38EE668A20EE270A20EEDE
:10740000088A88EE260AB7E777EE877AB4EEE78A2D
:10741000F1EE10FAAEDDB5F99A339FED0B7A00EE7E
:10742000103AB8EEC00A38EE678A20EE070A78EE06
:10743000E77A20EE088A88EE270A9DE70000000020
:10744000F04B002000007A440AD7233C002070470C
:1074500000207047002070477047000000F50E5074
:107460003030704700487047FC9A0C0800F54050D7
:10747000406803681B681847034808602F21117093
:1074800008221A60704700BFB0710C0800F5405028
:10749000406803689B6D184700F5405040680368DA
:1074A0005B6D184700F5405300F5AA405B68083053
:1074B0001B1A58425841704710B500F540500C4611
:1074C000406803689B6E9847012084ED000A10BD58
:1074D00010B500F540500C46406803685B6E984755
:1074E000012084ED000A10BD10B500F540500C4697
:1074F00040680368DB6E9847DFED037A20EE270AC9
:10750000012084ED000A10BD0AD7233C10F01EBDF7
:107510005EF010BB11F022BE62F042BB4CF0BABA72
:1075200028F0D0BE4FF0AABD17F016BE5BF0B6BA79
:1075300059F038BC0FF07EBE10F0EEBD06F0AABBCD
:1075400011F062BD05F080BB05F0DEB805F006B8AD
:1075500060F0AAB80EF0D6BCFFF70CBE0FF024BF47
:1075600010F038BD02F0CABF0FF0AABE5BF046BDF6
:1075700023F094BD05F0D4BF02F04ABC10F046BD24
:1075800006F036BB03F0E8BF06F08ABC05F076B81B
:1075900006F048B80FF044BEFFF7C8BD29F0AEB9F9
:1075A00010F052BA05F050BD09F0E4BD09F0CABCB4
:1075B00009F05CBC1FB500F54053044658680391C0
:1075C00003685B6A984760B1DFED070A03990023FF
:1075D00004F5B3400093B0EE600A1A463C300BF05D
:1075E000C1FC04B010BD00BF0000000013B500F5E1
:1075F0004053044658688DED010A03685B6A98475A
:107600009DED010A18B90024204602B010BD04F512
:10761000B3403C300AF0ECFE04460028F3D00248A8
:107620000121FFF70BFDEFE7F02B0020094A92F84C
:10763000E72F0B462AB100228A604A600A600120C7
:10764000704700F58040D0F88C2A783207CA83E86A
:107650000700F4E7F04B002070B51F4B036000F506
:1076600000530446D3F8740F1C4AC3F81C2E08B10B
:107670001AF020FA1A4B236004F5805393F8742F04
:1076800042B9D3F8705F2DB1284627F073FC284625
:107690001AF00CFA04F58C50083077F0C9FE04F5A6
:1076A0008A500C305EF01EF804F6C44504F66446B9
:1076B000B54204D0183D284627F08EF8F8E7094B6C
:1076C000C4F8983804F6941052F0EEFE04F51060F9
:1076D00052F0EAFE204670BD6C750C08D0720D08A1
:1076E000F44F0D08F01F0D0838B5474B044640F81D
:1076F000043B5EF03DFB04F1100017F0ADF904F11E
:1077000068004BF055FF04F5907022F063F904F522
:10771000866015F019FF04F254501AF0FFF904F6D0
:10772000980028F089FC04F544605EF0FFF804F549
:1077300051604AF00FFF04F5815018304FF06CFA99
:1077400004F58A500C305DF0B5FF04F58C5008301C
:1077500077F05AFE04F58D5004304CF0E5FA04F54C
:10776000945018305FF0E6FC04F580530025274A5A
:1077700083F8BC5204F5965004F595531C330C3035
:10778000136046F001FC294604F5995013F0B6FC4D
:1077900004F5CC5070F0E8FB04F5F050043074F0C0
:1077A00095FE04F5F8501C3076F088FF04F5FC5087
:1077B00077F0BEFB04F5FE50183015F0C3FD04F55C
:1077C0000450303071F000F904F50650303064F0A8
:1077D000C1FF04F50B505DF0FBFB04F5005304F50D
:1077E0000C5083F824530A4D3C3078F0E5F92B68AF
:1077F00013B1084889F0C2FA2046074949F074FDE0
:107800002C60204638BD00BFF44F0D089095002035
:10781000B48B0020D86D0C081C4F0D0810B50FF06C
:1078200037FF5BF023FD0368BDE810405B68184735
:10783000FFF7F4BF10B5044605F08EFF204610F0A8
:10784000D3FD204603F0FEFC2046BDE8104003F0C7
:107850003DBE0000FFF7EEBF70B500F54155143591
:107860000446284616F0D2FF1AF01EFF90F9213088
:107870008BB390F8403373B304F5405304F254567D
:10788000986A443052F048FC0346DFED130A93ED4A
:10789000000A9B20B7EE001A2AF0BCFE94F9883546
:1078A000012B284608BF86ED0E0A002116F074FD54
:1078B000DFED0A7A04F2AC7494ED287A20EE270A00
:1078C000DFED077AA7EE270A304684ED280ABDE8E7
:1078D00070401AF0F9BD70BD00000000CDCCCC3D69
:1078E0006666663FFFF7B8BF10B50121044610F089
:1078F000B5FD98B1174B586803689B6A984768B9FB
:10790000204602F08BF904F5A04393F8113D2BB902
:10791000204602F089F9204602F08EF94FF400115A
:10792000204610F09BFD40B104F5A04393F8113DB3
:107930001BB92AF05DF828F099FA4FF4802120460F
:1079400010F08CFD28B12AF053F8BDE8104028F063
:107950009BB910BDF05B0020FFF7C6BF7FB500F5F7
:1079600080460446D6F88C0A9FED550A6C302DF0FF
:10797000F7FF01A904F599508DED010ACDED020A3A
:107980008DED031A11F05AFE0221204610F066FD1B
:10799000A8B10121204610F061FD80B9494B58681B
:1079A00003689B6A984750B9204602F037F904F5FE
:1079B000A04393F8113D13B9204602F035F9012197
:1079C000204610F04BFD68B93E4B586803689B6A2F
:1079D000984738B904F5A04393F8113D13B92046F0
:1079E00002F02AF90121204610F038FD10B9204696
:1079F00002F07AF94FF40031204610F02FFD28B143
:107A000004F54053986A03689B6C984740212046D0
:107A100010F024FD68B104F58155183528464EF064
:107A2000B9FC04F5805393F94C3113B128464EF05C
:107A3000FBFD4FF48061204610F010FD20B104F5ED
:107A4000815018304EF048FD2021204610F006FDF0
:107A500050B104F54055686803681B69984798B1B0
:107A6000D6F8940A7DF050FC8021204610F0F6FCF8
:107A7000B0B129F0BDFF28F02BF91021204604B049
:107A8000BDE8704010F0EABC20460CF06FF9002809
:107A9000E6D1686803685B6998470028E0D0E3E7AF
:107AA0004FF48021204610F0D9FC0028E1D14FF49A
:107AB0000021204610F0D2FC0028DAD1DDE700BF1B
:107AC000E02E6542F05B0020FFF748BF10B50121B2
:107AD000044610F0C3FC10B1204602F005F98021E5
:107AE000204610F0BBFC58B14FF48021204610F026
:107AF000B5FC28B929F07CFFBDE8104028F0C4B8D7
:107B000010BD0000FFF7E2BF10B5044605F06AFBA8
:107B1000204605F0D7F9204605F0AAFB204611F0D3
:107B2000D5FC2046BDE8104003F070BBFFF7ECBF6A
:107B300010B500F53F5300221F331046012113F802
:107B4000014F14B101FA02F4204301321B2AF6D18D
:107B500010BD00002DE9F0434FF6FF7187B00446D9
:107B600010F07CFC38B12046FFF7E2FF0721024607
:107B7000204602F0EBF804F5405604F50055B36AD0
:107B800093F8CB306BB92046FFF7C0FAB06A95F88E
:107B9000B623036895F834145B6A9847B06A82F09C
:107BA000E3FE5DF011F95CF093FE204611F0ECFA73
:107BB00095F8E73F224A04F5A04683F0010353718C
:107BC00096F8113D04F580475BB9D7F88C8AD8F850
:107BD0000030D3F874904CF011F84BF063FC404641
:107BE000C847D7F8947A4CF009F807F5BA774BF004
:107BF00059FC38466FF05AFF96F8103DCBB995F90D
:107C0000C43CB3B10F4B04941B68986A03681D6DA4
:107C10000D4B059301240623CDE901344FF4C063D5
:107C2000009306AA12E90600084BA84720B186F87F
:107C3000104D07B0BDE8F083054816F0E9FF00BF1E
:107C4000D58A002008890020A175010832180D0886
:107C5000EC6D0C08FFF77EBF70B500F5805606F29C
:107C60007C5300F540541B68E36306F5B163DFED18
:107C7000117A1B68236406F5A76393ED000A30EEC2
:107C8000270A05462AF09CFCE36BA364236C84ED71
:107C9000110AE3644FF6FF71284610F0DFFB38B19C
:107CA000D6F82C2528460921BDE8704002F024B8FA
:107CB00070BD00BFDB0F494070B500F5405504466C
:107CC000AB6B002B50D000F5005696F8E83F002B28
:107CD0004AD0002386F8E83F5BF0C8FA0368DB6807
:107CE0009847002840D0D6F8D42CB2F90A3006EED6
:107CF000103AD6F8D83CB3F90A3007EE903AAB6B9D
:107D0000012BB8EEC66AF8EEE75A2ED195ED0F7A40
:107D100095ED105A67EE257A65EE656AE6EE057A0E
:107D2000E6EE076A04F5805404F27C5304F5B1646E
:107D300094ED007A93ED006A27EE877AA6EE867AB4
:107D4000BDEEC77A17EE101A518193ED007AD6F87E
:107D5000D82C67EE877A94ED007AE6EEC77AFDEECE
:107D6000E77A17EE903A538170BD95ED137AD5ED11
:107D7000127A67EE656AE6EE276A67EEA57AE6EEA6
:107D8000077ACFE738B505462DED028B00F5405454
:107D9000B1B128460FF020FBB0EE408A94ED110AF5
:107DA00030EE480A2AF022FCDFED157AB0EEC00A68
:107DB000B4EEE70AF1EE10FA0FD5BDEC028B38BD38
:107DC000A36B022BF9D10FF0F3FAF2EE047AB4EEC2
:107DD000E70AF1EE10FADCD5EFE79FED0A0A84ED31
:107DE000118A38EE008AB0EE480AF5F73BFC84EDC4
:107DF000120AB0EE480AF5F78BFD84ED130ADCE7B2
:107E0000C2B8B23DDB0F4940012100F5995013F093
:107E1000D5B80000FFF7F8BF10B5044610F09EF883
:107E20001021204610F01AFB70B1204601F048FEE8
:107E30004FF40011204610F011FB28B929F0D8FDAD
:107E4000BDE8104028F012B810BD0000FFF7E4BFF5
:107E5000F8B50446254605F051FF224B45F8383B5E
:107E6000214B6465C4E91634204BC4E91834204B17
:107E7000A36604F17C0019F0A1F904F1980019F04F
:107E80009DF904F1B40019F099F94FF6FF76194BFA
:107E9000C4F8C83004F1D000A4F8CC6019F08EF911
:107EA0004FF0FF37144B1549C4F82C7128461D605C
:107EB00049F01AFA04F5A070A4F87470A4F8906060
:107EC00019F07CF904F5AE7019F078F904F5BC707E
:107ED00019F074F9002384F88C31C4F8B0312046CD
:107EE000F8BD00BF20C40C08A9750108AD750108D4
:107EF000B17501080000FFFFA88A0020E02C0D08E2
:107F000010B5044605F0FAFE0A4B236001232387CF
:107F100004F13C0019F052F904F14C0019F04EF94B
:107F200004F15C0019F04AF904F16C0019F046F90B
:107F3000204610BD68CC0C082DE9F043044689B0FA
:107F4000FFF7D2FB874B236004F50F50203004F578
:107F5000005502F069F804F50E532433C5F8EC3CE3
:107F6000062385F8F03C4FF07C5705A904F53356FD
:107F700004F53450059752F031F906F15C0087F0B2
:107F800025FE04F5355619234FF0000904A985F89C
:107F90003C3D06F10C0085F8349D049752F01EF923
:107FA00004F5365706F1280087F010FE4FF001085F
:107FB0001823203785F8883D384685F8808D77F07E
:107FC000D3FE06AE684BC5F8A03D3146381D8DF88E
:107FD000188049F0ADFF04F53750203077F0AEFE41
:107FE000624B634FC5F8E03D04F5375031463830F9
:107FF000069752F0F3F804F53850314606970430EE
:1080000004F5385752F0EAF81C375A4BC5F81C3EB5
:1080100007F1080087F0DAFD0723C5F8783F85F8F7
:10802000708FA5F87C9F4FF4D27019F03DFDC5F814
:10803000740F04F53E5087F0C9FD04F53F5004303D
:1080400087F0C4FD4C4B1A6802B91F6004F5405814
:108050004A49384604F5B74749F046F91037484BC6
:10806000C5F81C3E4046C8F80470083079F068F93D
:10807000444B07934FF07E55434BC8F83C50C8F82B
:1080800048500694009304F5415096E80C004FF4D4
:108090000071143016F0AEF804F5565068F0B6F9D9
:1080A00004F5944003A95C30039552F0BDF804F543
:1080B000944003A97030039552F090F804F5944071
:1080C0007C3019F07BF804F595404FF400412830DE
:1080D00016F0C8FD04F59640283066F005FB04F55F
:1080E000964004F5804564304AF058F8274BC5F8AF
:1080F000643B04F59640264B2649783004F59746B4
:108100001860183649F0F0F8FF2385F8AC3B85F885
:10811000B43B2149304649F0E7F8204B1D6815B1C2
:108120001F4888F02BFE04F597403C301E604CF051
:1081300009FF1C4B1C48186004F5A84260322B460E
:1081400014269DB206FB05010133097C0029F8D1F4
:10815000164B1D80164BD3F80080B8F1000F2BD0C2
:108160001448DEE76C750C08546D0C08946D0C080F
:108170000000A040D0720D08C08E0020DC6E0D08FB
:10818000F4750C08A57501085C750C08B06D0C0839
:10819000949500203C810D08F4040E0828960020D8
:1081A000F86D0C08708B00206CB20C086E8B0020F0
:1081B0002C8B0020196E0C0804F5A8401A6003A946
:1081C000584B0393743052F009F804F5A94004F5B4
:1081D000A045143005F092FD534BC5F8943404F5D6
:1081E000A940503005F08AFD04F5AD464F4BC5F867
:1081F000D03404F5AA4060360830FFF729FE304637
:1082000005F07CFD4A4BC5F8E03606F1380086F0F3
:10821000D9F8484BC5F8183704F5B140383005F0A7
:108220006DFD454BC5F8B83804F5B140783005F020
:1082300065FD424BC5F8F83804F5B24085F8308941
:10824000343005F05BFD3E4BC5F8343904F5B240DF
:108250006C3005F053FD3B4BC5F86C3905F6A413A3
:10826000002604F5B3401E605E609E603C3005F061
:1082700045FD354BC5F8BC3904F5B340743005F005
:108280003DFD324BC5F8F43904F5B440383005F003
:1082900035FD2F4BC5F8383A04F5B440703005F081
:1082A0002DFD2C4BC5F8703A05F6EC2304F5B640CD
:1082B0001E605E600830FFF723FE384605F01EFDA5
:1082C000254BC5F8903B04F5B740483005F016FD46
:1082D000224BA5F8008C04F5B840C5F8C83B143013
:1082E000FFF70EFE1E4BC5F8143C012385F8993CA0
:1082F00004F5B94705F54A632C371E605E609E6041
:10830000384605F0FBFC174BC5F8AC3C05F6E845D4
:1083100007F148002E606E6087F058FC204609B0D7
:10832000BDE8F083CDCC4C3DE8C00C089CC10C08E6
:10833000D4C40C0874C50C0830C60C08E0C60C0880
:1083400090C70C0838C80C08E8C80C0888C90C0885
:1083500030CA0C08E0CA0C08E4CD0C0890CF0C0819
:1083600030CD0C0864D00C0838B5054B1C68236868
:108370000A461D68034B01462046A847002038BD29
:1083800008890020F02B002010B588F035F8064C45
:10839000064B18602046FFF7CFFD2046044A0549EA
:1083A000BDE81040ADF000BEF02B00200889002091
:1083B000A8F20020597601080120704790F82C306F
:1083C0008B4286BF0C3150F821000020704700001E
:1083D00090F82C308B4286BF0C3150F821000020E1
:1083E00070470000FA207047024B986B431E5842BA
:1083F00058417047F05B0020024B986B831E584237
:1084000058417047F05B0020034B986A08B181F037
:10841000BFB80248704700BFF05B0020E0750C0851
:1084200038B5036A374D43F4E0520262426A42F4BF
:10843000E0524262826A42F4E0528262D5F8942AA3
:108440000446E2B143F4F8430362D5F8940A7CF0A1
:108450002BFB38B1636A43F480436362A36A43F43D
:108460008043A362D5F8940A7CF00EFC38B1636AAD
:1084700043F400536362A36A43F40053A362224BA4
:108480001D6845B1192128464AF02EF918B1236A12
:1084900043F4807323621D4B93F8F43C6BB1636A21
:1084A00043F48073636245B1192128464AF04EF9BE
:1084B00018B1A36A43F48073A362154B93F8543444
:1084C000013B012B0BD8D4E9082343F480036362FA
:1084D000A36A42F4800243F480032262A362236A07
:1084E00043F080432362636A43F080436362094B35
:1084F0009B6A93F8C1301BB9A36A43F08043A3621F
:1085000038BD00BFF06B00207C8B0020F04B0020BA
:10851000F07B0020F05B002013B54FF45670019102
:1085200019F0BCFA044620B1019959F085FB024BC1
:108530002360204602B010BD9C760C0800207047D6
:10854000704700000320704708207047034B1878DD
:1085500010B9034B93F8F60F704700BF6C8A0020E8
:10856000F04B0020704700007047000008B50C4B2E
:10857000D3F8940A68B910230A4A926A43F040007B
:1085800022B192F8CB200AB143F0C00040F00100C4
:1085900008BD7CF089FA0028EDD01823ECE700BF75
:1085A000F06B0020F05B002038B5C5780B46352D08
:1085B000044628BF3525352200211846F7F77AFFF3
:1085C0002A4604F10C01BDE83840F7F78BBC0000E7
:1085D0001FB5184C94F81E11A4F1280014F09CFE4D
:1085E00078B194F81E11A4F1280014F097FE40B160
:1085F00094F81E11A4F1280004B0BDE8104014F056
:108600008FBE002301930293039312F065FD01A92D
:1086100012F01AFB20B101A82DF0A0FD04B010BD8E
:1086200022F07AFD90F8C432B02202FB030090EDF4
:108630002F0AF3E7F04B002008B50D4B986AA8B15C
:10864000443051F069FD034693ED000ADFED090A5D
:108650009B20B7EE001A29F0DDFFDFED077A20EE50
:10866000270ABDEEC00A10EE103A18B208BD00BFCE
:10867000F05B0020000000000000C8422DE9F04F30
:10868000DFF8D880344F8DB00446042508F5005635
:1086900017F8019BB8F9C03309F1FF3A43FA0AF31E
:1086A000D90742D5207C52F065FF8346207C53F0E9
:1086B00021FF00F121039B4505D2207C0DB0BDE8D0
:1086C000F04F54F059BBBAF1030F2ED8DFE80AF08F
:1086D0000234393ED6F88C0A03689B68984700F14B
:1086E00094035A69D3F800A0D3F804E0D868196954
:1086F000D3F818C008925A6A1B6ACDF82520CDF825
:10870000293062222123CDE9003206900791207C96
:10871000CDF80CA0192303AAC221CDF810E0CDF8A2
:1087200014C08DF8249052F08FFF013D15F0FF0525
:10873000AED10DB0BDE8F08FD6F88C0A0368DB68C7
:10874000CCE7D6F88C0A03681B69C7E7D6F8943AD9
:1087500003F50273C5E700BF60770C08F04B0020FB
:1087600013B504460748019108F032FB30B901996E
:10877000204602B0BDE8104054F0A2BB042002B075
:1087800010BD00BFF8800020014808F06BB900BFA1
:10879000F880002058F0B4B910B588B0044655F000
:1087A00081FD0B4B986A38B90A4A0621204608B069
:1087B000BDE8104055F05EBD69461E2280F0ECFE1B
:1087C000054A6B460621204655F054FD08B010BD01
:1087D000F05B002028760C0832BE0C08034A92F8A1
:1087E000D03C013382F8D03C54F0FABDF04B00206D
:1087F00007B50846019118F03BFE38B104480199CD
:1088000002F0D2FB002003B05DF804FB0420FAE77D
:1088100014890020162A10B40C4605D0542A03D01F
:108820005DF8044B54F06ABB0323237001205DF80C
:10883000044B704710B5074B93F9BC2B40F6CD3471
:1088400040F6CD13002A08BF1C4654F0FDFC20431F
:1088500010BD00BFF06B002010B5044619F026F9DA
:10886000204610BD10B50C4C94F8E73F7BB904F5D9
:108870008054606803689B6D984750B960680368CE
:108880005B6D984700280CBF0220032010BD01201B
:10889000FCE70420FAE700BFF04B002010B44C695D
:1088A000012C05D101465DF8044B034802F0ACBE33
:1088B0005DF8044B54F0B0BDF02B00202DE9F341DE
:1088C000B1F90430002B06460C46154635DB4FF057
:1088D0000008CDE900281A4FB1F902209FED190ACE
:1088E000D7F8D41C4FF47A7358F0FAFB0123CDE982
:1088F00000539FED140AB4F90020D7F8D81C4FF4A8
:108900007A73304658F0ECFB9FED0F0AB4F904205F
:10891000D7F8DC1C43463046CDE9005858F0E0FB60
:10892000CDE900589FED070AB4F90620D7F8E01CFE
:108930004FF47A73304658F0D3FB02B0BDE8F081B3
:10894000F04B00200000FA4400007A440B4B93F8EF
:108950007D2572B95A7F92060BD1A3F5805213F888
:10896000193C43B992F8ED3F002B14BF04200120BD
:108970007047052070470320704700BFF05B002060
:1089800008B5074B93F9B433032B03D0BDE8084077
:1089900055F0E8BC034A022155F06CFC042008BDE8
:1089A000F04B002040760C08084BD3F82C2492079B
:1089B00001D454F095BA03F52A5393ED000ADFED84
:1089C000047AB8EEC00A20EE270A7047F04B002068
:1089D0000AD7233C10B594B0044603A818F0EEFB68
:1089E0001C4B5868036803A91B6E984778B3002195
:1089F00003A818F0C1FC50B3247C88F0F1F9059B62
:108A0000DDED047A0893069B09930023F8EEE77ADC
:108A10009FED117A0B930C930D930E930F9310937C
:108A2000119312934FF6F853ADF84C300023962271
:108A300067EE877A8DF84E303323CDE90032079008
:108A400007AA57212046CDED0A7A52F0FDFD14B059
:108A500010BD00BFF05B00200AD7233C30B52DEDE0
:108A60000A8B604B05465868036891B05B6A98476B
:108A700000284ED05C4B1B68062B00F29F80DFE87D
:108A800003F00404044C6A85480058489FED588A56
:108A90000AF04CFC90ED00CAD0ED01BA90ED029ABC
:108AA000F0EE489AB0EE48AAF0EE488AF0EE48AAF6
:108AB000B0EE48BA40F6F8542D7C88F091F90023C6
:108AC0000D930E9301238C228DF83E303323CDE994
:108AD00000320390B1EE499AF1EE688AB1EE488A0D
:108AE00003AA552128468DED04CACDED05BA8DEDBA
:108AF000069A8DED07BACDED08AACDED098A8DED68
:108B00000AAACDED0B9A8DED0C8AADF83C4052F0DF
:108B10009BFD11B0BDEC0A8B30BD34480AF006FC59
:108B200090ED00CAD0ED01BA90ED029A2F480AF0FC
:108B300001FC90ED00BAD0ED01AAD0ED028A2B48DD
:108B40000AF0FCFB4FF4406490ED00AAD0ED019ACE
:108B500090ED028AB0E725489FED259A0AF0EAFBDE
:108B600090ED00BAD0ED01AAD0ED028A1F480AF0BC
:108B7000E5FBF0EE49BA90ED00AAD0ED019A90ED38
:108B8000028AB0EE49CA40F6074495E71748DFED80
:108B9000188A0AF0D3FBF0EE68AA90ED00AAD0ED97
:108BA000019A90ED028AB0EE68BAB0EE689AF0EEE3
:108BB00068BAB0EE68CA40F63F447DE79FED0C8A84
:108BC0000024F0EE489AB0EE48AAF0EE488AF0EEA3
:108BD00048AAB0EE48BAB0EE489AF0EE48BAB0EE05
:108BE00048CA69E7F05B0020E4890020AC850020DA
:108BF000000000002DE9F0412DED048B304B93F87F
:108C0000ED2F8AB0002A56D003F500579FED2D7A3C
:108C1000D7F88C2A90F81080D2ED1D7A92ED1B9A2D
:108C2000D2ED1C8A67EE877A03F58053FDEEE77A72
:108C30005E6817EE903A1CB2336830465B6E29EEE0
:108C4000079A68EE878A9847BDEEC00A304610EE54
:108C5000103A1DB233689B6E9847DFED1B7AD7F848
:108C6000943AB4EEE70A5F6B3368B0EE408AF1EEF7
:108C700010FADB6E58BFB0EE678A30469847BCEEFC
:108C8000C88A0023069318EE103AB722ADF82430B4
:108C90001A23CDE900323E2103AA40468DED039A06
:108CA000CDED048A05978DED070AADF82040ADF8AB
:108CB000225052F0C9FC0AB0BDEC048BBDE8F08133
:108CC000F04B0020E02E654200FF7F472DE9F04188
:108CD0000E46A0B0751E2249804648220EA8EDB26D
:108CE000F7F700F9112D30D820AB03EB850353F8CB
:108CF000487C3B683846DB6C98473B6804461B68F9
:108D0000384698472DB3174B012D04BF03201C464E
:108D10000023122202908DF8102098F8105003932F
:108D20008DF811608DF81230232221460DF11300C9
:108D300094B9F7F7BFFB86222E23CDE9003240F22B
:108D4000B31102AA284652F07FFC122020B0BDE8E1
:108D5000F081054C1B20DBE7F8F784FCEBE700BF54
:108D6000B45F0C0873110E0864760C082DE9F04FFF
:108D70002DED028B1A4B047CD3F88C3A8DB0D3F8CE
:108D80008480D3F88870D3F88C60D3F8905093ED3A
:108D9000258AD3F898B0D3F89CA0D3F8DC9088F05B
:108DA0001FF800238DF82C3016222523CDE9003240
:108DB000029002AA532120468DED078ACDF820B0FB
:108DC000CDF824A0CDF82890CDF80C800497059616
:108DD000069552F039FC0DB0BDEC028BBDE8F08F6A
:108DE000F06B0020054B9B6A2BB193F8CA0000285A
:108DF00008BF022070470220704700BFF05B0020D0
:108E000008B5034B586803681B68984708BD00BF46
:108E1000F05B0020014B93F8ED0F7047F04B002002
:108E200070B52B4E2DED028B0546706891ED018AD1
:108E3000036886B05B6A0C46984750B9BDEEC88A95
:108E400018EE103ADB0704D4022006B0BDEC028B0A
:108E500070BDD4E904012AF051FC0028F4D002A826
:108E600018F0ACF902AA2146284658F093F80028D9
:108E7000EAD0184902A818F007FB03460028E3D1FE
:108E8000DFED150A00900246B0EE600A134802A911
:108E90000AF068F8D0B1706803685B6A98470446C6
:108EA00008B10020D1E70E480222042105F0A2FA01
:108EB00060B1DFED090A094800942346B0EE600A6C
:108EC000224602A90AF04EF80028EAD10420BCE7A5
:108ED000F05B00206C76002000000000AC850020D4
:108EE000F02B002008B591F82020032A0B4617D15B
:108EF000D1ED027A9FED0B7A93ED060A0A4BF0EE64
:108F0000E77AF4EEC77AF1EE10FA4CBF01210021A6
:108F100058680FF04FFD002814BF0020042008BD42
:108F20000220FCE700000034F05B002010B52DEDBE
:108F3000028BD1ED007AF5EEC07AF1EE10FA82B034
:108F40000C4604DA042002B0BDEC028B10BD9FED8C
:108F50001C7AF4EEC77AF1EE10FAF3D891ED030A19
:108F60009FED188AF0EEC07AF4EEC87AF1EE10FAAE
:108F70001FD5D4ED037AD4ED010A94ED000A12480E
:108F8000F4EEC87AD4ED027AFDEEE77AF1EE10FA4B
:108F9000CDED017ADFED0D7A9DF9041060EEA70AA0
:108FA00020EE270AACBF0122002201F079FF002049
:108FB000C9E7F7EE000A29F03FFA0028C2D0D8E747
:108FC0000000B443000000341489002035FA8E3CC0
:108FD00091ED010ADFED187AB4EEE70AF1EE10FA2E
:108FE00007B526DBD1ED007AFCEEE77ACDED017A0C
:108FF0009DF80430042B04D8DFE803F007071116AE
:109000001B00042003B05DF804FB0C4B5868036898
:109010001B6F9847002814BF00200420F2E7074B7D
:10902000586803685B6FF4E7044B586803689B6FEC
:10903000EFE70220E6E700BF00000034F05B00200D
:1090400008B5D1ED007A9FED157AF0EEE77AF4EEEF
:10905000C77AF1EE10FA1DD5D1ED017AF0EEE77A7C
:10906000F4EEC77AF1EE10FA14D50D48022203216E
:1090700005F0C0F980B10A480121FDF7DFFF09487A
:1090800090F84435012B03D000F5A86030F03CF88F
:10909000002000E0022008BD0420FCE700000034AE
:1090A000F02B0020F07B002010B5D1ED007AFCEE13
:1090B000E77A17EE903A9CB2012C02D0022C06D02F
:1090C0004CB9064821465EF0B1FB002010BD0448B3
:1090D00003F040F8F9E70420F8E700BF68770020C4
:1090E000F02B00201FB5D1ED017A0B7CFCEEE77A66
:1090F000CDED027AD1ED007A0093FCEEE77AD1ED66
:10910000030ACDED037A91ED020A9DF808309DF82F
:109110000C20014602480DF071FF05B05DF804FB1C
:10912000F02B002010B5094C637FDB070CD4022222
:109130000521A4F5405005F05DF928B90222114639
:10914000A4F5405005F056F9002010BDF05B00205A
:1091500010B5D1ED007AFCEEE77A044617EE903AAE
:1091600013F0FF030FD10F4B58680368D3F8883012
:10917000984708B1002010BD0B4A2046062155F043
:1091800079F80420F7E7012B09D1064B58680368EA
:10919000D3F88C3098470028ECD1044AEDE7022040
:1091A000E9E700BFF05B002070760C0880760C08C1
:1091B0009FED0B7A01F10C03F1EC017AF4EE677A82
:1091C000F1EE10FA0AD6F0EEE77AF4EEC77AF1EE95
:1091D00010FA03DC9942EFD101207047002070475C
:1091E00000007A4430B52DED028B8DB0002305468A
:1091F00003930493059311F06FFF03A911F024FD6D
:1092000058B311F069FF00F55D7393E8070006ACF1
:1092100084E80700DDED060A9DED070A2D7CF1EEDE
:10922000600AB1EE400AF4F73FFC2046B0EE408AF7
:109230002CF094FFDFED0B7A089B0B93012228EEB4
:10924000278A0C23CDE90032A82109AA28468DEDF2
:10925000098A8DED0A0A52F0F7F90DB0BDEC028BC8
:1092600030BD00BFE02E6542282938B505461AD02A
:1092700008D8242922D0272908D02846BDE838401C
:1092800058F056BA4029F8D1012405E0122153F0D4
:1092900085FD044610B90024204638BD297C0C48C1
:1092A0004BF076F8F8E7162153F078FD04460028D5
:1092B000F1D0297C06484BF045F9EDE70C2153F03D
:1092C0006DFD04460028E6D02846FFF78BFFE3E754
:1092D000AC77002038B5144C637FDB070D4609D40A
:1092E000A36A93F8CB303BB901221146A4F518705C
:1092F000FDF70EFD002038BD14F8193C02226BB1B9
:109300000521A4F5405005F075F80028F2D095ED40
:10931000000A606801210FF04DFBEBE70921A4F57D
:10932000405005F067F8E5E7F05B002010B51E4CF3
:10933000637FDB070CD4A36A93F8CB3043B114F8F6
:10934000193C3BB101220821A4F51870FDF78AFDF4
:10935000002010BDD1ED007A9FED147AF0EEE77A8F
:10936000F4EEC77AF1EE10FA0BD511480222112162
:1093700005F040F890B9022211460D4805F03AF880
:10938000E6E7606803681B6898470428E0D06068D7
:1093900003681B6898471428E7D1D9E7054840F6C9
:1093A000C41108F02BFAD3E7F05B00200000003472
:1093B000F02B0020A884002070B58B8BC12B0546B4
:1093C0000C463CD8BB2B0CD8542B6AD02ED8113B62
:1093D00099B2052918D921462846BDE8704059F0B0
:1093E0005BB8BC3B052BF6D801A151F823F000BFB8
:1093F000DD940108EB940108D7930108D793010885
:109400008794010891940108052BE4D801A151F833
:1094100023F000BFC7940108D7930108D793010830
:10942000D794010839940108A3940108732B22D022
:10943000B22B24D0552BCED10222092145E04AF28D
:109440001146B34237D00AD8D12B26D0B3F5967F38
:1094500035D0D02BBFD1BDE87040FFF725BE4AF212
:109460001246B34223D04AF21346B342B3D1BDE809
:109470007040FFF75BBFBDE87040FFF757BDBDE828
:109480007040FFF7A5BD2146BDE87040FFF7C8BC9E
:109490002146BDE87040FFF75BBEBDE87040FFF7B6
:1094A00021BE21462846BDE87040FFF71BBDBDE840
:1094B0007040FFF70FBFBDE87040FFF733BEBDE857
:1094C0007040FFF7BDBD022205210A4804F092FF5B
:1094D00048B9042070BD02220621F6E702210648A1
:1094E00006F0EAF8F4E70020F4E70221024806F06B
:1094F000AFF8EDE7F02B0020F880002008B591EDE3
:10950000007AF6EE007AB4EEE77AF1EE10FA06DDB4
:10951000044801220521FDF7A5FC002008BD042018
:10952000FCE700BF9059002030B52DED028BCD78BF
:1095300093B0272D28BF27250C462722002108A8F5
:10954000F6F7B8FF2A4604F10C0108A8F6F7CAFCA2
:10955000454B586803685B6A984748B19DF8465088
:109560009DF94630690607D54048012109F020FAE7
:1095700013B0BDEC028B30BD00244FF07E52002BA7
:10958000049207940694059427DA04A82BF0A0FC13
:10959000EA0701940294039405F006032BD4002BF0
:1095A000E2D10D9B01930E9B02930F9B03932F48D7
:1095B00009F07CFA9DED100A0446F8B140F2F33050
:1095C000B7EE001AFFEE000A29F024F827482346D8
:1095D00001AA04A909F072FACAE7099B04930A9B3D
:1095E00005930B9B069304A80C9B07932BF076FC2A
:1095F0000028CDD1B8E7062BB6D1D8E7DFED1C0A9D
:1096000040F2F630B7EE001A29F004F8F6EE000A40
:10961000B0EE408A28F010FF18BBB6EE007A154B6A
:10962000DFED156AD3F8983AB4EEC78AF1EE10FA76
:109630000ADD38EE478A93ED060A38EE088A20EEF6
:10964000260A28EE000AC1E7D3ED077A37EE488AEA
:1096500067EEA67A38EE088AF0EEE77A27EEC80AB7
:10966000B4E79FED030AB1E7F05B0020AC85002072
:1096700000000000F06B00200AD7233C2DE9F047E2
:109680009CB0824608460EA9FEF78EFF7B4B5868B9
:1096900003685B6A984750B19DF86C20012A09D095
:1096A000D31F022B06D97648012109F081F91CB09D
:1096B000BDE8F087BDF8683003F0070803F038090B
:1096C00003F4E07703F4806603F400649B0501D59E
:1096D000002FE8D00025059506950795B8F1000FF5
:1096E0002FD1DDED117A0F9B0593083A109B06935D
:1096F000F1EE677A012ACDED077A07D8614805A90E
:1097000012F0B0F88DED050ACDED060A9DF86C302B
:10971000073B022B15D80B950C950D9511F0DCFC31
:109720000BA910F019FB0028BDD00BA905A82BF040
:10973000D1FDDDED077A9DED0D7A77EEC77ACDED9F
:10974000077A089509950A95B9F1000F1CD1DDED4E
:10975000147A129B0893F1EE677A139B099308A978
:109760005046CDED0A7AFFF723FD00289BD09DF8E7
:109770006C30083B012B07D8424808A912F05EF86C
:109780008DED080ACDED090A0B950C950D95B7B92D
:10979000159B0B93169B0C939DF86C30DDED177A9F
:1097A000083BF1EE677A012BCDED0D7A07D83548ED
:1097B0000BA912F043F88DED0B0ACDED0C0A0EBB90
:1097C0009DF86C309DED180A083B012B8CBF0023DF
:1097D0000123DCB9DDED190AB8F1000F19D1B9F197
:1097E000000F3AD1B4FA84F4B6FA86F66409760921
:1097F0000293019400960BAB08AA05A9204809F032
:1098000053FA54E79FED200A0023E2E7DFED1E0A3A
:10981000E2E7B9F1000F0FD10122B4FA84F4CDE9E7
:1098200001326409B6FA86F3154800945B090BAA65
:1098300008A909F0FDFC3AE7002F7FF434AF0122BC
:10984000CDE90032B4FA84F3B6FA86F20C485B092B
:1098500052090BA909F090FC29E7002F3FF423AF30
:10986000CDE90038B6FA86F2B4FA84F35B095209FE
:1098700005A9034809F0A2FA19E700BFF05B002030
:10988000AC850020103F0020000000002DE9F047CB
:10989000A2B08046084614A9FEF786FE6D4B5868B4
:1098A00003685B6A984760B1BDF88040A30504F087
:1098B000070904F4E07707D537B96748012109F0B3
:1098C00077F822B0BDE8F0870CAE304617F076FC92
:1098D000B9F1000F23D1DDE9150129F00FFF0028B0
:1098E000EBD09DF8841009AA404657F03DFB0028B4
:1098F000E3D0DDED177A9FED597A099B009367EE6F
:10990000877A10ADFDEEE77ADDE9151217EE903A91
:10991000284617F071FC95E80F0086E80F00002537
:1099200014F0380A0695079508950FD1DDED1A7ADF
:10993000189B0693F1EE677A199B079306A9404698
:10994000CDED087AFFF734FC0028B6D009950A95CA
:109950000B954FB9DDED1D7A1B9B0993F1EE677AEC
:109960001C9B0A93CDED0B7A14F480680CBF9DED1F
:109970001E0A9FED3B0A14F400640CBFDDED1F0AC4
:10998000DFED370AB9F1000F30D1BAF1000F51D134
:109990003046CDED050A8DED040A17F053FC03287F
:1099A0009DED040ADDED050A87D010A93046CDED06
:1099B000050A8DED040A10951195129517F03CFEDD
:1099C00000283FF47AAFB4FA84F46409B8FA88F353
:1099D000DDED050A9DED040ACDF804A000945B09B5
:1099E00006AA10A91C4809F0D7F96AE7BAF1000FD6
:1099F0000FD10123B4FA84F4CDE901A36409B8FAC4
:109A000088F3154800945B0909AA06A909F010FC1F
:109A100057E7002F7FF451AF0123CDE90073B8FA67
:109A200088F2B4FA84F30C485B09520909A909F0D9
:109A3000A3FB46E7002F3FF440AFB4FA84F3B8FA33
:109A400088F2CDF800905B0952093146024809F0CE
:109A500089FA36E7F05B0020AC8500200000C842A0
:109A60000000000030B48D7A4B7A43EA0523CD7AAA
:109A700043EA0543562B04460A461BD008D8522B0E
:109A800012D0542B13D02046114630BC57F08ABB5D
:109A900003F18073863B23F07F43012BF3D8017CD5
:109AA000064830BC4AF01ABE30BCFFF73DBD30BCA2
:109AB000FFF7E4BD30BCFFF7E9BE00BFAC77002084
:109AC0002DE9F0412DED028B044690B000F5974052
:109AD0000023012269463C3000934BF091FB08B90A
:109AE0004B4B009304F5405804F58045D8F804002A
:109AF00003685B699847002840F08580D5F8943A60
:109B0000D3F8CC7293EDBC8A04F536560C3601A915
:109B100030460EF07DFB18B94EF04AF93C4B0193EC
:109B20003722002102A8F6F7C5FCA3238DF80830E0
:109B300095238DF8093087F05BF9D5F88C3ACDF88C
:109B40000B00D8F82800D3F8DC20D3F8E030CDF8AB
:109B50000F104430CDF81320CDF8173050F0DCFA58
:109B60000346DFED2C0A93ED000AB7EE001A9B20A6
:109B700028F050FD10EE103AD8F82800CDF81B3030
:109B800003685B69984710EE103ACDF81F30D5F89E
:109B9000943ACDF82370D3F8B432CDF8273005F6D7
:109BA000582330461B68CDF82B30019BCDF82F3061
:109BB0000EF04AFB9FED187A28EE078A10EE103A55
:109BC000BDEEC88ACDF83330009BCDF8373018EEA3
:109BD000103AADF83B30D5F8943AD3EDB67A67EE4B
:109BE000877A04F58150FDEEE77A372217EE903A36
:109BF00002A91830ADF83D304DF0DAF810B0BDECE8
:109C0000028BBDE8F0819FED038A18EE107A7BE7A6
:109C10002292CA7F000000000000C84200F5804088
:109C2000D0F88C0A77F0A6BB00F58040D0F8941AE3
:109C3000D0F88C0A77F004BC70B54FF4805105461B
:109C40000EF00CFC00284ED005F5804605F5815439
:109C5000D6F88C0A03689B689847183400F1940280
:109C6000672120464CF030FFD6F88C0A0368DB6889
:109C70009847682100F1940220464CF025FFD6F861
:109C80008C0A03681B699847692100F194022046F9
:109C90004CF01AFFD6F8942A6A21204602F5027287
:109CA0004CF012FF202128460EF0D8FBD8B105F564
:109CB0004053586803681B69984778B1D6F8942ACE
:109CC000204688326C214CF0FFFED6F8942A2046BC
:109CD000B432BDE870406D214CF0F6BE28460AF063
:109CE00045F80028EAD170BD08B511F0F5F9BDE8D6
:109CF000084010F05BBF00007FB50E464FF6FF71C5
:109D0000044615460EF0AAFBE8B110220021684671
:109D1000F6F7D0FBA3238DF8003095238DF80130A2
:109D200003238DF8023087F063F8CDF8030004F5C3
:109D30008150CDF807101022694618308DF80B605D
:109D400003954DF0B5F804B070BD00007FB50E4628
:109D50004FF6FF71044615460EF080FBE8B1102265
:109D600000216846F6F7A6FBA3238DF80030952363
:109D70008DF8013004238DF8023087F039F8CDF8E2
:109D8000030004F58150CDF8071010226946183001
:109D90008DF80B6003954DF08BF804B070BD00009A
:109DA00030B52DED048B89B004460D461C220021F0
:109DB00001A8F0EE409AB0EE609AF0EE418AB0EE63
:109DC000618AF6F777FBA3238DF8043095238DF88D
:109DD000053006238DF8063087F00AF8CDF8070025
:109DE00004F58150CDF80B101C2201A918308DF814
:109DF0000F50CDED049A8DED059ACDED068A8DEDCF
:109E0000078A4CF0D5FF09B0BDEC048B30BD0000D3
:109E100010B54FF4801104460EF020FB28B104F574
:109E20009950BDE810400FF0F1BC10BD2DE9F04392
:109E30008FB01446054689463122002101A8DDE98C
:109E400016769846F6F736FBA3238DF80430952353
:109E50008DF8053008238DF8063086F0C9FF236899
:109E6000049363680593A36806933B68CDF81D309F
:109E70007B68CDF82130BB68CDF825303368CDF84C
:109E80000700CDF8293005F581507368CDF80B1027
:109E9000CDF82D303122B3688DF80F9001A918301C
:109EA0008DF81C80CDF831304CF082FF0FB0BDE84A
:109EB000F083000070B52DED068B8CB0144605467E
:109EC0000E462C22002101A8B0EE409AF0EE608AE6
:109ED000B0EE418AB0EE61AAF0EE429AF6F7EAFAE5
:109EE000A3238DF8043095238DF805300B238DF8CE
:109EF000063086F07DFFDFED1A7A94ED007ACDF81A
:109F0000070027EE277A29EE279A8DED077A94ED40
:109F1000017ACDF80B1027EE277A68EEA78A8DED2F
:109F2000087A94ED027A8DF80F6028EE278A05F5FD
:109F3000815067EE277A2C2201A918308DED049A02
:109F4000CDED058A8DED068ACDED097A8DED0AAA53
:109F5000CDED0B9A4CF02CFF0CB0BDEC068B70BD18
:109F6000E02E65422DE9F04188B080461B22002199
:109F700001A810EE107A10EE906A11EE105A11EE50
:109F8000904AF6F797FAA3238DF8043095238DF8BD
:109F900005300C238DF8063086F02AFFCDF8070037
:109FA00008F58150CDF80B101B2201A91830CDF80F
:109FB0000F70CDF81360CDF81750CDF81B404CF062
:109FC000F7FE08B0BDE8F0819E20704730B5144B15
:109FD000044689B004F58155986A694618351E22F1
:109FE0007FF0DAFA6A460F4928464DF07DF804F50D
:109FF0004053586803681B68984704F500530146AE
:10A0000093F8242328464DF093F804F5995011F065
:10A010002DFC04F5907020F0E3F809B030BD00BFCE
:10A02000F05B002032BE0C08112370B503712A4B7F
:10A03000836000238361C36103620364274A284B62
:10A04000826343644FF08042264B83640446C263BC
:10A05000583058F03BFF244E244BA36580256019EF
:10A0600059F040F966513035B5F5607FF7D104F508
:10A0700061705AF083FD002104F28C7081F0B2FE11
:10A080001B4BC4F840389FED1B1ADFED1B0A9FEDF8
:10A090001B0A04F6540077F09BFF9FED161A9FED04
:10A0A000180AF0EE410A04F66C0077F091FF9FED7C
:10A0B000111A9FED130AF0EE410A04F6840077F0BE
:10A0C00087FF20460F4947F00FF920460E4947F019
:10A0D0000BF9204670BD00BF303800200000C84199
:10A0E0000AD7233C0000E04090BB0C08A4BB0C083E
:10A0F00008830020000000009A99993E0000B443B4
:10A1000000804A433CAF0C088CB10C0830B500F518
:10A110000D5193B00446782228314BF05BFA04F5D8
:10A120000D50B7EE000A00220221383046F0DEFC66
:10A130000125002304F50651CDE90053284A3031AA
:10A14000452046F02FFC274A002304F50B51CDE9AA
:10A150000055FA2046F026FC234A1368D90705D497
:10A160002249156004F5045330330B6004F50F5099
:10A170001E490122203046F083FC0125002304F50E
:10A180008151CDE900531A4A1831FD2046F00AFCEE
:10A19000184B1A68D20705D4174A1D6004F58D5470
:10A1A00004341460154D1448012146F085FC0FCD90
:10A1B00002AC0FC40FCD0FC40FCD0FC495E80F0034
:10A1C00084E80F000022042102A846F0E7FB47F0D4
:10A1D00091FA0B4A138843F00103138013B030BD8A
:10A1E00064000E08047B0D080C890020D823002091
:10A1F00018570D0810890020E4230020FC5F0C088C
:10A20000608B002070B52A4C064694E80F00A4B07D
:10A210006D4685E80F00B7EE000A0021284646F09B
:10A2200011FB96F97469D6B910340FCC0CAD0FC57B
:10A230000FCC0FC50FCC0FC594E80F0085E80F00B9
:10A24000324604210CA846F0A9FB9FED1A0A1A48D1
:10A2500047F0F2FB1948B7EE000A47F0EDFB184C47
:10A260009FED180A0FCC04AD0FC594E80F0085E8E8
:10A270000F00002104A846F0E5FA9FED120A002124
:10A28000284646F0DFFA04F1100160220CA8F5F729
:10A2900029FE00240CAB18190021B7EE000A103477
:10A2A00046F0D0FA602CF5D15AF078FA24B070BD9F
:10A2B0003C600C08000000001CAF0C082BAF0C0821
:10A2C0008C600C08000034420F299DBF302303FB33
:10A2D0000100283000207047014B93F9AB03704711
:10A2E000F04B0020024B587F00F00100704700BF88
:10A2F000F05B0020044BB3F87033DB075ABF0069F2
:10A30000C0F3401000207047F04B0020014BD3F801
:10A31000E00C7047F04B002038B50D1E2DDB174CBC
:10A3200094F8F02CEBB29A4227D3D4F8EC3C0122FB
:10A33000595DA4F5005004F05DF8F0B158F096FFB7
:10A34000032159F0C7FFC0B958F090FF0D2159F013
:10A35000C1FF90B994F99033EB40DB075CBF94F9EF
:10A36000AA13E940A4F5005048BF0221BDE83840D7
:10A3700058BF01F00101FCF773BE38BDF04B00205F
:10A38000022A10B50C4605D1BDE810400848352218
:10A3900004F030B8074B586803681B689847A04220
:10A3A00005D158F063FFBDE8104058F063BE10BD02
:10A3B000F02B0020F05B002029B1022907D1044BCB
:10A3C000C3F8FC1F7047024B0122C3F8FC2F7047F3
:10A3D000F04B002029B1022905D1034B01221A704C
:10A3E0007047014B19707047F05B002010B52DEDE0
:10A3F000048B90F828330446F3B19FED1B8A0023A9
:10A4000080F82833F0EE488A10F066FEF0EE480A35
:10A41000B0EE680A012111F069F84DF0C9FC26215F
:10A420004DF05EFA57F0EEFBBDEC048B0F4ABDE831
:10A430001040062152F096BA58F06CFEB0F90A307E
:10A440009FED0B9A204608EE903A58F06DFEB0F959
:10A450000A3008EE103AF8EEE88AB8EEC88A68EEDC
:10A46000898A28EE098ACFE70000000024B90C0889
:10A47000D402373910B50446D9B1022918D1124B8C
:10A48000586803681B6B984738B957F0BBFBBDE8A9
:10A4900010400E4A062152F065BA57F0B3FB0C4A41
:10A4A000062152F05FFA0B4A0123137284F8283315
:10A4B00010BD90F82833002BFAD0064B1972BDE876
:10A4C0001040FFF793BF00BFF05B002030B90C08CD
:10A4D00052B90C08D58A002008B5064A002380F836
:10A4E0002833137257F08EFBBDE80840024A06215C
:10A4F00052F038BAD58A002064B90C0873B590F8C8
:10A50000283305469BB31B4C606803681B6B984758
:10A5100028B9284602B0BDE87040FFF7DDBF14F847
:10A52000126C36B157F06EFB134A042152F01AFA3E
:10A53000EFE704F58054F3EE047AD4F88C3A93ED07
:10A540001B7A87EE270A93ED1C7A8DED010AC7EE80
:10A55000270ACDED000A10F0BFFDDDED000A9DEDEC
